:020000040800F2
:1000000000000120A9DA0308F5DA0308F90801085D
:10001000F5DA0308F5DA0308F5DA03080000000052
:10002000000000000000000000000000F5DA0308F6
:10003000F5DA030800000000F5DA0308BD1B01082B
:10004000F5DA0308F5DA0308F5DA0308F5DA030848
:10005000F5DA0308F5DA0308B9200108E5210108FB
:10006000A92101086D2101083121010845B60008C8
:1000700035B6000825B6000815B6000805B6000814
:10008000F1B50008DDB50008F5DA0308F5DA030874
:10009000F5DA0308F5DA0308F5DA0308F5200108B4
:1000A000F5DA0308F5DA0308F5DA0308F5DA0308E8
:1000B000F5DA030895AA0008F5DA0308F5DA03086B
:1000C000F5DA0308F5DA0308F5DA0308F5DA0308C8
:1000D000F5DA0308F5A00008E9A00008DDA0000893
:1000E0007D200108F5DA0308F5DA0308F5DA0308DC
:1000F00081AA0008F5DA030871AA0008C9B500084A
:10010000F5DA0308F5DA030885AA0008F5DA03082A
:10011000D1A00008C5A00008F5DA030895C50308BA
:10012000B5B50008A1B500088DB5000879B500087F
:1001300065B500080000000000000000000000009D
:1001400000000000000000000000000095B8020858
:1001500051B500083DB5000829B50008F5DA0308D7
:10016000F5DA0308F5DA0308F5DA0308F5DA030827
:10017000F5DA0308F5DA03080000000000000000CB
:10018000F5DA0308F5DA0308F5DA0308F5DA030807
:10019000F5DA0308F5DA030800000000F5DA0308D1
:1001A000000000000000000000000000F5DA030875
:1001B000F5DA0308F5DA030800000000000000008B
:1001C000000000000000000000000000000000002F
:1001D000000000000000000000000000F5DA030845
:0801E000E8D503000100000056
:1001E8000C020100D8240120D424012000000000C2
:1001F80048060008160008009C2D0120B42D012097
:10020800000000004A06000827000400642F0120AF
:10021800D02F012000000000520600080101040050
:1002280014300120B04D0120000000000000000043
:1002380008020C00664D0120B44D012000000000AA
:10024800BD0F010802000C00744D0120C04D0120B3
:100258000000000000000000F7010600604D0120CA
:10026800CC4D0120000000005606000803123300A0
:100278005B53012028530120000000005C060008A1
:1002880025005A0054520120AE52012000000000FF
:1002980000000000F6110C00A85101209C5101201B
:1002A800000000009006000815007000BC500120F6
:1002B8002C51012000000000000000002A0060000E
:1002C800FC4F01205C50012000000000CDF1020825
:1002D8002C001000085301201853012000000000D2
:1002E800FD1802082B002400B25301208E53012070
:1002F80000000000CD18020829005000B451012068
:100308000452012000000000000000000510060053
:1003180022570120A0570120000000009C06000879
:100328000C002400EA560120A85701200000000014
:100338009DE501080E20EA00DE550120CC5701207A
:100348000000000041F20208130004005057012089
:10035800B858012000000000A406000802010300AC
:10036800C9550120BC58012000000000C5E501085E
:10037800F5216C00FE540120C05801200000000047
:10038800A5B9000803000100E05A0120E85A01203D
:10039800000000000000000022000C00845E012024
:1003A800606C012000000000A80600081B00F40093
:1003B800F45A01206C6C0120000000001989020821
:1003C80026000E00706D0120606D01200000000005
:1003D800097C02081400020060710120BC71012030
:1003E80000000000B40600080E020200A8700120F8
:1003F800C071012000000000B606000810000300CC
:10040800F0700120C471012000000000B806000847
:1004180028001000E0700120C871012000000000D1
:10042800699A020823001000D0700120D8710120B9
:10043800000000009D48030819000500C87001204D
:10044800E871012000000000BC060008F811010056
:10045800C4700120F071012000000000C2060008ED
:1004680000010400C0700120F471012000000000A8
:10047800C40600082F001100AC700120F87101209B
:1004880000000000C8060008010205002C740120C5
:1004980070760120000000009DC7020800020500D8
:1004A8000C72012078760120000000000000000096
:1004B8001E00040034740120807601200000000032
:1004C800DA0600080B201000F4780120407A012099
:1004D80000000000DE06000801200800348001202A
:1004E8005480012000000000EE0600081A000800F1
:1004F8001C8001205C80012000000000F606000836
:100508001F000E00DC810120FC810120000000009A
:10051800FE06000805020100C48101200C820120AA
:10052800000000000C07000803010A003C810120BC
:1005380010820120000000000E07000818102C008F
:10054800AC8F01200C90012000000000911B0208D4
:100558000D003400D88F01203890012000000000E1
:1005680009E6010802020300048901206C900120B9
:100578000000000000000000FB010100109E0120A7
:10058800D49E012000000000F50E0108FC010900BE
:10059800DC9C0120D89E012000000000C10E01084B
:1005A8000A101200B09C0120E49E01200000000007
:1005B800180700083400100000940120F89E01205C
:1005C80000000000F5F1020812200C00149F012021
:1005D800089F0120000000002A070008040080008E
:1005E800FCA1012040B5012000000000000000002F
:1005F800F9010400509F0120C0B50120000000004F
:10060800AD0F0108FD011E00309F0120C4B5012077
:1006180000000000390F010806001600D0A30120D1
:10062800E4B501200000000061F202080A020A0095
:10063800CCB60120DCB60120000000003607000817
:100648000100C40900001901282820030000120134
:100658000000000000000000000000000000000092
:100668000000000000000000000000000000000082
:100678000000000000000000000000000000000072
:100688000000000000000100000000000000000061
:1006980000000000200003010000000018200000F6
:1006A800C800141E010064002C012800030000008B
:1006B800000105000000280100000400900100006E
:1006C8000000000000000000000000000000000022
:1006D8000000000001002B21231E6400020000001E
:1006E80001000A012900E8036400040A00017E05EC
:1006F800EA05B40532000000000000000100000017
:10070800000500000000040101006C160000000054
:1007180000300100005A0000000090012C01C800C0
:100728006400000000010005415746370000000042
:080738004A01B400D6010000E3
:1007400001010000FFFFFFFFFF00000001010000AA
:10075000982B040830670408000000000000000027
:10076000A82B0408B02B04080000000001200000A2
:10077000B42B0408BC2B040800000000014000005A
:10078000C02B0408043F0408000000000120000002
:10079000CC2B0408D82B0408000000000400000043
:1007A000DC2B040838580408000000000400000096
:1007B000E82B0408A4570408000000000100000012
:1007C000020100000000803F0000803FBCFC0308E5
:1007D000050804000000000090160408501D0408DD
:1007E0007C16040800000000E8FC030805080A0065
:1007F0000000000090160408501D04089C15040811
:1008000000000000FFFFFFFF010101007D39020829
:100810000000000040020120086104080000000000
:100820000000000000000000000000003067040825
:100830000000000000000000C802012004000000C9
:10084000B46004080D00000099410208801A0120DC
:1008500000000000E85A04080D000000C141020831
:10086000741A012000000000E85B04080800000082
:1008700000000000681A012004000000545B040816
:100880000D000000253A02085C1A0120000000005B
:10089000F85B0408030000009DAE0308501A012015
:1008A0000000000018610408030000009DAE03086A
:1008B000441A0120000000005C58040801000000F8
:1008C0000000000000000000000000000000000028
:1008D0000E0000000000000000000000000000000A
:1008E0000861040800000000000000000000000093
:1008F0000000000030670408000000000000000055
:10090000C802012004000000606004080300000029
:10091000593F0208381A012008000000545B0408FF
:100920000D000000253A02085C1A012000000000BA
:10093000F85B0408030000009DAE0308501A012074
:100940000000000018610408030000009DAE0308C9
:10095000441A0120000000005C5804080100000057
:100960000000000000000000000000000000000087
:100970000E00000000000000000000000000000069
:1009800020610408000000000000000000000000DA
:1009900000000000306704080000000000000000B4
:1009A000C802012004000000686004080300000081
:1009B0009DAE03088C1A0120000000005C5804085A
:1009C0000100000000000000000000000000000026
:1009D000000000000E000000000000000000000009
:1009E0000000000020700020702D72000000000048
:1009F00000000000F4150120FFFFFFFFFA000000D7
:100A000001000000010000002D202D2D202D2D2D96
:100A10002D202D2D2D000000000000000000000002
:100A200000000000000000002058040828580408B6
:100A300054580408000000000000000000000000FE
:100A4000000000000C58040804000000D13E020819
:100A500000000000000000005C58040801000000D5
:100A60000000000000000000000000000000000086
:100A70000E00000000000000000000000000000068
:100A8000DA5C01200100C40900000000D85C0120EC
:100A90000100C40900000000D65C01200100C40967
:100AA00000000000D45C01200100C4090000000027
:100AB000D05C01200100C40900000000D25C0120CC
:100AC0000100C40900000000CE5C01200100C4093F
:100AD00000000000CC5C01200100C40900000000FF
:100AE000745501200100C80001000000725501206A
:100AF000320030753200000070550120055A0500A3
:100B00006B55012000FF01006F550120010000001E
:100B1000E80201206D550120020000009015040834
:100B20006A55012000FF01006E5501200100000000
:100B3000E80201206C550120020000009015040815
:100B40000000000000000000F00201208081012070
:100B50009CFF2C0100000000C80001200A000000DA
:100B60009C150408F0540120E0150C17000000004B
:100B7000CA00012008000000501D0408C90001201F
:100B80000500000090160408F25401200200000045
:100B9000B4150408285701200100FF7F0100000060
:100BA0002157012002000000C0150408D255012081
:100BB00003000000D0150408D155012003000000F7
:100BC000D0150408D05601200000F40101000000F7
:100BD000CE5601200000F40101000000CC56012097
:100BE0000000F40101000000CA5601200000F401D9
:100BF00001000000C856012000FF0100E856012056
:100C0000E803D0070A000000E65601200064010056
:100C10000A000000E256012000640100E1560120B4
:100C200000640100E7560120006401000A00000092
:100C3000E0560120006401000A000000E556012092
:100C4000006401000A000000E45601200064010075
:100C50000A000000E3560120006401000A000000C1
:100C6000DF56012000FF01000A000000DE560120CF
:100C700000FF01000A000000DA5501200000F40125
:100C800001000000D85501200000F401010000001F
:100C9000D65501200000F40101000000D4550120C8
:100CA0000000F40101000000DA5601201400E803FE
:100CB00001000000D8560120E80330750100000053
:100CC000D756012000C80100D656012000C80100F7
:100CD000D556012000C80100D4560120006401004F
:100CE0000A000000D356012000FF01000A000000A6
:100CF0001757012000C801001657012000C8010045
:100D00001557012000C801001457012000C8010038
:100D10001357012000C801001257012000C801002C
:100D20001157012000C801001057012000C8010020
:100D30000F57012000C80100885804080000000077
:100D400000000000000000000000000098580408A7
:100D500009000000000000009403012004000000CE
:100D6000A0580408090000000000000088030120CA
:100D7000040000002C5E04080900000000000000D0
:100D80007C030120040000009C2A040809000000E4
:100D9000000000007003012004000000A8580408AF
:100DA00009000000000000006403012004000000AE
:100DB000B05804080900000000000000580301209A
:100DC00004000000B85804080900000000000000FA
:100DD0004C03012004000000C05804080900000072
:100DE0000000000040030120040000005C580408DB
:100DF00001000000000000000000000000000000F2
:100E0000000000000E0000000000000000000000D4
:100E100000000000D4590408000000000000000099
:100E20000000000000000000884E040807000000D9
:100E300000000000B803012000000000E45904088D
:100E40000800000000000000AC03012000000000CA
:100E5000F05904080800000000000000A003012071
:100E6000000000005C5804080100000000000000C1
:100E70000000000000000000000000000E00000064
:100E8000000000000000000000000000F859040805
:100E90000000000000000000000000000000000052
:100EA000085A04080D00000000000000F4030120AF
:100EB00000000000105A04080D00000000000000AF
:100EC000E803012000000000185A04080700000091
:100ED00000000000E003012000000000205A040888
:100EE0000D00000000000000D403012000000000FD
:100EF000285A04080D00000000000000C80301206B
:100F000000000000305A0408070000000000000044
:100F1000C0030120000000005C580408010000002C
:100F200000000000000000000000000000000000C1
:100F30000E000000000000000000000000000000A3
:100F4000385A040800000000000000000000000003
:100F500000000000884E04080C00000000000000A3
:100F600076550120000000004C5A04080C000000D7
:100F70000000000078550120000000005C5A0408C1
:100F80000C00000000000000AE5501200000000031
:100F90006C5A04080C00000000000000A25501205B
:100FA00000000000805A04080C000000000000004F
:100FB0007A550120000000008C5A04080C00000043
:100FC000000000007C55012000000000945A040835
:100FD0000C000000000000007E5501200000000011
:100FE000A85A04080C0000000000000080550120F1
:100FF00000000000B05A04080C00000000000000CF
:101000008255012000000000B85A04080C000000BE
:1010100000000000C055012000000000D05A040864
:101020000C000000000000008455012000000000BA
:10103000DC5A04080C000000000000008655012066
:1010400000000000A84904080C0000000000000097
:101050008855012000000000E45A04080C0000003C
:10106000000000008A55012000000000F05A04082A
:101070000C000000000000008C5501200000000062
:10108000FC5A04080C000000000000008E550120EE
:1010900000000000085B04080C00000000000000D5
:1010A0009055012000000000145B04080C000000B3
:1010B000000000009255012000000000205B0408A1
:1010C0000C00000000000000A655012000000000F8
:1010D000285B04080C00000000000000A45501205B
:1010E00000000000305B04080C000000000000005D
:1010F000B2550120000000003C5B04080C00000019
:1011000000000000B455012000000000485B040806
:101110000C00000000000000BA5501200000000093
:101120006C5904080C0000000000000094550120D8
:1011300000000000545B04080C00000000000000E8
:101140009C550120000000005C5B04080C000000BE
:10115000000000009655012000000000685B0408B4
:101160000C00000000000000985501200000000065
:10117000745B04080C000000000000009A55012078
:10118000000000007C5B04080C0000000000000070
:101190009E55012000000000A84E04080C0000002D
:1011A00000000000A855012000000000885B040832
:1011B0000C00000000000000A0550120000000000D
:1011C000945B04080C00000000000000B0550120F2
:1011D00000000000A05B04080C00000000000000FC
:1011E000AA55012000000000A85B04080C000000C4
:1011F00000000000AC55012000000000B05B0408B6
:101200000C00000000000000B655012000000000A6
:10121000B85B04080C00000000000000B855012075
:10122000000000005C5804080100000000000000FD
:101230000000000000000000000000000E000000A0
:10124000000000000000000000000000C05B040877
:10125000000000000000000000000000000000008E
:10126000D05B04080500000000000000D0550120FC
:10127000000000005C5804080100000000000000AD
:101280000000000000000000000000000E00000050
:10129000000000000000000000000000D85B04080F
:1012A000000000000000000000000000000000003E
:1012B00030670408000000000000000053200120F7
:1012C00004000000E45B04080D000000353F020844
:1012D0004804012000000000B46004080D00000074
:1012E000353902083C04012000000000E85A0408D7
:1012F0000D00000019390208300401200000000030
:10130000E85B04080800000000000000240401203D
:1013100004000000545B04080D000000653802085A
:101320001804012000000000F05B04080900000020
:10133000000000000C04012004000000F85B040819
:10134000030000009DAE030800040120000000001F
:101350005C580408010000000000000000000000CC
:1013600000000000000000000E000000000000006F
:101370000000000000000000FC5B0408000000000A
:101380000000000000000000000000000C5C0408E9
:101390000D000000000000006004012000000000BB
:1013A000145C04080A00000000000000345701200B
:1013B00000000000205C04080A000000000000009B
:1013C0003C57012000000000285C04080A000000CF
:1013D000000000004457012000000000305C0408B9
:1013E000080000000000000054040120000000007C
:1013F0005C5804080100000000000000000000002C
:1014000000000000000000000E00000000000000CE
:101410000000000000000000385C0408000000002C
:101420000000000000000000000000004C5C040808
:101430000D00000000000000780401200000000002
:101440005C5C0408040000003D420208000000004B
:1014500000000000645C04080D00000000000000B3
:101460006C04012000000000785C04080400000007
:101470001942020800000000000000005C58040847
:10148000010000000000000000000000000000005B
:10149000000000000E00000000000000000000003E
:1014A00000000000805C0408000000000000000054
:1014B0000000000000000000945C04080700000029
:1014C00000000000B404012000000000A05C04083B
:1014D0000800000000000000A80401200000000037
:1014E000AC5C040808000000000000009C0401201F
:1014F00000000000B85C04080800000000000000C4
:101500009004012000000000C45C040808000000F2
:101510000000000084040120000000005C58040862
:1015200001000000000000000000000000000000BA
:10153000000000000E00000000000000000000009D
:1015400000000000D05C0408000000000000000063
:10155000A702012000000000C82904080B000000B9
:10156000000000002C05012000000000DC5C0408E5
:101570000B0000000000000020050120000000001A
:10158000E85C04080B0000000000000014050120C6
:1015900000000000F45C04080B00000000000000E4
:1015A0000805012000000000005D04080B00000099
:1015B00000000000FC04012000000000D029040805
:1015C0000B00000000000000F004012000000000FB
:1015D0000C5D04080B00000000000000E404012082
:1015E00000000000185D0408070000000000000073
:1015F000DC04012000000000205D0408070000005A
:1016000000000000D4040120000000002C5D04084C
:101610000B00000000000000C804012000000000D2
:10162000385D04080800000000000000BC04012030
:10163000000000005C5804080100000000000000E9
:101640000000000000000000000000000E0000008C
:10165000000000000000000000000000445D0408DD
:10166000000000000000000000000000000000007A
:10167000585D040808000000000000005C0501201F
:1016800000000000645D0408080000000000000085
:101690005005012000000000705D040808000000F3
:1016A0000000000044050120000000007C5D0408EB
:1016B00008000000000000003805012000000000C4
:1016C0005C58040801000000000000000000000059
:1016D00000000000000000000E00000000000000FC
:1016E0000000000000000000845D0408000000000D
:1016F00000000000A402012000000000945D040826
:101700000B00000000000000A40501200000000004
:10171000A05D04080B0000000000000098050120F7
:1017200000000000AC5D040807000000000000009D
:101730009005012000000000B85D040807000000CB
:10174000000000008805012000000000C45D0408BE
:1017500007000000000000008005012000000000DC
:10176000D05D04080800000000000000740501209E
:1017700000000000D85D0408080000000000000020
:1017800068050120000000005C580408010000000A
:101790000000000000000000000000000000000049
:1017A0000E0000000000000000000000000000002B
:1017B000E05D04080000000000000000A402012019
:1017C00000000000EC5D04080700000000000000BD
:1017D000F005012000000000F45D0408070000008F
:1017E00000000000E805012000000000FC5D040886
:1017F0000700000000000000E005012000000000DC
:10180000642A04080700000000000000D805012039
:10181000000000006C2A040807000000000000001F
:10182000D005012000000000742A04080700000011
:1018300000000000C805012000000000045E04084C
:101840000700000000000000C005012000000000AB
:101850000C5E04080700000000000000B80501202D
:1018600000000000145E04080700000000000000F3
:10187000B0050120000000005C58040801000000D1
:101880000000000000000000000000000000000058
:101890000E0000000000000000000000000000003A
:1018A00000000000093C0208F8050120CE55012087
:1018B0001B000000E0150408CD5501200A3201008C
:1018C000CC55012001FA0100C855012000C80100D3
:1018D000C6550120E803D00701000000414C4945EE
:1018E0004E57484F4F50463700000000FC5401202F
:1018F00000030100FB540120000301002D3B0208FE
:10190000093B0208D4060120C93A0208813A0208BC
:101910004C070120693B0208513B020800080120E6
:101920001F3C0208E94102080C0B0120A138020803
:10193000000000005C0B0120993F02088D3E020868
:10194000380C0120453C020800000000D80C0120A2
:10195000E93C0208B93C0208640D0120753D02080B
:10196000BD3D0208040E0120DC56012001030100E8
:10197000853C0208593C02081C0F0120193D020851
:1019800061420208A80F0120E93D0208BD42020899
:1019900070100120D2560120010301001C5E0408D2
:1019A0000000000000000000000000000000000037
:1019B000285E0408080000000000000090110120CB
:1019C00000000000305E0408070000000000000076
:1019D0008811012000000000405E0408070000009C
:1019E0000000000080110120000000004C5E04088F
:1019F0000700000000000000781101200000000036
:101A0000585E04080D000000000000006C11012069
:101A100000000000645E0408030000009DAE03089F
:101A200060110120000000005C5804080100000063
:101A300000000000000000000000000000000000A6
:101A40000E00000000000000000000000000000088
:101A50006C5E0408000000000000000000000000B0
:101A6000000000007C5E04080A0000000000000086
:101A7000F42B040800000000845E04080A00000043
:101A800000000000782B0408000000008C5E0408B1
:101A90000A000000000000001857012000000000AC
:101AA000945E04080A000000000000009C11012060
:101AB000000000005C580408010000000000000065
:101AC0000000000000000000000000000E00000008
:101AD0000000000000000000000000009C5E040800
:101AE00000000000000000000000000000000000F6
:101AF000A85E0408030000009DAE0308D411012075
:101B000000000000B45E0408030000009DAE03085E
:101B1000C811012000000000BC5E040803000000A2
:101B20009DAE0308BC11012000000000C45E040843
:101B30000500000000000000FA5401200000000031
:101B4000CC5E04080700000000000000B411012072
:101B500000000000D85E040807000000000000003C
:101B6000AC110120000000005C58040801000000D6
:101B70000000000000000000000000000000000065
:101B80000E00000000000000000000000000000047
:101B9000E45E0408000000000000000000000000F7
:101BA00000000000F85E0408030000009DAE03087A
:101BB000F811012000000000045F04080300000089
:101BC0009DAE0308CC000120000000000C5F04085B
:101BD000030000009DAE0308EC110120000000008E
:101BE000145F0408030000009DAE0308E01101200B
:101BF000000000005C580408010000000000000024
:101C00000000000000000000000000000E000000C6
:101C1000000000000000000000000000205F040839
:101C200000000000000000000000000000000000B4
:101C30002C5F040807000000094302085412012029
:101C400000000000785B0408030000009DAE03085C
:101C50004812012000000000385F04080300000063
:101C60009DAE03083C12012000000000405F040804
:101C7000030000009DAE03083012012000000000A8
:101C8000485F040807000000ED4202082812012006
:101C900000000000F8290408030000009DAE0308BE
:101CA0001C12012000000000545F04080300000023
:101CB0009DAE03081012012000000000605F0408C0
:101CC000030000009DAE0308041201200000000084
:101CD0005C58040801000000000000000000000043
:101CE00000000000000000000E00000000000000E6
:101CF0000000000000000000C53B0208813B020814
:101D00005C120120593E020800000000101301205F
:101D1000653A0208493A02089C13012000000000BD
:101D20000000000050140120313E02082543020843
:101D3000DC1401206C5F04080000000000000000BB
:101D40000000000000000000785F040803000000AD
:101D50009DAE0308E815012000000000805F040824
:101D6000030000009DAE0308DC1501200000000008
:101D7000EC490408030000009DAE0308D0150120C3
:101D8000000000008C5F0408030000009DAE030803
:101D9000C415012000000000985F04080300000043
:101DA0009DAE0308B815012000000000A05F0408E4
:101DB0000200000041430208000000000000000093
:101DC000A85F04080200000041430208010000006F
:101DD00000000000B45F0408020000004143020854
:101DE0000200000000000000000000000E000000E3
:101DF000000000000000000000000000F654012078
:101E000088136F1701000000F854012088136F1722
:101E100000000000C05F0408000000000000000097
:101E20000000000000000000D05F0408080000006F
:101E300000000000C816012004000000DC5F040858
:101E40000800000000000000BC1601200000000097
:101E5000F85B040804000000ED3F020800000000E9
:101E6000000000005C5804080100000000000000B1
:101E70000000000000000000000000000E00000054
:101E8000000000000000000000000000F4540120E9
:101E900088136F1701000000BC81012088136F17A1
:101EA00000000000DD39020800000000D416012007
:101EB0004C5701200100000050160408BE8101208B
:101EC000010000005C160408B4810120020000003B
:101ED00064160408C2A201200000000000000000F7
:101EE000C0A201200000000000000000BEA20120EE
:101EF0000000000000000000BCA201200000000063
:101F000000000000BAA20120000000000000000054
:101F1000B8A2012000000000000000008C20012079
:101F20000000000000000000F35401200200000047
:101F3000701604081860040800000000000000008B
:101F40000000000000000000D05F0408080000004E
:101F5000000000005817012004000000DC5F0408A6
:101F600008000000000000004C17012000000000E5
:101F7000F85B040804000000B1390208000000000A
:101F8000000000005C580408010000000000000090
:101F90000000000000000000000000000E00000033
:101FA000000000000000000000000000286004089D
:101FB0000000000000000000000000000000000021
:101FC000386004080D0000003D4102088817012018
:101FD00004000000446004080D000000013A0208FB
:101FE0007C17012004000000506004080D00000070
:101FF0000141020870170120000000005C60040825
:1020000003000000793F0208641701200800000067
:1020100068600408030000009DAE03088C1A0120CC
:10202000000000005C5804080100000000000000EF
:102030000000000000000000000000000E00000092
:1020400000000000000000000000000054580408D8
:102050000000000000000000000000000000000080
:102060000C580408040000000940020800000000A9
:10207000000000005C58040801000000000000009F
:102080000000000000000000000000000E00000042
:10209000000000000000000000000000BC60040818
:1020A0000000000000000000000000000000000030
:1020B000605104080D00000000000000E817012036
:1020C00004000000CC6004080800000000000000CC
:1020D000DC17012004000000D8600408080000009C
:1020E00000000000D017012004000000E060040898
:1020F0000800000000000000C417012004000000D8
:10210000E86004080800000000000000B817012083
:1021100004000000F0600408080000000000000057
:10212000AC17012004000000F8600408080000005B
:1021300000000000A0170120040000000061040856
:1021400008000000000000009417012004000000B7
:102150005C580408010000000000000000000000BE
:1021600000000000000000000E0000000000000061
:102170000000000000000000C93902080000000053
:10218000F417012000000000000000006C1801207E
:1021900000000000000000000C190120BA8101209D
:1021A000040000007C160408B8810120E0150C171B
:1021B00000000000B781012008000000501D040845
:1021C000B681012005000000901604080000000000
:1021D000000000005C19012000000101FFFF000069
:1021E00000010101010000001A03000000000000CE
:1021F00000000000000000000000000000000000DF
:102200000000000004030904120100020200004063
:102210008304405700020102030100000A06000285
:10222000000000400100000009074300020104C053
:10223000320904000001020201000524001001051A
:10224000240100010424020205240600010705827E
:10225000030800FF09040100020A0000000705014D
:10226000024000000705810240000000090243000F
:10227000020100C03209040000010202010005242D
:1022800000100105240100010424020205240600B7
:10229000010705820308001009040100020A00007A
:1022A000000705010200020007058102000200008C
:1022B00009024300020100C03209040000010202C9
:1022C000010005240010010524010001042402027C
:1022D0000524060001070582030800100904010017
:1022E000020A000000070501024000000705810204
:1022F00040000000E0010800D44E04080000000087
:1023000000000000D9E50108A086010004000000DB
:1023100000000000000000000000000000000000BD
:10232000000000000000000000000000785B0408CE
:10233000004A040800000000C58301087D00000079
:102340000600000000000000000000000000000087
:10235000000000000000000000000000000000007D
:10236000346704080000000000000000210201089A
:10237000E80300000300000000000000000000006F
:10238000000000000000000000000000000000004D
:10239000000000003C67040800000000000000008E
:1023A000ADF3020810270000030000000000000049
:1023B000000000000000000000000000000000001D
:1023C0000000000000000000486704080000000052
:1023D000F152030879DB0008204E000005000000E0
:1023E00000000000000000000000000000000000ED
:1023F0000000000000000000000000006050040821
:10240000000000000000000059090108102700002A
:1024100001000000000000000000000000000000BB
:1024200000000000000000000000000000000000AC
:102430004C670408000000000000000045DB0008B5
:10244000E80300000500000000000000000000009C
:10245000000000000000000000000000000000007C
:1024600000000000586704080000000000000000A1
:1024700079E80108204E0000030000000000000081
:10248000000000000000000000000000000000004C
:102490000000000000000000686704080000000061
:1024A00000000000ADE60108204E0000030000001F
:1024B000000000000000000000000000000000001C
:1024C0000000000000000000000000007867040821
:1024D00000000000000000002D060108400D030070
:1024E00003000000000000000000000000000000E9
:1024F00000000000000000000000000000000000DC
:10250000984F04080000000000000000E9F30108F3
:102510001027000001000000000000000000000083
:1025200000000000000000000000000000000000AB
:10253000000000001C4A0408000000000000000029
:102540005DD4020810270000030000000000000016
:10255000000000000000000000000000000000007B
:102560000000000000000000886704080000000070
:10257000000000002D670108A08601000100000096
:10258000000000000000000000000000000000004B
:102590000000000000000000000000006850040877
:1025A0000000000000000000893B0108A00F0000AF
:1025B000010000000000000000000000000000001A
:1025C000000000000000000000000000000000000B
:1025D000906704080000000000000000E18202088B
:1025E00010270000010000000000000000000000B3
:1025F00000000000000000000000000000000000DB
:1026000000000000EC490408000000000000000089
:1026100005D400081A41000001000000000000007D
:1026200000000000000000000000000000000000AA
:102630000000000000000000CC5004080000000072
:1026400000000000C91A0308102700000100000064
:10265000000000000000000000000000000000007A
:10266000000000000000000000000000E84904082D
:102670000000000000000000E54402081A410000CC
:102680000100000000000000000000000000000049
:10269000000000000000000000000000000000003A
:1026A0009C67040800000000000000003DCA030809
:1026B000400D0300000000000000000000000000CA
:1026C000000000000000000000000000000000000A
:1026D00000000000A46704080000000000000000E3
:1026E000C9D10108400D03000000000000000000F7
:1026F00000000000000000000000000000000000DA
:102700000000000000000000AC67040800000000AA
:1027100000000000A5D80208A08601000300000008
:1027200000000000000000000000000000000000A9
:102730000000000000000000000000000000803FDA
:102740000000000000000000000000000000803FCA
:102750000000000000000000000000000000000079
:102760000000000000000000000000000000000069
:10277000000000000000803F00000000000000009A
:102780000000000000FFFF0000000000AA55050146
:102790000000012D202D2D202D2D2D2D202D2D2D16
:1027A0002D000000000000000000000000000000FC
:1027B0000000AA550B010000AA5507010000AA5508
:1027C000090200000000000001000000C012AA552C
:1027D00003009F0000E6DF0C01B70208F5B602080F
:1027E0005DB8020871B80208ADB6020849B802081F
:1027F00035B80208095D020889550208ADB702081C
:10280000000000003DB7020899B7020865B702084A
:1028100000000000000000000000000025B70208D2
:1028200031B7020819B702080DB702086BC40308D4
:1028300051C4030805C40308EDC303080101D60110
:10284000354E0308000000000000000001000000F9
:102850000000803F00600240106002400000000065
:10286000000B00000000200000000000000000003D
:10287000006002402860024000000000060C0000DA
:102880000000200000000000000000000060024086
:102890004060024000000000100D00000000200019
:1028A000000000000000000000600240586002408C
:1028B00000000000160E00000000200000000000D4
:1028C0000000000000600240706002400000000054
:1028D000200F0000000020000000000000000000A9
:1028E00000600240886002400000000026100000E6
:1028F0000000200000000000000000000060024016
:10290000A060024000000000301100000000200024
:10291000000000000000000000600240B8600240BB
:1029200000000000362F0000000020000000000022
:10293000000000000064024010640240000000003B
:10294000003800000000400000000000000000000F
:1029500000640240286402400000000006390000C4
:102960000000400000000000000000000064024081
:102970004064024000000000103A000000004000E7
:1029800000000000000000000064024058640240A3
:1029900000000000163B00000000400000000000A6
:1029A000000000000064024070640240000000006B
:1029B000203C00000000400000000000000000007B
:1029C00000640240886402400000000026440000C9
:1029D0000000400000000000000000000064024011
:1029E000A0640240000000003045000000004000EC
:1029F000000000000000000000640240B8640240D3
:102A0000000000003646000000004000000000000A
:102A1000000000000000803F0000000000000000F7
:102A20000000000000C201000000080001000000DA
:102A3000F42201200000000000000000000000005F
:102A40000000000000000000000000000000000086
:102A50000000000000000000000000000000000076
:102A60000000000000000000000000000000000066
:102A70000000000000000000000000000000000056
:102A80000000000000000000000000000000000046
:102A900000000000430000000000000000000000F3
:102AA0000000000000000000000000000000000026
:102AB00000000000430000000000000000000000D3
:102AC0000000000000000000000000000000000006
:102AD00000000000430000000000000000000000B3
:102AE00000000000000000000000000000000000E6
:102AF0000000000043000000000000000000000093
:102B000000000000000000000000000000000000C5
:102B10000000000043000000000000000000000072
:102B200000000000000000000000000000000000A5
:102B30000000000043000000000000000000000052
:102B40000000000000000000000000000000000085
:102B50000000000043000000000000000000000032
:102B60000000000000000000000000000000000065
:102B70000000000015E4030879E2030800000000EB
:102B8000BB69040808580408206804082068040881
:102B900020680408206804082068040820680408E5
:102BA000206804082068040820680408FFFFFFFF6D
:102BB000FFFFFFFFFFFFFFFFFFFF0000010041538A
:102BC0004349490000000000000000000000000030
:102BD0000000000000000000000000000000415361
:102BE0004349490000000000000000000000000010
:102BF00000000000000000000000000000000000D5
:042C000001000000CF
:108000004378007840EA032010FB01F04FF48071C0
:1080100090FBF1F000F30F0000B2704710B5064C72
:1080200023780BB9002010BD09F082FC6368C01AE8
:10803000D0F5FA50F6D410BDC82401204FF40063E7
:10804000038370474FF4006303837047012380F874
:1080500049307047D0F8F420034630B46AB1C168A3
:10806000D0F80C214469881A013A205C08BF0A46FE
:10807000C0B2C3F80C2130BC7047006A5D69411C76
:10808000DC68285CA14228BF1146C0B2196230BC2E
:108090007047D0F8F83013B190F88C017047836ABC
:1080A000406A181AB0FA80F040097047416A836A42
:1080B00099420ED3CB1AD0F8F810026981B1D0F8EA
:1080C0007811501E0A685268134483420BD2C01ABA
:1080D000704702691144CB1AD0F8F8100029EED18C
:1080E000501EC01A704700207047D0F8F4306BB1B2
:1080F000D0F87C31D0F80C211B685B68934201D327
:10810000981A7047C068801A18447047C269036A99
:108110009A4203D2C0681044C01A7047D01A704700
:10812000BFF34F8F0549064BCA6802F4E062134360
:10813000CB60BFF34F8F00BFFDE700BF00ED00E055
:108140000400FA058C4B1A78002A00F0EB808B496A
:1081500040F20D300B68F0B49F6C0026884C894DBE
:108160003C40AB4240EA04009864D86840F4807018
:10817000D8605E6200F0FA808348834200F0F680A7
:108180001868012A40F00100186000F0CA80D1F898
:10819000283140F20D307A4C00269F6C794D3C40DE
:1081A000AB4240EA04009864D86840F48070D8601C
:1081B0005E6200F0D6807448834200F0D280186876
:1081C000022A40F00100186000F0AB80D1F8503274
:1081D00040F20D306A4C00269F6C6A4D3C40AB4229
:1081E00040EA04009864D86840F48070D8605E6209
:1081F00000F0B2806448834200F0AE801868032A21
:1082000040F00100186000F08C80D1F8783340F223
:108210000D305B4C00269F6C5A4D3C40AB4240EA0F
:1082200004009864D86840F48070D8605E6200F002
:108230008E805548834200F08A801868042A40F0F6
:10824000010018606DD0D1F8A03440F20D304C4CD4
:1082500000269F6C4B4D3C40AB4240EA04009864C2
:10826000D86840F48070D8605E626BD04648834224
:1082700068D01868052A40F00100186051D0D1F884
:10828000C83540F20D303E4C00269F6C3D4D3C40C1
:10829000AB4240EA04009864D86840F48070D8602B
:1082A0005E624AD03848834247D01868062A40F0B8
:1082B0000100186035D0D1F8F03640F20D30304C66
:1082C00000269F6C2F4D3C40AB4240EA040098646E
:1082D000D86840F48070D8605E6229D02A48834212
:1082E00026D01868072A40F00100186019D0D1F88C
:1082F000183840F20D32224900249D6C2148294053
:10830000834242EA01029A64DA6842F48072DA60D7
:108310005C6208D01C4A934205D01A6842F0010200
:108320001A60F0BC70475A6C42F400425A64F4E799
:10833000586C40F400405864D3E7586C40F4004057
:108340005864B2E7586C40F40040586491E7586CA8
:1083500040F40040586470E7586C40F400405864A2
:108360004CE7586C40F40040586428E7586C40F4DF
:108370000040586404E700BFF8AB0120FCAB0120CB
:10838000E0E0FFFF0000014000040140F8B590F874
:10839000813190F88221134303F02103212B0FD068
:1083A000436A846AA3420CD802690023121B92B26A
:1083B00090F8811100258362202980F88C5103D028
:1083C000F8BD1A1B92B2F3E78369E34203EB0401A1
:1083D000F6D0B2FA82F46409002CF1D190F8803121
:1083E000012BEDD005460127A0F86A211346A0F81D
:1083F00068214FF0210ED0F87861C0F86411C0F800
:108400008441304685F880710C4A0D4F85F881E132
:10841000F76332640B4FD5F8182134652832F764BE
:1084200029F0AEFCD5F8183140221A6285F8804157
:108430009A6842F080029A60C2E700BF21520208A7
:108440005D520208B9510208426A10B48469A1540D
:10845000426A04690132D0F8F810A24228BF002213
:10846000426241B10B68DB0702D55DF8044B7047EF
:108470005DF8044B8AE7D0F818215DF8044B1368C7
:1084800043F080031360704738B504460D46FFF78C
:10849000C5FD246808B109F099FA054B002249216D
:1084A00020461A702A465B7809F0FAFE012038BD92
:1084B000C82401202DE9F0470569C3681D4028D074
:1084C0000F4606464FF000484FF00009B5FA85F315
:1084D00028FA03F21B3BD24332611540042B16D815
:1084E000DFE803F03129211903007B6A002B32D029
:1084F00003F1FF3AC7F824901FFA8AFA3C6A34B1B4
:1085000023682046514698476468002CF8D1002D16
:10851000DCD1BDE8F0873868716B036889B2984791
:10852000002DD3D1F5E77868B16B036889B298471D
:10853000002DCBD1EDE7B868F16B036889B298479D
:10854000002DC3D1E5E7F868316C036889B298471C
:10855000002DBBD1DDE7F36A1FFA83FACEE72DE9E0
:10856000F04F8BB090F859300290002B40F0A0856E
:10857000029A137C1032022B039204D110466B2115
:10858000802209F07DFF4FF0640AB44CB44D4FF0E7
:10859000100CDFF8D4924FF47A76B248DFF8CCE2D0
:1085A000D9F80430C3F30803002B40F07F84EFF3C5
:1085B0001183002B40F07A842168826800BF236811
:1085C0009942F9D12F6806FB07F39B1AB3FBF7F327
:1085D00006FB013101270191D9F80430C3F30803E8
:1085E000002B40F02884EFF31183002B40F023840C
:1085F0002368816800BF22689342F9D1D5F800B0A2
:1086000006FB0BF2521AB2FBFBF206FB0323019AA4
:108610009B1AB3F57A7FDFD3BAF1010AC0D1029B6E
:108620001B7C022B04D107226821039809F028FF44
:108630004FF0640ADFF830924FF01008894E4FF483
:108640007A77DFF828C2D9F80430C3F30803002B87
:1086500040F00F84EFF31183002B40F00A8421686F
:10866000B26800BF23689942F9D1286807FB00F37C
:108670009B1AB3FBF0F307FB013101200191D9F8FC
:108680000430C3F30803002B40F0B883EFF31183E9
:10869000002B40F0B3832368B16800BF2268934287
:1086A000F9D1D5F800B007FB0BF2521AB2FBFBF27E
:1086B00007FB0323019A9B1AB3F57A7FDFD3BAF144
:1086C000010AC0D1029B1B7C022B04D152466B21B4
:1086D000039809F0D5FE4FF0640ADFF88C914FF053
:1086E000100C60484FF47A76DFF880E1D9F8043056
:1086F000C3F30803002B40F08584EFF31183002BB4
:1087000040F080842168826800BF23689942F9D1D3
:108710002F6806FB07F39B1AB3FBF7F306FB013147
:1087200001270191D9F80430C3F30803002B40F06E
:108730004883EFF31183002B40F043832368816863
:1087400000BF22689342F9D1D5F800B006FB0BF2C6
:10875000521AB2FBFBF206FB0323019A9B1AB3F5F4
:108760007A7FDFD3BAF1010AC0D1029B1B7C022BB6
:1087700004D101226B21039809F082FE4FF00F0A09
:10878000DFF8E4904FF0100C36484FF47A76DFF8BB
:10879000DCE0D9F80430C3F30803002B40F0158463
:1087A000EFF31183002B40F010842168826800BF32
:1087B00023689942F9D12F6806FB07F39B1AB3FB94
:1087C000F7F306FB013101270191D9F80430C3F317
:1087D0000803002B40F0D882EFF31183002B40F008
:1087E000D3822368816800BF22689342F9D1D5F80B
:1087F00000B006FB0BF2521AB2FBFBF206FB03239E
:10880000019A9B1AB3F57A7FDFD3BAF1010AC0D17E
:10881000029991F853200B7C042A34BF18221A22A3
:10882000022B03D11B21039809F02AFE4FF00F0AF7
:10883000DFF834904FF0100C0A484FF47A76DFF8E6
:108840002CE0D9F80430C3F30803002B40F0138464
:10885000EFF31183002B40F00E8409E02CB90120C6
:1088600030B9012010E000E000ED00E028B901205F
:108870002168826800BF23689942F9D12F6806FBFE
:1088800007F39B1AB3FBF7F306FB013101270191B4
:10889000D9F80430C3F30803002B40F05882EFF3FB
:1088A0001183002B40F053822368816800BF226847
:1088B0009342F9D1D5F800B006FB0BF2521AB2FB85
:1088C000FBF206FB0323019A9B1AB3F57A7FDFD3F1
:1088D000BAF1010AB5D1029B1B7C022B04D11822EC
:1088E0001C21039809F0CCFD4FF00F0ADFF8D0925D
:1088F0004FF0100CB0484FF47A76DFF8C0E2D9F8A8
:108900000430C3F30803002B40F09983EFF3118385
:10891000002B40F094832168826800BF236899424D
:10892000F9D12F6806FB07F39B1AB3FBF7F306FB9D
:10893000013101270191D9F80430C3F30803002B5A
:1089400040F0E881EFF31183002B40F0E3812368CE
:10895000816800BF22689342F9D1D5F800B006FBC8
:108960000BF2521AB2FBFBF206FB0323019A9B1A8D
:10897000B3F57A7FDFD3BAF1010AC0D1029B1B7C29
:10898000022B06D1029B1A21039893F8522009F07A
:1089900077FD4FF00F0ADFF828924FF0100C864851
:1089A0004FF47A76DFF814E2D9F80430C3F3080301
:1089B000002B40F0B482EFF31183002B40F0AF8224
:1089C0002168826800BF23689942F9D12F6806FBAD
:1089D00007F39B1AB3FBF7F306FB01310127019163
:1089E000D9F80430C3F30803002B40F07681EFF38D
:1089F0001183002B40F071812368816800BF2268D9
:108A00009342F9D1D5F800B006FB0BF2521AB2FB33
:108A1000FBF206FB0323019A9B1AB3F57A7FDFD39F
:108A2000BAF1010AC0D1029B1B7C022B06D1029B2A
:108A30001921039893F8542009F022FD4FF0640A9D
:108A4000DFF87C914FF0100C5B484FF47A76DFF83A
:108A50006CE1D9F80430C3F30803002B40F04382E3
:108A6000EFF31183002B40F03E822168826800BF43
:108A700023689942F9D12F6806FB07F39B1AB3FBD1
:108A8000F7F306FB013101270191D9F80430C3F354
:108A90000803002B40F00481EFF31183002B40F01A
:108AA000FF802368816800BF22689342F9D1D5F81E
:108AB00000B006FB0BF2521AB2FBFBF206FB0323DB
:108AC000019A9B1AB3F57A7FDFD3BAF1010AC0D1BC
:108AD000029B1B7C022B04D110223721039809F042
:108AE000CFFC4FF00F0ADFF8D8904FF0100C32484F
:108AF0004FF47A76DFF8C4E0D9F80430C3F3080302
:108B0000002B40F04682EFF31183002B40F04182AE
:108B10002168826800BF23689942F9D12F6806FB5B
:108B200007F39B1AB3FBF7F306FB01310127019111
:108B3000D9F80430C3F30803002B40F09480EFF31E
:108B40001183002B40F08F802368816800BF22686A
:108B50009342F9D1D5F800B006FB0BF2521AB2FBE2
:108B6000FBF206FB0323019A9B1AB3F57A7FDFD34E
:108B7000BAF1010AC0D1029B1B7C022B04D10398DD
:108B80000122382109F07CFC4FF00F09DFF830801A
:108B90004FF0100E08494FF47A70084FD8F804309F
:108BA000C3F30803002B40F0D681EFF31183002BB1
:108BB00040F0D18106E000BF10E000E028B90120BC
:108BC00000ED00E022688E6800BF23689A42F9D168
:108BD000D5F800C000FB0CF39B1BB3FBFCF300FBC0
:108BE000023301930126D8F80430C3F30803F3B924
:108BF000EFF31183DBB92368D1F808A000BF226826
:108C00009342F8D1D5F800B000FB0BFCACEB0A0C9A
:108C1000BCFBFBFC00FB03C3019A9B1AB3F57A7FF4
:108C2000E1D3B9F10109B9D10BB0BDE8F08FEFF391
:108C3000118A8EF312888A680B68DB0301D53E60C7
:108C40008A6823685FFA8AFAD7F800C08AF3118825
:108C5000D5F800A09C4400FB0AF39B1AB3FBFAF37F
:108C600000FB0C33D8E7EFF311888CF3128881688E
:108C70000368DB0302D5CEF80070816823685FFAD1
:108C800088F8DEF8002088F31188D5F800801A44AF
:108C900006FB08F35B1AB3FBF8F306FB023362E74B
:108CA000EFF311888CF3128881680368DB0302D527
:108CB000CEF80070816823685FFA88F8DEF800203B
:108CC00088F31188D5F800801A4406FB08F35B1A74
:108CD000B3FBF8F306FB0233F2E6EFF311888CF3F3
:108CE000128881680368DB0302D5CEF800708168C2
:108CF00023685FFA88F8DEF8002088F31188D5F839
:108D000000801A4406FB08F35B1AB3FBF8F306FB7A
:108D1000023380E6EFF311888CF3128881680368D0
:108D2000DB0302D5CEF80070816823685FFA88F80B
:108D3000DEF8002088F31188D5F800801A4406FB7D
:108D400008F35B1AB3FBF8F306FB02330EE6EFF30E
:108D500011888CF3128881680368DB0302D5CEF892
:108D60000070816823685FFA88F8DEF8002088F3D5
:108D70001188D5F800801A4406FB08F35B1AB3FB90
:108D8000F8F306FB02339EE5EFF311888CF31288AB
:108D900081680368DB0302D5CEF800708168236820
:108DA0005FFA88F8DEF8002088F31188D5F8008093
:108DB0001A4406FB08F35B1AB3FBF8F306FB023315
:108DC0001EE5EFF311888CF3128881680368DB03DA
:108DD00002D5CEF80070816823685FFA88F8DEF863
:108DE000002088F31188D5F800801A4406FB08F3A8
:108DF0005B1AB3FBF8F306FB0233AEE4EFF3118E1C
:108E000088F31288B1683368DB0302D5CCF8000020
:108E1000B16823685FFA8EFEDCF800208EF31188BB
:108E2000D5F800E01A4407FB0EF35B1AB3FBFEF320
:108E300007FB02333EE4EFF311888CF3128881685C
:108E40000368DB0302D5CEF80070816823685FFAFF
:108E500088F8DEF8002088F31188D5F800801A44DD
:108E600006FB08F35B1AB3FBF8F306FB0233FFF7CC
:108E7000CEBBEFF3118288F31288B0683368D90350
:108E800003D50123CCF80030B0682368D2B2DCF8F7
:108E9000001082F311882A68194407FB02F31B1A99
:108EA000B3FBF2F307FB0131FFF7E7BBEFF31182EE
:108EB0008CF3128887680368D90303D50123CEF8A1
:108EC000003087682368D2B2DEF8001082F3118880
:108ED0002A68194406FB02F3DB1BB3FBF2F306FB23
:108EE0000131FFF777BBEFF311828CF312888768AB
:108EF0000368D90303D50123CEF8003087682368BF
:108F0000D2B2DEF8001082F311882A68194406FBF9
:108F100002F3DB1BB3FBF2F306FB0131B3E5EFF326
:108F200011828CF3128887680368D90303D5012363
:108F3000CEF8003087682368D2B2DEF8001082F3E2
:108F400011882A68194406FB02F3DB1BB3FBF2F31A
:108F500006FB013142E5EFF311868EF31288D1F85A
:108F600008C00B68DA0303D501233B60D1F808C0C1
:108F70002368F6B23A6886F311882E681A4400FB1B
:108F800006F3A3EB0C03B3FBF6F300FB02330193F0
:108F900028E6EFF311828CF3128887680368D903FF
:108FA00003D50123CEF8003087682368D2B2DEF8FB
:108FB000001082F311882A68194406FB02F3DB1BB8
:108FC000B3FBF2F306FB0131B0E5EFF311828CF352
:108FD000128887680368D90303D50123CEF80030CF
:108FE00087682368D2B2DEF8001082F311882A68FD
:108FF000194406FB02F3DB1BB3FBF2F306FB013162
:10900000FFF7E1BBEFF311828CF3128887680368E6
:10901000D90303D50123CEF8003087682368D2B284
:10902000DEF8001082F311882A68194406FB02F367
:10903000DB1BB3FBF2F306FB0131FFF771BBEFF370
:1090400011828CF3128887680368D90303D5012342
:10905000CEF8003087682368D2B2DEF8001082F3C1
:1090600011882A68194406FB02F3DB1BB3FBF2F3F9
:1090700006FB01315DE4EFF311828CF312888768FF
:109080000368D90303D50123CEF80030876823682D
:10909000D2B2DEF8001082F311882A68194406FB68
:1090A00002F3DB1BB3FBF2F306FB0131FFF7EEBB70
:1090B0001C0903F00F03013C042C51D82B4A32F851
:1090C000140040FA03F2D5074AD5012505FA03F347
:1090D000013B184034F064FB254B26491B5D1844C6
:1090E00011EBC0023CD051F8300096880369334040
:1090F0007FF43EAA2021B6FA86F4D3719171C4F1AF
:109100001F041D4A0299CA60621C3FF431AA1B4A1F
:1091100005A91B4F05960793089309933E5D069298
:109120001CF0CCFA029B174803F10C021649835D30
:1091300041F82420F02B7FF71BAABB19F022032152
:109140001C7C825566B23046760929F085FE04F013
:109150001F030E4A05FA03F342F82630FFF708BA58
:10916000054B029AD360FFF703BA00BF1C1E040828
:10917000141E04087C8501204D8000080000111099
:10918000E0F50308384D0120F84C012000E100E033
:109190002DE9F04FA84A83B043690190934200F053
:1091A000908102F58062934200F08B8138211A6829
:1091B0001027A24C4FF47A7522F04002DFF8888223
:1091C0009F4E1A601A6822F038020A431A601A6821
:1091D00042F040021A6008F0ABFBDFF870E2844610
:1091E00098490120DEF80430C3F30803002B40F057
:1091F0002F81EFF31183002B40F02A812368D1F8EF
:10920000089000BF22689342F8D1D8F800A005FB6F
:109210000AF2A2EB0902B2FBFAF205FB03239C451A
:10922000E0D0019D2846FFF79AF9EA691AB19388C0
:1092300012681B049361019B5A6940F2E93302E012
:10924000002B00F056819168013B11F0020F9BB298
:10925000F6D06A2140F2E933117302E0002B00F0EE
:109260005E819168013B11F0010F9BB2F6D0D3688B
:10927000019B5A6940F2E93302E0002B00F02381A0
:109280009168013B11F0020F9BB2F6D0102140F221
:10929000E933117302E0002B00F015819168013B66
:1092A00011F0010F9BB2F6D0D368019BDB6913B1BB
:1092B0001A689B8893614FF0640ADFF890914FF031
:1092C000100E60484FF47A755D4FD9F80430C3F33F
:1092D0000803002B40F0DA80EFF31183002B40F0FD
:1092E000D5802168826800BF23689942F9D1D8F8F7
:1092F000006005FB06F39B1AB3FBF6F305FB013197
:1093000001260091D9F80430C3F30803002B5BD188
:10931000EFF31183002B57D12368816800BF2268C7
:109320009342F9D1D8F800B005FB0BF2521AB2FB08
:10933000FBF205FB0323009A9B1AB3F57A7FE1D376
:10934000BAF1010AC1D1019B3B4A5B69934205D046
:1093500002F58062934218BF4FF0080A1A684FF472
:109360007A76384D22F04002354F1A601A6822F0A2
:10937000380242EA0A021A601A6842F040021A6091
:1093800008F0D6FADFF8C4C081464FF0100E012075
:10939000DCF80430C3F308038BBBEFF3118373BB1A
:1093A0002368A96800BF22689342F9D1D8F800A0C9
:1093B00006FB0AF2521AB2FBFAF206FB03239945A6
:1093C000E6D003B0BDE8F08FEFF3118C8EF3128876
:1093D00081680368DA0301D53E60816823685FFA1B
:1093E0008CFC3A688CF31188D8F800C01A4405FB4D
:1093F0000CF35B1AB3FBFCF305FB02339BE7EFF3C3
:1094000011818EF31288D5F808A02B68DB0302D5F2
:109410003860D5F808A02368C9B23A6881F311888A
:10942000D8F800101A4406FB01F3A3EB0A03B3FBC0
:10943000F1F306FB0233C2E7003800402CB90120EB
:1094400028B9012010E000E030B9012000ED00E073
:10945000EFF3118987F31288D1F808A00B68DB03BA
:1094600002D53060D1F808A023685FFA89F9326824
:1094700089F31188D8F800901A4405FB09F3A3EB8F
:109480000A03B3FBF9F305FB0233C8E6EFF31182DD
:109490008EF3128886680368D90302D501233B60E6
:1094A00086682368D2B2396882F31188D8F8002020
:1094B000194405FB02F39B1BB3FBF2F305FB0131DF
:1094C0001EE7302173E625498A4208D0244B9A4290
:1094D00041D003F580639A427FF4E7AE0223214A2C
:1094E000D82101FB03239A89013292B29A819B8988
:1094F000DBE61A498A4208D0194B9A4229D003F573
:1095000080639A427FF4B6AE02231649D82000FB4E
:1095100003139989013189B299819B89AAE60F4980
:109520008A4208D00E4B9A4211D003F580639A42CA
:109530007FF49EAE02230B4AD82101FB03239A89B4
:10954000013292B29A819B89019B5A6992E601236A
:10955000F1E70123D9E70123C1E700BF0030014053
:10956000003800401C820120406994301CF050BE3D
:1095700041690C4B10B503EB0124B4F8FC2002EB5D
:10958000811203EB8203D86F1CF042FE63681B68F4
:109590001A6822F001021A60DA6822F48072DA6036
:1095A00010BD00BFF8A30120426910B50832184C65
:1095B00054F822001CF02CFE164B1A8823460C2A65
:1095C0000DD8DFE802F0070C0C0C130C0C0C190C76
:1095D0000C0C1F002168CA6822F40072CA600122C4
:1095E00083F83D2000220C4B1A7010BD2168CA6818
:1095F00022F48062CA60F2E72168CA6822F400623D
:10960000CA60ECE72168CA6822F48052CA60E6E7C3
:10961000B46B0120B06B0120A65C0120F8B5D0F836
:1096200018310446DA69910615D5586AE36AC0B262
:10963000002B00F0A980216B9847D4F818311A68E4
:1096400022F480721A609A6822F001029A609A6984
:1096500042F008029A61DA69D20701D501221A6242
:10966000DA69970701D502221A62DA69560701D52D
:1096700004221A62DA69150701D508221A62D4F8A1
:10968000F820002A00F08C80D969490600D4F8BD82
:10969000D96904F58C701E680F079D6819D18F0673
:1096A00002D5B50600F1FE800F0602D5350600F1A1
:1096B000DB80480602D5710600F1AF80002AE6D0B3
:1096C000626AA36A9A4240F08480012384F88C3154
:1096D000F8BD15F0010540F0818016F4907FE3D0CD
:1096E00011F0010700F0DC8016F480777AD13D4656
:1096F00005EA91073FB104271F62D4F8847147F04F
:109700000207C4F884710F070AD5B70640F19680A6
:1097100008251D62D4F8845145F00805C4F8845129
:10972000D4F88451002DC9D08F0605D5B50603D5D0
:109730001CF086F9D4F81831D4F88421110774D5B7
:109740001A68202122F490721A609A6822F00102AD
:109750009A6084F882119A6852066CD59968D4F898
:109760007C2121F040019960002A64D092F83530C4
:109770005A49022B116565D08023104653651BF0B2
:1097800013FDD4F8F82099E7E3696269D054E369DE
:10979000E1680133B3FBF1F201FB1233E3614CE703
:1097A000D96908067FF570AF94F8811121293FF43B
:1097B0006BAFA16A606A81424FD0A069405C013101
:1097C000C0B298622569B1FBF5F005FB1011A162EA
:1097D0005AE72046BDE8F840FEF7D8BDCF0709D5C7
:1097E000F70507D501271F62D4F8847147F00107F8
:1097F000C4F88471EDB215EA51073FF479AF4FF028
:10980000020E3D46C1F38007C3F820E0D4F884E19E
:109810004EF0040EC4F884E16CE71968202021F0B2
:109820004001196084F8810148E79A6812F040020B
:1098300086D1C4F88421D4F8F8203FE7002D3FF406
:109840006FAF65E71168052382F835300B68D4F8EF
:10985000F82023F001030B6030E7A4F86A211968AF
:1098600021F0800119600FE794F8811121297FF41C
:1098700025AFB4F86A1189B2C9B1D4F82011B1F595
:10988000805F1DD0D4F86411481CC4F864010978C5
:109890009962B4F86A31013B9BB2A4F86A310DE7D2
:1098A0003D4630E71CF0CCF8D4F8F82006E71968FC
:1098B00021F080011960196841F040011960FDE64E
:1098C000D4F828110029DDD1D4F8641131F8020B45
:1098D000C0F308009862C4F86411DAE7A9510208DD
:1098E000F8B5A34BA3491A680D6822F040021A602C
:1098F0001A6822F0380242F010021A601A6842F028
:1099000040021A601DB1AB882A681B0493619A4B10
:109910001B78012B00F03E82C0F0FB81022B40F04F
:109920009D810822954B4FF0080E1A704FF4C372B8
:1099300011468F4B92480180196821F0400119604F
:10994000196821F0380141F010011960196841F0DF
:10995000400119601DB1AB8829681B048B61102080
:109960008349884C01265FFA80FC40F2E93302E02B
:10997000002B00F088818F68013B17F0020F9BB22B
:10998000F6D081F80CC040F2E93302E0002B00F081
:109990007A818F68013B17F0010F9BB2F6D0CB683C
:1099A00040F2E93302E0002B00F064818F68013B54
:1099B00017F0020F9BB2F6D00E7340F2E93302E0CB
:1099C000002B00F057818F68013B17F0010F9BB20D
:1099D000F6D0CB6801302028C5D115B12B68A988F5
:1099E0009961634B196821F040011960196821F0F1
:1099F00038011960196841F040011960196821F0B7
:109A000040011960196821F0380141F01001196016
:109A1000196841F0400119601DB1AB8829681B0429
:109A20008B6140F2E933524802E0002B00F03581AF
:109A30008168013B11F0020F9BB2F6D0002140F289
:109A4000E9334B4C017302E0002B00F02681A16842
:109A5000013B11F0010F9BB2F6D0E36840F2E9330D
:109A6000434802E0002B00F09E818168013B11F029
:109A7000020F9BB2F6D080F80CE040F2E9333C488C
:109A800002E0002B00F08F818168013B11F0010F93
:109A90009BB2F6D0C3683C4940F2E93334480C78B5
:109AA00002E0002B00F089818168013B11F0020F78
:109AB0009BB2F6D0022140F2E9332D4E017302E051
:109AC000002B00F07A81B168013B11F0010F9BB2CD
:109AD000F6D0F36840F2E933254802E0002B00F0AD
:109AE000E6808168013B11F0020F9BB2F6D004734F
:109AF00040F2E9331E4802E0002B00F0D880816874
:109B0000013B11F0010F9BB2F6D0C3681F4940F230
:109B1000E93317480C7802E0002B00F0D28081680E
:109B2000013B11F0020F9BB2F6D0032140F2E93362
:109B30000F4E017302E0002B00F0C380B168013BBF
:109B400011F0010F9BB2F6D0F36840F2E9330848F8
:109B500002E0002B00F0BF808168013B11F0020F92
:109B60009BB2F6D0047340F2E933014813E000BF22
:109B700000380040FC88012000890120B61B01202C
:109B8000B41B01201C8201200789012008890120C3
:109B9000002B00F0A0808168013B11F0010F9BB207
:109BA000F6D0C368974940F2E93397480C7844F0FF
:109BB000040402E0002B00F098808168013B11F062
:109BC000020F9BB2F6D0042140F2E9338E4E0173AE
:109BD00002E0002B00F08980B168013B11F0010F19
:109BE0009BB2F6D0F36840F2E933874802E0002BDD
:109BF00000F085808168013B11F0020F9BB2F6D026
:109C0000047340F2E933804801E0002B77D081688B
:109C1000013B11F0010F9BB2F7D0C36815B12B685F
:109C2000A9889961784B0021784D1C68784824F008
:109C300040041C601C6824F038041C601C6844F05C
:109C400040041C6035F05DFC2B782BB3714B1B7806
:109C5000002B00F0BC8000232B70F8BD6E4B93F8F6
:109C600000E01EF0400F0CBF4FF4C3724FF4F072CF
:109C700011465EE6B4F8E43001339BB2A4F8E43058
:109C8000B4F8E430A6E6B4F8E43001339BB2A4F8AB
:109C9000E430B4F8E43083E6F8BD6049B1F8E4306C
:109CA00001339BB2A1F8E430B1F8E430D6E65B4969
:109CB000B1F8E43001339BB2A1F8E430B1F8E430FC
:109CC00024E75649B1F8E43001339BB2A1F8E430FF
:109CD000B1F8E43039E75149B1F8E43001339BB2CF
:109CE000A1F8E430B1F8E4305CE74C49B1F8E43075
:109CF00001339BB2A1F8E430B1F8E43073E747498F
:109D0000B1F8E43001339BB2A1F8E430B1F8E430AB
:109D100084E740F2E9333C4901E0002B5CD08A68DB
:109D2000013B12F0020F9BB2F7D0A02240F2E933C0
:109D300035480A7301E0002B4ED08268013B12F0D7
:109D4000010F9BB2F7D0C36840F2E9332E4901E01E
:109D5000002B4BD08A68013B12F0020F9BB2F7D068
:109D6000002240F2E93328480A7301E0002B3DD07D
:109D70008268013B12F0010F9BB2F7D0C368DBB2DF
:109D800003F00602022A3FF4CCAD03F00503012BD9
:109D90007FF4C7AD4822204B4FF0480E1A704FF4A5
:109DA000F0721146C5E51D49B1F8E43001339BB2AC
:109DB000A1F8E430B1F8E4306DE61849B1F8E430C8
:109DC00001339BB2A1F8E430B1F8E43082E602F04E
:109DD000FDF800232B70F8BD104AB2F8E4300133CF
:109DE0009BB2A2F8E430B2F8E430ADE70B4AB2F827
:109DF000E43001339BB2A2F8E430B2F8E430DBB2D5
:109E0000BEE700BF3C2901200038004000000120CF
:109E10000425012029740120B61B01201C82012089
:109E200008B508F0A1FA0A2007F0D0FD012008BD0E
:109E3000F8B50F4D144646680F466A702521027A20
:109E4000304642F08002FFF7EBFF3A4626213046CB
:109E5000FFF7E6FF04F00F022721304642F08002B0
:109E6000FFF7DEFF07F064FD686001202870F8BD91
:109E7000C824012070B504780E461546032C16D16F
:109E800044682521027A2046FFF7CAFF3246262180
:109E90002046FFF7C5FF2A4663212046FFF7C0FF93
:109EA000812227212046FFF7BBFF012070BD022C35
:109EB00003D1BDE8704008F0E3BA002070BD2DE981
:109EC000F0410E46017890461F46032921D144688F
:109ED0002521027A204642F08002FFF7A1FF324698
:109EE00026212046FFF79CFF07F00F02272120467E
:109EF00042F08002FFF794FF042007F0C1FD72B624
:109F000049213B464246204608F0CAF962B6BDE800
:109F1000F081022905D146F08001BDE8F04108F04A
:109F2000BFB90020BDE8F08137B500F10C0405464B
:109F300000220A212046FFF79DFF0F220A2120461A
:109F4000FFF798FF01AA032310212046FFF7B7FF70
:109F50009DF8043000220A2180332046EB839DF8CF
:109F6000053080332B849DF8063080336B84FFF7F7
:109F700081FF0DF10302012302212046FFF79FFF1D
:109F800001230DF1030209212046FFF798FF11225A
:109F90000A212046FFF76EFF012003B030BD2DE9F6
:109FA000FF47037B0546884600F10C061BB1022BD8
:109FB00006D9032B3DD00024204604B0BDE8F0872D
:109FC00001230DF1070202213046FFF778FF002838
:109FD000F1D09DF80730D907EDD5072302AA032158
:109FE0003046FFF76CFF0446002CE4D09DF80E705D
:109FF00011220A213046FFF73DFF3B07DBD4B5F9BC
:10A000001E1002A8FDF7FCFF4042A8F800000DF169
:10A010000A00B5F92010FDF7F3FF4042A8F802004E
:10A0200003A8B5F92210FDF7EBFF4042A8F80400A1
:10A03000C2E7234F4FF0010A0024B9463B7A012BB7
:10A040001BD00FD3022BCFD1FDF7E8FF81460028AC
:10A05000B1D102A905F11000FEF716FA87F80890B1
:10A060000446C1E73B7823B9012202213046FFF7BD
:10A07000DFFE012389F808309DE7FDF7CFFF0028B8
:10A0800099D102A905F11000FEF7FEF99DF80830FC
:10A09000044608B1DA0707D4002389F80830BAF17A
:10A0A000000F88D09A46C9E73B7823B907220321DD
:10A0B0003046FFF7BDFE022389F808307BE700BF7A
:10A0C000C8240120014B1869FFF7A8BA404D0120B0
:10A0D000014BD868FFF7A2BA404D0120014B9868A8
:10A0E000FFF79CBA404D0120014B5868FFF796BA24
:10A0F000404D0120014B1868FFF790BA404D0120F8
:10A10000F8B510F58C75044614D0D0F81821242128
:10A11000002380F88111116821F0010111601360A2
:10A1200053609360C0F8843180F8803180F88131C9
:10A1300080F88231A279A36812F00401C4F81C31BE
:10A1400000F0F8804FF48053C4F8203112F002037D
:10A1500000F029814FF400534FF48061C4F824319A
:10A1600063790020C4F8281113F00101C4F830010C
:10A17000C4F83801C4F82C0102D00420C4F82C0122
:10A1800013F0020605D0D4F82C0140F00800C4F802
:10A190002C01D0070DD549B1D4F83C014FF48037DC
:10A1A00040F00200C4F84471C4F83C01002E40F0B5
:10A1B000E88012072AD5002D58D094F8813103F099
:10A1C000FF02002B00F0E880D4F818212423284651
:10A1D00084F88131136823F0010313601BF022FE21
:10A1E000012840D0D4F83C31002B40F0D880D4F87E
:10A1F000183128465A6822F490425A609A6822F030
:10A2000022029A609A6842F0080225E075B394F839
:10A21000813103F0FF020BB984F88021D4F81821B2
:10A220002423284684F88131136823F00103136046
:10A230001BF0F8FD012816D0D4F83C3113B12846A4
:10A240001BF0A6FBD4F8183128465A6822F4904235
:10A250005A609A6822F02A029A601A6842F0010253
:10A260001A601BF05FFB637903F0010100292ED017
:10A27000D4F8F420002A75D00023D4F8FC004FF461
:10A28000806E4FF4803104F134074FF48076E3633D
:10A290002364A364E364A365E36563662366626382
:10A2A000A0633846C4F844E06165266527F0ACFD3C
:10A2B000384627F0E7FD94F88231C4F87C71202BF2
:10A2C000E5667AD0626B63795268C4F80C219B070B
:10A2D0002FD5D4F8F820002A3DD0002340204FF499
:10A2E0008031C4F8942004F19406D4F800214FF48E
:10A2F0008067C4F89C00C4F898203046C4F8A030A9
:10A30000C4F8A830C4F8AC30C4F8B030C4F8B830E1
:10A31000C4F8BC30C4F8C430C4F8C030C4F8A47069
:10A32000C4F8B41027F070FD304627F0ABFD50B1F3
:10A33000FEE7F8BD12F00203C4F8201138D1C4F8CA
:10A34000243119460CE7D4F89430C4F87861C4F885
:10A35000CC505860F8BDD4F88821136843F08003CE
:10A360001360F8BDD4F88821116841F48071116040
:10A37000916841F001019160116841F02001116084
:10A38000A5E7D4F83C014FF4003640F00100C4F8D2
:10A390004061C4F83C010CE784F8802114E72846AA
:10A3A0001BF0F6FA23E7C4F824314FF48061D7E6B6
:10A3B0004FF40053C4F82431D2E6E368626999B2DD
:10A3C000002A3FF47FAFB1FA81F67609002E7FF4C0
:10A3D00079AF94F8800101283FF474AF0B46A4F8DC
:10A3E000701138461549164F4FF0010C4FF0220EF0
:10A3F00061672767D4F81811124FC4F884612431BB
:10A40000C4F86C21C4F8846084F880C184F882E1C7
:10A41000C4F8807027F0B4FCD4F8183184F8806157
:10A420001A6842F480721A609A6842F001029A60D7
:10A430009A6842F040029A6044E700BF2552020841
:10A4400029520208B9510208417159E6816057E664
:10A45000B0B5BB4BB8B0BB491A6C00AFBA4842F0BC
:10A460008052BA4C1A641A6C02F08052C7F8D82095
:10A47000D7F8D8201A6B42F480221A631A6B02F4C0
:10A480008022C7F8D420D7F8D4200A6842F480721A
:10A490000A600268A24200F04882AD4C4FF6FF0508
:10A4A000AC4AE168AC4829400A43E2605A6F026056
:10A4B0001A6B42F480221A631A6B02F48022C7F8E6
:10A4C000DC20D7F8DC201A6B42F480121A631A6B76
:10A4D00002F48012C7F8D020D7F8D0201A6B42F4CB
:10A4E00080021A631A6B02F48002C7F8CC20D7F8F6
:10A4F000CC201A6B42F000521A631A6B02F0005221
:10A50000C7F8C820D7F8C8201A6B42F080421A63F7
:10A510001A6B02F08042C7F8C420D7F8C4201A6B27
:10A5200042F001021A631A6B02F00102C7F8C02060
:10A53000D7F8C0201A6B42F002021A631A6B02F0BD
:10A540000202C7F8BC20D7F8BC201A6B42F0040204
:10A550001A631A6B02F00402C7F8B820D7F8B820C3
:10A560001A6B42F008021A631A6B02F00802C7F86D
:10A57000B420D7F8B4201A6B42F010021A631A6B99
:10A5800002F01002C7F8B020D7F8B0201A6B42F0E2
:10A5900020021A631A6B02F02002C7F8AC20D7F829
:10A5A000AC201A6B42F040021A631A6B02F04002B0
:10A5B000C7F8A820D7F8A8201A6B42F080021A63C7
:10A5C0001A6B02F08002C7F8A420D7F8A4201A6BF7
:10A5D00042F480721A631A6B02F48072C7F8A020EA
:10A5E000D7F8A0201A6C42F001021A641A6C02F02B
:10A5F0000102C7F89C20D7F89C201A6C42F0020296
:10A600001A641A6C02F00202C7F89820D7F8982052
:10A610001A6C42F004021A641A6C02F00402C7F8C1
:10A620009420D7F894201A6C42F008021A641A6C2D
:10A6300002F00802C7F89020D7F890201A6C42F078
:10A6400010021A641A6C02F01002C7F88C20D7F8B6
:10A650008C201A6C42F020021A641A6C02F020025C
:10A66000C7F88820D7F888201A6C42F040021A6494
:10A670001A6C02F04002C7F88420D7F884201A6CC4
:10A6800042F080021A641A6C02F08002C7F880203F
:10A69000D7F880201A6C42F480721A641A6C02F4A3
:10A6A0008072FA67FA6F1A6C42F400721A641A6CBC
:10A6B00002F40072BA67BA6F1A6C42F480421A64EC
:10A6C0001A6C02F480427A677A6F1A6C42F4004284
:10A6D0001A641A6C02F400423A673A6F1A6C42F438
:10A6E00000321A641A6C02F40032FA66FA6E1A6CBE
:10A6F00042F480221A641A6C02F48022BA66BA6E9E
:10A700001A6C42F400221A641A6C02F400227A666F
:10A710007A6E1A6C42F480121A641A6C02F4801277
:10A720003A663A6E1A6C42F400121A641A6C02F419
:10A730000012FA65FA6D1A6C42F480020EE000BF56
:10A74000003802400070004004400240EFBEADDE21
:10A7500000ED00E00005FA052C9F01201A641A6C38
:10A7600002F48002BA65BA6D1A6C42F400021A64EF
:10A770001A6C02F400027A657A6D1A6C42F000726B
:10A780001A641A6C02F000723A653A6D1A6C42F063
:10A7900000521A641A6C02F00052FA64FA6C1A6CD5
:10A7A00042F080421A641A6C02F08042BA64BA6CB9
:10A7B0001A6C42F000421A641A6C02F000427A6489
:10A7C0007A6C5A6C42F001025A645A6C02F001022F
:10A7D0003A643A6C5A6C42F002025A645A6C02F0C3
:10A7E0000202FA63FA6B5A6C42F010025A645A6C15
:10A7F00002F01002BA63BA6B5A6C42F020025A643B
:10A800005A6C02F020027A637A6B5A6C42F48072BE
:10A810005A645A6C02F480723A633A6B5A6C42F48E
:10A8200000725A645A6C02F40072FA62FA6A5A6C44
:10A8300042F480625A645A6C02F48062BA62BA6A64
:10A840005A6C42F400625A645A6C02F400627A62F2
:10A850007A6A5A6C42F480525A645A6C02F48052FA
:10A860003A623A6A5A6C42F400525A645A6C02F4E0
:10A870000052FA61FA695A6C42F480325A645A6C96
:10A8800002F48032BA61BA695A6C42F400325A64F6
:10A890005A6C02F400327A617A695A6C42F480226E
:10A8A0005A645A6C02F480223A613A695A6C42F452
:10A8B00080125A645A6C02F48012FA60FA685A6C78
:10A8C00042F480025A645A6C02F48002BA60BA6898
:10A8D0005A6C42F400025A645B6C03F400037B6020
:10A8E0007B681BF063FA1D4B02461D491B681D481F
:10A8F000A1FB03131C49A0FB02029B09920C013B24
:10A900000A60B3F1807F08D2184AF02500200721A1
:10A91000536084F8235090601160144AE037136844
:10A9200043F004031360BD46B0BD114A01F5484130
:10A9300002605A6C0F4842F480425A645B6C03F424
:10A940008043C7F8DC30D7F8DC300A6803680A6057
:10A9500083F30888084B1B689847FEE79420012082
:10A96000D34D621083DE1B4330B9012010E000E0BC
:10A97000EDFEFECA0000F01F0400F01F08B5054BF5
:10A980001B6803B19847044B044A1A6072B6FDF77E
:10A99000C7FB00BF846D012004400240EFBEADDE66
:10A9A00008B5034B1B6803B1984772B6FDF7B8FBB7
:10A9B000846D012030B439240C4D0022A0422B4676
:10A9C00006D001322433052A0CD01C79A042F8D1DC
:10A9D0009C79214201D10029F3D102EBC20205EB9F
:10A9E000820000E0002030BC704700BFA81E0408B1
:10A9F00030B5A02285B000211A4834F082FD1A4AF1
:10AA00001A4C0423116C04F1B40541F002011164E5
:10AA1000116C01F0020101910199116C41F00801E2
:10AA20001164116C01F0080102910299516C41F01E
:10AA300002015164526C02F002020392039A2BB994
:10AA40002434AC420CD0A379002BF9D020792434E3
:10AA500007F0EAF914F81C1C28F0E0FBAC42F2D134
:10AA600005B030BD00B6012000380240A81E040821
:10AA700001490248FDF71EBD50B601200004014007
:10AA8000FFF7F6BF01490248FDF714BD28B60120C3
:10AA9000000C004001490248FDF70CBD00B6012042
:10AAA0000004004003682DE9F0439B0A464CA34292
:10AAB0007ED03E34A34258D0403CA34201D0BDE8F2
:10AAC000F08300244079414F8608002953D04FEA93
:10AAD000841E02254FEA840C57F80E8005FA06F012
:10AAE0000CEB040ED8F80C9006EB4E05DFF8E0E016
:10AAF00040EA09002E1D4EF825104EF82620C8F811
:10AB00000C00314A934257D03E32934252D0403AE1
:10AB10009342D4D100260CEB0403DB0003F12000A8
:10AB20007044EFF31185502282F312881033002213
:10AB300073441968013211B1016018680430042AA5
:10AB400003F10403F5D10023EDB2036085F311880E
:10AB50006444B6010EEBC404BA59236A73B3D368D4
:10AB600043F00103D360BDE8F08340790224174F1E
:10AB700086080029ABD1A5014FF0020E4FEA840CE4
:10AB800057F8058020FA0EF00CEB04050EFA00FED3
:10AB9000D8F80C0006EB450520EA0E00DFF830E09F
:10ABA0002E1DC8F80C004EF825104EF82620A8E7F8
:10ABB000012487E70226AEE70126ACE7D36823F03D
:10ABC0000103D360BDE8F08303001000FC8701207F
:10ABD00000B60120F0B5830A4F4C85B0A34200F0C7
:10ABE00095803E34A34200F08F80403CA34201D0C8
:10ABF00005B0F0BD0025AD01484E74597319A0424F
:10AC0000F6D00446464801394FF0000E0768184652
:10AC100089B2C3F810E0C3F808E0D960C3F814E0C3
:10AC20007451B7FBF2F2013A5A6027F0CDF93D4971
:10AC3000B4F1804F18BF8C420CBF0121002111D00C
:10AC4000394B9C420ED003F580639C420AD0374AB0
:10AC500003F57C439C4218BF944203D003F5705324
:10AC60009C42C5D1721900234FF4805792F83C00E2
:10AC700001930128029303930097B9D070590227DA
:10AC8000DFF8B0E04FF0010C82F83D70876807EA0A
:10AC90000E0E274FC0F808E0D0F808E00EEA0707CC
:10ACA000876082F83C3082F83DC0B9B91E4B9C42A7
:10ACB00014D003F580639C4210D003F580639C425E
:10ACC00003D003F578439C4292D17219002392F885
:10ACD0003C200093012A0193029389D073591148B3
:10ACE0005A688342996813D000F5806083420FD080
:10ACF00022F0700221F08001354400205A609960F2
:10AD000085F83C0005B0F0BD022574E7012572E727
:10AD100022F47002ECE700BF03001000FC87012062
:10AD2000942001200000014000040040000C00407D
:10AD3000F8FFFEFF8800FEFFF8B5464F05027C19BC
:10AD40006368002B3ED09B69002B3BD0227C0646DB
:10AD5000414B002042EA4101207420468AB21B6820
:10AD6000111281EA1211514001F00F0141EA021162
:10AD700089B2984763685B799B08B0B194F8FE107C
:10AD80004A2200EB861412FB0131344A053405F1E6
:10AD9000140302EB810207EB84043B4453F8041BC9
:10ADA0001032A34242F8081CF8D13D44B5F8FC30FB
:10ADB00003EB861607EB8607FA6F92F83530DBB2A5
:10ADC000012B00D0F8BD92F834100129FAD092F886
:10ADD000351095F8FE600129EC6D956D82F83430E0
:10ADE00003D0002382F83430ECE74FF0020E002746
:10ADF00003B2116882F835E04C34576503FA0EF35C
:10AE0000174F4FF4947E08680EFB0676976820F47F
:10AE10008020402F08604B6018D08E60CC60D06DD1
:10AE20003F23126C8340AB600B6843F016030B604A
:10AE30004B6943F080034B611AB10B6843F0080380
:10AE40000B600B6843F001030B60F8BD8C60CE60B3
:10AE5000E5E700BFF8A30120ECA30120FCAB012033
:10AE600004AC012030B44468012B24F480544460C5
:10AE70001CDD40F2E93401E0013C35D08568AD07C6
:10AE8000FAD500293DD031F8024B848140F2E934F3
:10AE900001E0013C28D08568ED07FAD5C468A4B26A
:10AEA0000AB122F8024B023B012BE2DC446844F475
:10AEB0008054446013B340F2E93301E0013B37D0E2
:10AEC0008468A407FAD5002936D00B78037340F2C2
:10AED000E93301E0013B2BD08168C907FAD5C3688B
:10AEE000DBB25AB1137009E0144B98420CD0144BEA
:10AEF000984219D003F58063984217D0012030BCE6
:10AF000070474FF6FF74C0E723460E4AD82101FB75
:10AF100003239A89013292B29A81988980B20030D3
:10AF200030BC18BF012070470123EEE70223ECE795
:10AF3000024A9042DBD1E8E7FF23C7E70030014037
:10AF4000003800401C82012070B5C36982B00446FD
:10AF50001BB19A88196812048A6107236A4611494D
:10AF60006069FFF77FFFE36913B11A689B889361FB
:10AF70009DF8013001209DF802109DF8036041EA20
:10AF800003219DF804209DF805509DF8063042EA03
:10AF90000622A18743EA0523E287A4F8403002B0E5
:10AFA00070BD00BFF8F50308037C022B01D0002020
:10AFB000704770B5C36982B01BB19A8819681204D2
:10AFC0008A61426940F2E93301E0002B39D091688F
:10AFD000013B11F0020F9BB2F7D0C32140F2E933DD
:10AFE000117301E0002B41D09168013B11F0010F7A
:10AFF0009BB2F7D0D368426904460623104600216D
:10B000006A46FFF72FFFE36913B11A689B889361C3
:10B010009DF8003001209DF801109DF8026041EA82
:10B0200003219DF803209DF804509DF8053042EA65
:10B030000622A18743EA0523E287A4F8403002B044
:10B0400070BD17498A4207D0164B9A4224D003F5A7
:10B0500080639A42D0D102231349D82404FB0313FE
:10B060009989013189B299819B89C5E70C498A4246
:10B0700007D00C4B9A4211D003F580639A42BAD1A3
:10B080000223094AD82101FB03239A89013292B293
:10B090009A819B894269AFE70123DDE70123F0E74D
:10B0A00000300140003800401C820120037A022B4E
:10B0B00001D00020704770B5436982B01BB19A88F7
:10B0C000196812048A61C26840F2E93301E0002B7A
:10B0D00038D09168013B11F0020F9BB2F7D0BB2131
:10B0E00040F2E933117301E0002B40D09168013B3D
:10B0F00011F0010F9BB2F7D0D368C2680446062353
:10B10000104600216A46FFF7ADFE636913B11A6865
:10B110009B8893619DF8003001209DF801109DF8F7
:10B12000026041EA03219DF803209DF804509DF838
:10B13000053042EA0622618343EA0523A283E383C2
:10B1400002B070BD17498A4207D0174B9A4224D0EB
:10B1500003F580639A42D1D102231449D82404FB19
:10B1600003139989013189B299819B89C6E70D49F9
:10B170008A4207D00C4B9A4211D003F580639A4261
:10B18000BBD10223094AD82101FB03239A8901324A
:10B1900092B29A819B89C268B0E70123DDE701235F
:10B1A000F0E700BF00300140003800401C82012061
:10B1B000F8B55B4DD823044603FB0053661C187991
:10B1C00006F032FE0746F6B210B11223C671837143
:10B1D000D82303FB0453587906F026FE10B113233D
:10B1E000C6718371D82303FB0453987906F01CFEC3
:10B1F00010B11423C6718371D82303FB04539A7BC7
:10B20000002A5CD0DA7938464E2106F0D7FED826DF
:10B2100006FB04F6AF19787906F006FE3A7A2E217D
:10B2200006F0CCFEB87906F0FFFD7A7A0E2106F022
:10B23000C5FEAB593B491A688B4222F040021A60A6
:10B240004ED0394A934255D0384A93425DD0384A5D
:10B2500093423AD0374A934209D102F56842516A83
:10B2600041F480115162516A21F480115162D82257
:10B27000596802FB045441F48051A27B5960002AB2
:10B28000196814BF0024022449060FD41D6882F0F7
:10B290000102294829492840024342F445722243C9
:10B2A0001A605A68114041F4E0615960DA6922F489
:10B2B0000062DA611A6842F040021A60F8BDDA7979
:10B2C00038462E2106F07AFEA1E702F58232516A55
:10B2D00041F400515162516A21F400515162C6E7B4
:10B2E000174A516A41F480515162516A21F48051E8
:10B2F0005162BCE702F50032116A41F480411162EB
:10B30000116A21F480411162B1E702F5FE32116A3F
:10B3100041F400411162116A21F400411162A6E773
:10B320001C8201200030014000380040003C0040F9
:10B3300000340140005001404000FFFFFBF0FFFFE0
:10B340000038024070B5C0EBC000104C104E82B007
:10B3500004EB8004306B256928433063366B94F925
:10B360000D003540A160636191090195019B27F0B3
:10B3700073FD94F90D300122064903F01F005B09AB
:10B38000824041F8232002B070BD00BF142101208B
:10B390000038024000E100E02DE9F0475C4C82B04B
:10B3A00054F82040002C00F08E80D4F890514FF4D7
:10B3B000007704F5CB7CDFF86C816E6804F2963E72
:10B3C000A1602969C4F88861C4F80080C4F814C079
:10B3D000C4F818E0E760276121B1AF68C4F8F41041
:10B3E000C4F8FC709846EB6891460746002B00F0C5
:10B3F0008D80AA684FF00B0CC4F8F8307E1CC4F89E
:10B40000002195F823004349C0EBC002424B01EBF9
:10B410008201D3F830E00A6942EA0E0EC3F830E048
:10B42000D3F830E023464E7602EA0E0281F818C0C7
:10B430003A49019295F82520019EFFF783FFD4F841
:10B4400088616A6806F128032436C4F81821C4F814
:10B450001031C4F8146194F8950106F0E5FC064635
:10B4600094F8940106F0E0FC331C824618BF0123D7
:10B4700018F0080F2BD053B318F0110F07F1010784
:10B480004FF00B033046F77118BF4A21B37108BF64
:10B490003A2195F8222006F091FDD4F8FC3093B9BA
:10B4A00095F8261095F92400890927F0D5FC95F820
:10B4B000243001211A485AB203F01F03520901FA3D
:10B4C00003F340F82230204602B0BDE8F08719F0BF
:10B4D000020F09D043B10B227B1C3046B271F371CD
:10B4E00095F8221027F09AFEBAF1000FD5D019F086
:10B4F000010FD2D001370C2350468AF807708AF822
:10B50000063095F8221027F089FEC6E7324699E703
:10B51000404D0120142101200038024069950008A7
:10B5200000E100E000F603080348D0F8AC3113B1A5
:10B5300000F5D27018477047142101200348D0F855
:10B54000903113B100F5C4701847704714210120E1
:10B550000348D0F8743113B100F5B670184770473E
:10B56000142101200348D0F8583113B100F5A87018
:10B5700018477047142101200348D0F83C3113B11B
:10B5800000F59A7018477047142101200348D0F83D
:10B59000203113B100F58C70184770471421012039
:10B5A0000348D0F804310BB1FC301847704700BF96
:10B5B000142101200348D0F8E8300BB1E0301847DF
:10B5C000704700BF142101200348D0F8CC300BB1E4
:10B5D000C4301847704700BF142101200348D0F839
:10B5E000B0300BB1A8301847704700BF14210120BC
:10B5F0000348D0F894300BB18C301847704700BF27
:10B60000142101200248836F0BB170301847704736
:10B61000142101200248C36D0BB154301847704704
:10B62000142101200248036C0BB1383018477047D1
:10B63000142101200248436A0BB11C30184770479F
:10B64000142101200248836803B11847704700BFE6
:10B6500014210120A54A0021A54BA64870B5D2F8B7
:10B6600088404FF00065A44EA4B044F47004C2F8C2
:10B6700088401C6844F001041C6099601C682040EC
:10B6800018605E60186820F480201860D9609560AA
:10B69000BFF34F8FBFF36F8FC2F85012516941F45F
:10B6A00000315161BFF34F8FBFF36F8F196C934A15
:10B6B00041F080511964196C01F080510291029996
:10B6C000116841F440411160126802F44042019255
:10B6D000019A9A6802F00C02042A52D09A6802F089
:10B6E0000C02082A4AD0824B854C1A68194642F44B
:10B6F00080321A60226803E023689B1A642B3CD8CE
:10B700000B689803F8D57A4B9A6802F00C02082A65
:10B7100033D01A68184622F080721A60226803E05B
:10B7200023689B1A022B28D803689B01F8D447F69C
:10B73000C07393FAA3F34FF44031B3FA83F291FA52
:10B74000A1F14FF0706191FAA1F10926B1FA81F1EE
:10B750004FF4D8736B4D8E406549934033431D437E
:10B760004560036843F08073036022680B689E01A4
:10B770000BD423689B1A022BF8D9FEE75B685C02A6
:10B78000B1D55B4B5E4C1B68BDE7086C5B4A40F073
:10B79000805013460864096C01F0805103910399AD
:10B7A000116841F48031116021685A68D50305D4CD
:10B7B0002268521AB2F57A7FF7D9FEE71A684F4924
:10B7C00042F400321A60226804E023689B1AB3F541
:10B7D0007A7FF2D84B689803F7D54FF400164FF0F4
:10B7E00000654FF4C0710722032304A80496219535
:10B7F000089109920A9332F085F900B1FEE7424AB6
:10B80000136803F00F03062B1BD9394B9A6822F0FB
:10B81000F0029A601A68920167D59A68184641F258
:10B82000883122F0030242F002029A6022688368A3
:10B8300003F00C03082B10D023689B1A8B42F6D917
:10B840000AE0136823F00F0343F007031360136843
:10B8500003F00F03072BD8D0FEE72B4A136803F041
:10B860000F03072B35D8224CA36823F4E05343F48D
:10B87000A053A360A36823F4604343F40043A36090
:10B880001AF094FAA368F02292FAA2F2B2FA82F2C3
:10B8900003F0F0031D4ED3401D4D334493F8483060
:10B8A00020FA03F32B6027F00BFB0023194A04A8AE
:10B8B0000492139314931593169317931893199353
:10B8C0001A931B931C931D931E9332F01BF918B30C
:10B8D000FEE7136823F00F0343F0070313601368B8
:10B8E00003F00F03072BB7D1BDE7B5E700ED00E08C
:10B8F00000380240FFFFF6FE1030002400700040C8
:10B90000E893012008004020003C0240E0F50308D5
:10B9100094200120C0FF0300D4F88C3023F0807302
:10B92000C4F88C30D4F88C3043F08073C4F88C3079
:10B93000A36803F00C03042B27D0082B0DD0154B64
:10B94000154A16499268C2F30312164496F8482025
:10B95000D3408B422B601AD0FEE7616862684B02CD
:10B96000616802F03F024CBF0D4B0A4BB3FBF2F390
:10B97000C1F3881203FB02F3074A5268C2F3014283
:10B9800001325200B3FBF2F3DAE7054BD8E724B0FB
:10B9900070BD00BF0024F4000038024000E6DF0C58
:10B9A00000127A00831E00F14E02EA2123F8021FE2
:10B9B0009342FBD140F6491300224385012380F8CE
:10B9C000632080F85E3080F85F3080F8603080F867
:10B9D000613080F8623080F8643080F8693080F837
:10B9E000673080F855304FF6FF7380F86520A0F877
:10B9F0005A304FF4206380F86820A0F8563040F6A3
:10BA0000012380F8662080F86A2040F69802A0F8AA
:10BA100058301423A0F85020642280F8543080F865
:10BA20005C302823A0F8522080F85D307047054B29
:10BA300093F855302BB94FF4A4735843642390FB0B
:10BA4000F3F07047FE5401200E4B1B78022B17D0E9
:10BA50000D4A5378127803EB830302EB82025B00FA
:10BA6000C01AC3EB4203C0EBC00090FBF3F0062802
:10BA7000A8BF062020EAE070C0F19600C0B270476F
:10BA8000972070477D5C0120F4780120034B93F8E8
:10BA90005530002B0CBF0F200C207047FE540120A6
:10BAA00013B5947813780194527800920A460249AB
:10BAB00007F09EFB02B010BD9027040873B5642404
:10BAC00006460846FFF7B3FF104B1149054690FBA9
:10BAD000F4F4002CB8BF64420028B8BF6442002AC6
:10BAE00008BF1946FFF7D2FF64220090304695FB4D
:10BAF000F2F302FB13530A2293FBF2F3002B2246CC
:10BB0000B8BF5B4207F074FB02B070BDAA270408FF
:10BB10009F27040870B50B4C054616460B46024697
:10BB20000221206806F08AFB2A46074B1421206870
:10BB300006F084FB33462A4620681621BDE8704093
:10BB400006F07CBB804D01209C4D0408012806D0E6
:10BB500003D3022806D00020704705F0E9BE034B4E
:10BB600018687047014B5868704700BFE4240120F3
:10BB70001C4B37B503EB42020446B2F8565005F0B1
:10BB80000F0039B1621CD0B102288CBF20239C2346
:10BB900023701446FFF7DAFF13493C23C5F303155E
:10BBA000B0FBF1F191FBF3F2012D03FB121308D06E
:10BBB0000E49204603B0BDE8304007F019BB9B2377
:10BBC000E6E742F210716425B0FBF1F0B0FBF5F14D
:10BBD00005FB110006490090204607F009FB03B061
:10BBE00030BD00BFFE54012040420F00B4270408BE
:10BBF000BE27040830B585B0054601A807F0EAF86D
:10BC0000044618B92870204605B030BD044A012307
:10BC100001A92846B2F9002007F002FBF3E700BFB4
:10BC2000A87001202DE9F84F01228F4B8F490A702F
:10BC30001A6822F040021A601A6822F0380242F0B4
:10BC400010021A601A6842F040021A60884B1968A4
:10BC500019B18B880A681B04936140F2E93382486A
:10BC600002E0002B00F04C818268013B12F0020FD1
:10BC70009BB2F6D0802240F2E9337B4C027302E0A3
:10BC8000002B00F03D81A268013B12F0010F9BB236
:10BC9000F6D0E36840F2E933734802E0002B00F08D
:10BCA00039818268013B12F0020F9BB2F6D000226C
:10BCB00040F2E9336C4C027302E0002B00F02A8161
:10BCC000A268013B12F0010F9BB2F6D0E068C0B24F
:10BCD00011B10B688A889A61634B664C1A68664D8D
:10BCE00022F040021A601A6822F038021A601A68BC
:10BCF00042F040021A6022782C6882423FD05F4EA8
:10BD0000FDF7EEFD5E4B0020F28B4FF0050BB3F814
:10BD100000A00346DFF87491B71819F802505C1DB3
:10BD200002F1010E97F820C0F1184FEA12283444AE
:10BD3000AC4513D081F803224FF0060C4FF00702F8
:10BD40000633013081F800B281F8018281F802C225
:10BD500081F8042287F8205084F800521FFA8EF2EE
:10BD60000130524580F094806328D5DDF283002BAA
:10BD700040F0938000233D4A1370BDE8F88F41489E
:10BD80003E4E00780028BDD17069201AB0F57A7F48
:10BD9000B8D9186820F040001860186820F0380002
:10BDA00040F010001860186840F04000186019B1A9
:10BDB00088880B680004986140F2E9332A4F02E05A
:10BDC000002B00F0CD80B868013B10F0020F9BB251
:10BDD000F6D0A02040F2E9333873234F02E0002B65
:10BDE00000F0BE80B868013B10F0010F9BB2F6D0A6
:10BDF000FB6840F2E9331C4F02E0002B00F0BA80F0
:10BE0000B868013B10F0020F9BB2F6D0002040F260
:10BE1000E9333873144F02E0002B00F0AB80B868B0
:10BE2000013B10F0010F9BB2F6D0F868C0B211B11F
:10BE30000B68898899610C4B134F196821F04001F8
:10BE40001960196821F038011960196841F0400142
:10BE500019603B78182B00F09880410765D50023C6
:10BE6000B36174614EE700BF0038004029740120BF
:10BE7000FC880120B61B01202CB90120E4240120FC
:10BE8000B41B012000890120C88001201472012008
:10BE90000022F283002B3FF46DAF464A116821F077
:10BEA00040011160116821F0380141F0100111606A
:10BEB000116841F0400111603F4A12681AB191883F
:10BEC00010680904816100223C493A48FEF7CAFF24
:10BED000394B1B6813B11A689B889361354B1A68FC
:10BEE00022F040021A601A6822F038021A601A68BA
:10BEF00042F040021A600023314A1370BDE8F88F07
:10BF0000304AB2F8E43001339BB2A2F8E430B2F820
:10BF1000E430BFE62B4AB2F8E43001339BB2A2F81A
:10BF2000E430B2F8E400C0B2D2E600F00500012827
:10BF30003AD0002895D1530693D5B2692B68002AD0
:10BF400035D09B1A642B8CD9FDF7CAFC3B78182B93
:10BF500087D1B38B1C4A01339BB2B383938080E7B4
:10BF60001848B0F8E43001339BB2A0F8E430B0F8E0
:10BF7000E4303EE71348B0F8E43001339BB2A0F858
:10BF8000E430B0F8E400C0B251E702F040030E49DB
:10BF900000F0070E002B0B807346A1F802E014BFDF
:10BFA00010230D23CB8058E75206C6D559E7B3615D
:10BFB00057E700BF00380040FC880120E42601203C
:10BFC000297401201C820120CC800120AC4B01226D
:10BFD000AC492DE9F043DFF8C4E2D1F800908EF8C7
:10BFE00000201A6822F040021A601A6822F0380213
:10BFF00042F010021A601A6842F040021A60B9F169
:10C00000000F05D0B9F80430D9F800201B04936163
:10C0100040F2E9339A4902E0002B00F09F818A68E0
:10C02000013B12F0020F9BB2F6D0052240F2E93339
:10C0300093480A7302E0002B00F090818268013B74
:10C0400012F0010F9BB2F6D0C36840F2E9338C497D
:10C0500002E0002B00F0DC818A68013B12F0020F45
:10C060009BB2F6D0002240F2E93385480A7302E021
:10C07000002B00F0CD818268013B12F0010F9BB2D2
:10C08000F6D0C36840F2E9337D4902E0002B00F0AE
:10C09000B5818A68013B12F0020F9BB2F6D00622EE
:10C0A00040F2E93376480A7302E0002B00F0A681E3
:10C0B0008268013B12F0010F9BB2F6D0C36840F2D8
:10C0C000E9336F4902E0002B00F08E818A68013B62
:10C0D00012F0020F9BB2F6D0002240F2E93368481A
:10C0E0000A7302E0002B00F07F818268013B12F0AE
:10C0F000010F9BB2F6D0C368634A40F2E93360494E
:10C1000092F858C44CF0010002E0002B00F062816C
:10C110008A68013B12F0020F9BB2F6D0042240F273
:10C12000E933574C0A7302E0002B00F05381A268F8
:10C13000013B12F0010F9BB2F6D0E36840F2E93305
:10C140004F4902E0002B00F03B818A68013B12F06E
:10C15000020F9BB2F6D0087340F2E933484902E07F
:10C16000002B00F02D818A68013B12F0010F9BB279
:10C17000F6D0CB68454B1D88002D42D04449072698
:10C1800044480D443E4A444C91F8018040F2E93362
:10C1900002E0002B00F0D0809768013B17F0020FFF
:10C1A0009BB2F6D0167340F2E93302E0002B00F0A8
:10C1B000C3809768013B17F0010F9BB2F6D0D3689C
:10C1C00040F2E93302E0002B00F0BF809768013BAA
:10C1D00017F0020F9BB2F6D082F80C8040F2E933E0
:10C1E00002E0002B00F0B1809768013B17F0010FCF
:10C1F0009BB2F6D0D36811F8013F8D4200F8013FA1
:10C20000C2D140F2E9331E4902E0002B00F0CE809B
:10C210008A68013B12F0020F9BB2F6D0072240F26F
:10C22000E93317480A7302E0002B00F0BF808268F0
:10C23000013B12F0010F9BB2F6D0C36840F2E93324
:10C240000F4902E0002B00F0A7808A68013B12F042
:10C25000020F9BB2F6D0FF2240F2E93308480A737E
:10C2600002E0002B00F098808268013B12F0010F81
:10C270009BB2F6D0C36840F2E933014912E000BF37
:10C2800000380040FC880120E4240120B41B012078
:10C2900013720120032501201C8201202974012032
:10C2A000002B6FD08A68013B12F0020F9BB2F7D0CF
:10C2B000042240F2E9335B480A7301E0002B61D0AD
:10C2C0008268013B12F0010F9BB2F7D0C36840F2C5
:10C2D000E933544901E0002B4AD08A68013B12F04F
:10C2E000020F9BB2F7D081F80CC040F2E9334D4900
:10C2F00001E0002B3CD08A68013B12F0010F9BB299
:10C30000F7D0CB68B9F1000F04D0D9F80030B9F8F4
:10C3100004209A61434B00211A6822F040021A60FF
:10C320001A6822F038021A601A6842F040021A6055
:10C330008EF80010BDE8F083B4F8E43001339BB20E
:10C34000A4F8E430B4F8E4303AE7B4F8E430013368
:10C350009BB2A4F8E430B4F8E4304CE7324AB2F8C7
:10C36000E43001339BB2A2F8E430B2F8E4306CE67A
:10C370002D4AB2F8E43001339BB2A2F8E430B2F8AF
:10C38000E430BFE7284AB2F8E43001339BB2A2F8A8
:10C39000E430B2F8E4309AE7234AB2F8E4300133EB
:10C3A0009BB2A2F8E430B2F8E43064E71E4AB2F877
:10C3B000E43001339BB2A2F8E430B2F8E4303DE758
:10C3C000194AB2F8E43001339BB2A2F8E430B2F873
:10C3D000E430CFE6144AB2F8E43001339BB2A2F85D
:10C3E000E430B2F8E430A9E60F4AB2F8E4300133A1
:10C3F0009BB2A2F8E430B2F8E4307DE60A4AB2F823
:10C40000E43001339BB2A2F8E430B2F8E43056E6EF
:10C41000054AB2F8E43001339BB2A2F8E430B2F836
:10C42000E4302FE6003800401C8201202DE9F0475F
:10C43000DFF8D0A29AF8003003B1FEE7AC4B01223E
:10C44000AC4C8AF800201A68D4F800C022F04002F0
:10C450001A601A6822F0380242F010021A601A6854
:10C4600042F040021A60BCF1000F05D0BCF8043065
:10C47000DCF800201B0493619F4A012540F2E93358
:10C480009B4C157002E0002B00F0BF81A268013BBD
:10C4900012F0020F9BB2F6D0002240F2E933944D25
:10C4A000227302E0002B00F0B081AA68013B12F079
:10C4B000010F9BB2F6D0EB6840F2E9338C4C02E0FE
:10C4C000002B00F0D481A268013B12F0020F9BB256
:10C4D000F6D0002240F2E933854D227302E0002BB2
:10C4E00000F0C581AA68013B12F0010F9BB2F6D0A3
:10C4F000EB6840F2E9337E4C02E0002B00F0AD81A6
:10C50000A268013B12F0020F9BB2F6D0092240F262
:10C51000E933774D227302E0002B00F09E81AA6878
:10C52000013B12F0010F9BB2F6D0EB6840F2E93309
:10C530006F4C02E0002B00F08681A268013B12F0F4
:10C54000020F9BB2F6D0207340F2E933684802E054
:10C55000002B00F078818268013B12F0010F9BB242
:10C56000F6D0C368654A4D1E614B002114684FF038
:10C570000A0E63480B265FFA81F840F2E93202E0C6
:10C58000002A00F00B819F68013A17F0020F92B267
:10C59000F6D083F80CE040F2E93202E0002A00F025
:10C5A000FD809F68013A17F0010F92B2F6D0DA6869
:10C5B00040F2E93202E0002A00F0F9809F68013A77
:10C5C00017F0020F92B2F6D083F80C8040F2E932F5
:10C5D00002E0002A00F0EB809F68013A17F0010F9B
:10C5E00092B2F6D0DA6815F8018F40F2E93202E033
:10C5F000002A00F0E5809F68013A17F0020F92B21E
:10C60000F6D01E7340F2E93202E0002A00F0D88032
:10C610009F68013A17F0010F92B2F6D0DA6840F243
:10C62000E93202E0002A00F0D4809F68013A17F056
:10C63000020F92B2F6D083F80C8040F2E93202E0A9
:10C64000002A00F0C6809F68013A17F0010F92B2ED
:10C65000F6D0DA6844B12768A288D7F8149012EAB5
:10C66000090F18BF1204BA610131362983D140F293
:10C67000E9331F4902E0002B00F0DB808A68013BB0
:10C6800012F0020F9BB2F6D0082240F2E9331848AC
:10C690000A7302E0002B00F0CC808268013B12F0AC
:10C6A000010F9BB2F6D0C36840F2E933104902E0B3
:10C6B000002B00F0B4808A68013B12F0020F9BB29D
:10C6C000F6D0A02240F2E93309480A7302E0002BB9
:10C6D00000F0A5808268013B12F0010F9BB2F6D0FA
:10C6E000C368034AA0240649002040F2E9330DE064
:10C6F00000380040FC88012031740120F8B8012086
:10C700001C82012029740120002B6BD09568013B0D
:10C7100015F0020F9BB2F7D0147340F2E93301E039
:10C72000002B5FD09568013B15F0010F9BB2F7D04D
:10C73000D36840F2E93301E0002B5CD09568013BFF
:10C7400015F0020F9BB2F7D0107340F2E93301E00D
:10C75000002B50D09568013B15F0010F9BB2F7D02C
:10C76000D368DBB29B06C0D4BCF1000F04D0DCF868
:10C770000030BCF804209A61424B00211A6822F074
:10C7800040021A601A6822F038021A601A6842F0F1
:10C7900040021A608AF80010BDE8F087B0F8E42083
:10C7A000013292B2A0F8E420B0F8E42000E7B0F83B
:10C7B000E420013292B2A0F8E420B0F8E42012E7BD
:10C7C000B0F8E420013292B2A0F8E420B0F8E420FE
:10C7D00025E7B0F8E420013292B2A0F8E420B0F8E6
:10C7E000E42037E7B1F8E43001339BB2A1F8E4303C
:10C7F000B1F8E4309DE7B1F8E43001339BB2A1F821
:10C80000E430B1F8E430DBB2ACE71F4AB2F8E43010
:10C8100001339BB2A2F8E430B2F8E4304CE61A4A95
:10C82000B2F8E43001339BB2A2F8E430B2F8E4305D
:10C8300057E7154AB2F8E43001339BB2A2F8E4306E
:10C84000B2F8E43030E7104AB2F8E43001339BB27A
:10C85000A2F8E430B2F8E43084E60B4AB2F8E430EF
:10C8600001339BB2A2F8E430B2F8E4305EE6064A47
:10C87000B2F8E43001339BB2A2F8E430B2F8E4300D
:10C8800037E600BF003800401C82012030B4147825
:10C890007CB11E23084D13FB0101801A2944831823
:10C8A00001311D2BD8BF01F8014C12F8014F002CAB
:10C8B000F5D130BC704700BF147201203B4BC1F171
:10C8C00003011A6841EA800122F04002F0B41A60C4
:10C8D000CDB21A68364C22F03802266842F01002B7
:10C8E0001A601A6842F040021A601EB1B3883268BA
:10C8F0001B04936110202D4A2E4CC7B240F2E9333D
:10C9000001E0002B3FD09168013B11F0020F9BB278
:10C91000F7D0177340F2E93301E0002B33D0916870
:10C92000013B11F0010F9BB2F7D0D36840F2E9331D
:10C9300001E0002B30D09168013B11F0020F9BB257
:10C94000F7D0157340F2E93300E02BB39168013B57
:10C9500011F0010F9BB2F8D0D36801302028CCD160
:10C9600016B13368B2889A61104B1A6822F04002FF
:10C970001A601A6822F038021A601A6842F04002FF
:10C98000F0BC1A607047B4F8E43001339BB2A4F8ED
:10C99000E430B4F8E430C9E7B4F8E43001339BB2D2
:10C9A000A4F8E430B4F8E430D7E700BF0038004022
:10C9B000FC8801201C8201203E4A30B492F8585471
:10C9C00000285FD105F0F7053B4B82F858541A68F0
:10C9D0003A4922F0400208681A601A6822F03802C8
:10C9E00042F010021A601A6842F040021A6018B150
:10C9F000838802681B04936140F2E9332E4901E009
:10CA0000002B4CD08A68013B12F0020F9BB2F7D08A
:10CA1000042240F2E933284C0A7301E0002B3ED097
:10CA2000A268013B12F0010F9BB2F7D0E36840F21D
:10CA3000E933214900E043B38A68013B12F0020F59
:10CA40009BB2F8D00D7340F2E9331B4900E0E3B12B
:10CA50008A68013B12F0010F9BB2F8D0CB6810B18D
:10CA6000036882889A61144B1A6822F040021A60A7
:10CA70001A6822F038021A601A6842F0400230BC8C
:10CA80001A60704745F008059EE70D4AB2F8E43099
:10CA900001339BB2A2F8E430B2F8E430DFE7084A91
:10CAA000B2F8E43001339BB2A2F8E430B2F8E430DB
:10CAB000BDE700BFE424012000380040FC880120CD
:10CAC0001C820120A74A2DE9F04F32F8104091B0A6
:10CAD0000646230540F1708206F01F01012340093C
:10CAE0008B40A14951F820100B4204D09F4B1B787A
:10CAF000002B40F0618204F01F05C4F34414272E7C
:10CB000000F25A82DFE816F028003700F001080230
:10CB10005B020701070181019E01B801D6015200A5
:10CB2000630075006B00010184028B0293029B027B
:10CB3000A902B302580382008200720382038203B7
:10CB40009F03E703A400D200F1030904E5002404D5
:10CB500030040D013C044104854B08A885491A881E
:10CB60006423534301229B12632BA8BF632306F067
:10CB70003FFB08AB5BE1804B0A211E887F4B01FB2A
:10CB800006F01B7890FBF3F0FEF75EFF8DF82000B7
:10CB90000DF12100B6FBF1F201FB1263062192B206
:10CBA00000919BB2764906F023FBE2E7754B6421C6
:10CBB0009A201B68009008A8002BB8BF5B4293FB2B
:10CBC000F1F201FB1233704906F012FBD1E76D4A16
:10CBD00007236E4908A8926806F00AFBC9E76C4B68
:10CBE0001E226C4908A81B7D00931F2306F000FB42
:10CBF000BFE7674B08A86849DA89242353434FF4F9
:10CC00007A7293FBF2F206F0F3FAB2E7604B182E59
:10CC1000624903A893E8840012BF60236423174687
:10CC20005F4A8DF8203097FBF2F206F0E1FA3A46BF
:10CC30005A4905A806F0DCFA03A830F097F805ABCE
:10CC400003AA584903440DF1210006F0D1FA90E7F8
:10CC5000554B1B7803F00303032B23D1534B1B8845
:10CC6000E3B1534A0A21534BB2F90420B3F900301F
:10CC700092FBF1F29B1A4FF4B4721B0103F5B95306
:10CC80001433B3FBF2F3C3F1080303F00F03603373
:10CC90008DF8203000238DF821306AE705238DF8C8
:10CCA0002030F7E72D238DF82030F3E73E4B1B783B
:10CCB00003F00303032BF5D13C4B1888FEF7B7FEB6
:10CCC0000246FEF7E3FE3C49034608A806F090FA48
:10CCD0004FE7374B0A22B3F9043093FBF2F31B0101
:10CCE0004FF4B47203F5B9531433B3FBF2F3334A80
:10CCF00003F00F03134408AA186859681B7A03C28B
:10CD0000137000238DF8293033E70122002108A891
:10CD1000FEF7D4FE2DE7721F012108A8FEF728FFB9
:10CD200027E7184B9FED267A9968B2F8503007EE46
:10CD3000901AF8EEE76A07EE903AF8EEE77A67EEB7
:10CD4000877AF4EEE76AF1EE10FA04D51D4908A8D7
:10CD500006F04EFA0DE78B4238DA1B4908A806F0B8
:10CD600047FA06E7FE5401201C740120010001204F
:10CD70007A5C012000280408D4810120EA81012086
:10CD8000E42704082C770120ED270408F82704087D
:10CD9000589F0120FE270408052804086D61040837
:10CDA000809698000A2804085E790120687901209D
:10CDB00008790120385E01201028040838F603089D
:10CDC000CDCCCC3D152804081B2804085B1AB74AB3
:10CDD0003C2108A807EE903AB54BB8EEE77AD3EDC0
:10CDE000007AF8EE677A67EE277A87EEA67AFDEE8C
:10CDF000C77A17EE903AB3FBF2F393FBF1F201FB23
:10CE00001233AC4906F0F4F9B3E624F0C9FAAA4AA1
:10CE1000AA4B002808BF1346A94A128857050DD40B
:10CE2000D6070DD412F0020FA64A18BF1346A64823
:10CE300022462946006805F001FABDE0A34BF6E75B
:10CE4000A34BF4E7A34F0DF120083A7822B9A24989
:10CE5000404632F07BFB8CE6002617F806904846E9
:10CE600006F038F808F80600B9F1000F3FF481AE7B
:10CE70000136102EF1D17CE6042398490DF12200F1
:10CE80008DF8203005238DF82130954BB3F906201D
:10CE90000A23B2F5FA6FA8BF4FF4FA62B2F57A7FAF
:10CEA000B8BF4FF47A72A2F57A7292FBF3F206F0F1
:10CEB0009FF95EE68B498C4A0B78D65C8B4B4A789F
:10CEC00053F822708B788DF814300B7A13B105A8C3
:10CED00020F010FF9DF814303246854908A80093D1
:10CEE0003B4606F085F944E6774B0D25186805F0BA
:10CEF000C9F92623B0F5F07F8DF820304FF07E037E
:10CF00000CBF072406248DF8213027238DF822300A
:10CF100000238DF823302CE692F85D3092F85C50B7
:10CF200003EB8303734A05EB85055B00B2F9001040
:10CF30006D005F42B94203DB8B42A8BF0B461F4620
:10CF4000B2F90230C5F100094B4503DBAB42A8BF83
:10CF50002B4699465C4C4FF0400A4FF0090B206875
:10CF6000A046192405F08EF9B0F5F07F04FB09F412
:10CF70004FEA870918BF022694FBF5F40A25293CDD
:10CF800099FBFAF31B1B512B0DD8D8F8000093FB2B
:10CF9000FBF202EBC20132445B1AD2B22946803B5B
:10CFA000DBB205F041F90135A9EB0709EDB2132D0C
:10CFB000E6D10420FFF786FD11B0BDE8F08F424CAA
:10CFC0006FF00205206805F05DF9B0F5F07F0CBF49
:10CFD000072706277E19132307212068F6B201359B
:10CFE000324605F021F9132332461521206805F059
:10CFF0001BF9042DEED13A4603230821206805F0E1
:10D0000013F902233A461421206805F00DF9D3E7FD
:10D01000394B08A839491A68FEF742FDA9E5364B95
:10D0200008A837491A680332FEF73AFDA1E5324BEA
:10D0300008A834491A680632FEF732FD99E5324BEA
:10D0400008A832491A88324B1B6853434FF47A724E
:10D0500093FBF2F206F0CCF88BE52E4A08A82E4995
:10D06000537812780133013206F0C2F881E5B2F844
:10D070005A702A4B38071E7806D5022E04D128494B
:10D0800008A806F0B5F874E5B9064DD5232024F0BC
:10D090003BF9002848D0232024F092F9002843D0FF
:10D0A000204908A806F0A4F863E500BF40420F003D
:10D0B000E4240120B4270408CD270408D22704085B
:10D0C0005C790120E0270408804D0120D627040860
:10D0D000DB270408AC700120212804086D610408D6
:10D0E000CC5C01203C810120461D0408501D040831
:10D0F0002C280408087901206079012035280408CB
:10D10000392804083D280408D48101204128040856
:10D110002C770120149F0120462804087D5C012003
:10D120004C28040856280408FA0718D5002024F0D3
:10D1300047F9A0B19A4B1A688AB10023012101FA7C
:10D1400003F0104207D0974A08A8974952F82320C5
:10D1500006F04EF80DE50133112BF0D109E57B0700
:10D1600006D5012E04D1914908A806F041F800E542
:10D17000B80713D58E4B1B7899070FD476B98D4A13
:10D180008D4B11781B888D4A93FBF1F3927B9A4269
:10D1900004D98B4908A806F02BF8EAE4FA067FF5D3
:10D1A0000BAF884B93F85934002B3FF405AF8649F9
:10D1B00008A806F01DF8DCE47F4B0A211B885943C0
:10D1C0007C4B1B7891FBF3F10846FEF73DFC642392
:10D1D0008DF82000062091FBF3F200900DF1210064
:10D1E00003FB1213794906F003F8C2E47849B1F958
:10D1F0000600B1F90230B1F90020019008A8B1F998
:10D2000004100091734905F0F3FFB2E41A2E724B3B
:10D210004FF00A010CBFB3F90200B3F9000090FB14
:10D22000F1F3002801FB130108A8ACBF20222D2236
:10D230000029B8BF4942002B0091B8BF5B42674943
:10D2400005F0D6FF95E45D4B8B261A89644B9B68ED
:10D25000D31A9342A8BF134623EAE37307EE903A2A
:10D260000B23B2FBF3F207EE102AF8EEE77AB8EEE2
:10D27000C77AC7EE876A16EE900A2FF0E3FE41ECFC
:10D28000100B31F0E5F851EC100B30F0C9F98A239E
:10D29000C0B20DF121028DF820308D21012398427A
:10D2A00003F1010302F10102DBB22CBF02F8016CB1
:10D2B00002F8011C0C2BF2D18F238DF82C30431E69
:10D2C000092B04D810AB18448E2300F81F3C002310
:10D2D0008DF82D304DE4364B1B78DB073FF56CAEF7
:10D2E000404908A805F084FF43E43B4B0A224FF471
:10D2F000B47108A8B3F9043093FBF2F31A0102F5F4
:10D30000B9521432B2FBF1F2C2F10802364902F00E
:10D310000F02603205F06CFF2BE40020FEF787FB64
:10D3200064210A2290FBF1F301FB130191FBF2F15E
:10D330000029B8BF4942002B0091B8BF5B422B497E
:10D340000028ACBF6822602208A805F051FF10E455
:10D350001C4BD3F85C240AB192F901200E23244916
:10D3600008A805F045FF04E4164BD3F85C240AB185
:10D37000B2F908201F4908A805F03AFFFFF7F9BBEA
:10D3800008A8FEF737FCFFF7F4BB1B4B08A81B4AA5
:10D390001B6812681A4905F02BFFFFF7EABB00BFB4
:10D3A0005879012058FD0308314A0408612804080F
:10D3B00034810120EA810120D4810120F478012008
:10D3C0006D280408E42401207B280408B52F0408F4
:10D3D000CC800120852804080879012099280408B8
:10D3E0002C770120A5280408AE280408B5280408D5
:10D3F000102804086D61040804000120202A01207F
:10D40000C1280408694B2DE9F04F1B788BB0074603
:10D41000674C13B1012384F85934D4F86024531CA9
:10D42000C4F860340523B2FBF3F303EB8303D21A91
:10D4300040F062835F486049037880460D788946F2
:10D4400003F001039D4222D0002B00F0A1804FF495
:10D45000FA735A4DA2816381632328682281E38194
:10D4600022826282626004F011FF554B07220C2178
:10D47000286804F0E3FE07F5F423524A03F590739D
:10D48000136098F8003003F0010389F800304E4B28
:10D4900064224E4E1B885A434D4BD9892423C2F334
:10D4A00087224B434FF47A7184F8642493FBF1F3A1
:10D4B000B4F908101BB29942B4F90A10B8BF23811D
:10D4C000444B1B8899424FF06401C8BF63813368A5
:10D4D00093FBF1F3B4F90C101BB29942B8BFA381CE
:10D4E000B4F90E309342B4F91030C8BFE281002B7A
:10D4F00001DA00232382384A1378914603F00303AC
:10D50000032B06D1354BB4F912201B889A42B8BFC1
:10D51000638298F80030DA0708D5D4F868342268B6
:10D52000FB1A1A442260626813446360DFF8948037
:10D53000C4F86874D8F800304146204D002B00F044
:10D540008481FB1A002B80F27A81254A40F2D6634F
:10D55000B2F90600984203DCB2F902209A4201DDDA
:10D5600000230B60286804F05BFE002384F8593424
:10D57000124B1B6823B193F90E30002B00F3D382BA
:10D58000184A136823F4005313600BB0BDE8F08F02
:10D59000DFF854A0564603EB0A0292F85E20002AF8
:10D5A00040F0B08201330D2BF5D16AE7A45C012075
:10D5B000E424012034810120844D0120804D01208C
:10D5C000A8280408247401207A5C01202C7701200B
:10D5D000589F0120D48101205E79012068790120C3
:10D5E000CC5C012058790120FE54012002A8FEF7EE
:10D5F00001FB18B9AB4902A805F0FAFD286804251B
:10D6000002AB0322022104F019FE96F86630A3B1A2
:10D61000002202A805F1010A1146FEF7A9FAB6F8A0
:10D6200056305FFA8AFAA04903F00F0328465546A0
:10D6300002AA51F82310FEF76DFA96F86730A3B1ED
:10D640000122002102A805F1010AFEF791FAB6F8BD
:10D6500058305FFA8AFA944903F00F03284655467A
:10D6600002AA51F82310FEF755FA96F85E3093B1EE
:10D670008E4B1B7899070ED505F1010A02A9B4F962
:10D6800008005FFA8AFA25F0ADFE2846554602AA40
:10D690008749FEF73FFA96F86830ABB105F1010A09
:10D6A000B4F91200FEF7C3F902465FFA8AFAFEF7F0
:10D6B000EDF98049034602A805F09AFD2846554633
:10D6C00002AA7D49FEF726FA96F85F30BBB1B4F99D
:10D6D0000A100A2305F1010A02A891FBF3F203FBE9
:10D6E000121306215FFA8AFA00911BB2734905F002
:10D6F0007FFD2846554602AA7149FEF70BFA96F8B7
:10D700006530C3B16F4B05F1010A02A819880A23DD
:10D710005FFA8AFAB1FBF3F203FB1213062192B20D
:10D7200000919BB2654905F063FD2846554602AA63
:10D730006549FEF7EFF996F8603093B105F1010AFB
:10D7400002A9B4F90E005FFA8AFA25F04BFE5F4990
:10D7500002A831F0DEFE2846554602AA5C49FEF7D3
:10D76000D9F95C4B9B794BB396F8613093B105F1D5
:10D77000010A02A9B4F90C005FFA8AFA25F032FE18
:10D78000554902A831F0C5FE2846554602AA53491C
:10D79000FEF7C0F996F8623083B105F1010A504AEC
:10D7A000072344495FFA8AFA926802A805F020FD2F
:10D7B0002846554602AA4B49FEF7ACF996F8633065
:10D7C0007BB105F1010A0022B4F9101002A85FFA3A
:10D7D0008AFAFEF773F92846554602AA4249FEF72F
:10D7E00099F996F8643093B1404B9B787BB1032B49
:10D7F0000DD005F1010A3E4902A85FFA8AFA05F048
:10D80000F7FC2846554602AA3A49FEF783F996F8EE
:10D8100069306BB1354B9B7853B1032B08D002A90B
:10D82000002025F0DFFD02AA33492846FEF772F9F1
:10D830000023324A6360324B3B44136021E6286880
:10D8400004F024FD0023C8F800302E4BB7FBF3F79B
:10D850002D4B07F001071F702C4F3B681B0104D5AF
:10D86000FF2025F08BF9C4F85C042B6823B193F9F1
:10D870000E30002B3FF779AE00204FF06408FEF722
:10D88000D6F8234B94F8642493F854109B46DFF8A1
:10D8900084A0914290FBF8F83ED8DAF8003023F0EB
:10D8A00001033DE0C9280408901504085E790120B1
:10D8B000D028040810280408DA280408E4270408FB
:10D8C000E7280408D4810120F32804083D4D04080A
:10D8D000FF280408F4780120732F0408082904089D
:10D8E0002C770120142904081D290408225701203F
:10D8F0002A2904083029040839290408247401203D
:10D9000000879303400D030001000120D49C0120F7
:10D91000FE5401201C740120DAF8003043F00103AA
:10D92000834A1278BABB23F4C00323F0020399F8A8
:10D930000020900742D443F48043BBF85690CAF8C5
:10D94000003009F00F00FEF701F97A4A4FEA192377
:10D95000534325D1DAF8003023F02003BBF8589068
:10D96000CAF8003009F00F00FEF7F0F8714A4FEAEC
:10D97000192353431BD1DAF8003023F04003BBF8DE
:10D980005010B26891421CDDDAF8042023F0102315
:10D9900022F020021BE043F4C00343F00203C6E779
:10D9A0009842D7D3DAF8003043F02003D6E7834219
:10D9B000E1D8DAF8003043F04003E0E723F4804395
:10D9C000BBE7DAF8042043F0102342F02002CAF843
:10D9D0000420BBF8522028689045ACBF43F40043B4
:10D9E00023F40043CAF8003004F050FC132023F065
:10D9F000E7FC00287FF4B6AD4F4E3268910702D5A0
:10DA00000320FFF75FF80120FFF75CF80020FFF725
:10DA100059F80220FFF756F80520FFF753F80620C3
:10DA2000FFF750F82520FFF74DF80720FFF74AF8D9
:10DA30000920FFF747F80A20FFF744F80B20FFF70B
:10DA400041F80C20FFF73EF80820FFF73BF80F20C5
:10DA5000FFF738F81020FFF735F81120FFF732F8FC
:10DA60001220FFF72FF81320FFF72CF81420FFF7F0
:10DA700029F81520FFF726F81620FFF723F81920BC
:10DA8000FFF720F81A20FFF71DF81B20FFF71AF800
:10DA90001C20FFF717F81D20FFF714F82020FFF7D0
:10DAA00011F82120FFF70EF82220FFF70BF833685A
:10DAB0009A0611D50E20FFF705F80D20FFF702F8A2
:10DAC0001820FEF7FFFF1720FEF7FCFF1F20FEF7D0
:10DAD000F9FF1E20FEF7F6FF3B681B0105D523204A
:10DAE000FEF7F0FF2420FEF7EDFF2620FEF7EAFF09
:10DAF0002720FEF7E7FF35E5104B18680368DB6861
:10DB0000984735E50D4D286804F0C0FB02220C4B08
:10DB10001146286804F092FB9AF86A30002B7FF4D3
:10DB200065AD032571E54FF4005010F04FFC2CE576
:10DB30007D5C01200087930304790120804D012042
:10DB40004429040838B50B4C23688BB15A68054644
:10DB5000821A002A04DA0CE05A68AA1A002A07DBA3
:10DB60009A6818461B68226098472368002BF3D1F7
:10DB700038BD38BDB093012044F620635D4A5E494C
:10DB800003442DE9F04F2DED088B93B014780B6012
:10DB90000790002C00F07487584B07991B68994236
:10DBA000574B049340F290801E68013C554B5649F8
:10DBB00006F480560293554B039114700693002E81
:10DBC00040F08E80524B1B78022B00F02387042BF1
:10DBD0000AD103F0ADFE4F4B4F4A1B68C31A934264
:10DBE000C2BF4E4B00221A804D4B079A9A42069BA9
:10DBF0009B7800F21D86002B40F01E86494B059352
:10DC0000049B1E6816F4805740F0DA86DFF84091D6
:10DC1000029BB3F90610039B5D8BA942B4BF00259C
:10DC20000125DFF82881D8F8003013F0805300F088
:10DC30009180059A127812F0010200F09280039808
:10DC4000408C884241F36A82002D40F09180364C2E
:10DC500094F88810002940F08B803448002434491F
:10DC600000680C6090F82D004C608C6031490028F1
:10DC70007FD10870002A00F08180F1067ED52E4AFF
:10DC80001278D2067AD4002F78D1002B76D1740284
:10DC900074D42A4B1B78002B02F0D581284B9B783B
:10DCA000002D42F05E823BB1264A274B12681B686A
:10DCB0009B1A002BC2F26B8210201B4C11F050FB00
:10DCC000012384F8893059E01E680E4B0E4A06F491
:10DCD000805602930D4B03920693002E3FF472AFD1
:10DCE00000211A4805F080FE00287FF46BAF2BF06E
:10DCF0004BFF67E7AC93012044920120A8930120D9
:10DD0000D49C0120CC5C0120AC8F0120805C0120E0
:10DD1000A6920120B02D012060E316007A5C01205C
:10DD2000404B4C00348101205029012060790120B2
:10DD300000710120342F01205E790120EC220120A6
:10DD4000F07001202CB90120ACB60120D8B8012018
:10DD50000452012070023FF56CAF059A127802F070
:10DD60000102574C002184F88810002D3FF475AF54
:10DD7000544901200870002A7FF47FAF524B197874
:10DD8000002940F0C183039A029C568BB4F90070BD
:10DD90002346908BBE42B4BF80220022B3F904E038
:10DDA000B4F9024042F0400CB842CCBF634613467F
:10DDB000029A9B08B2F9067043F08002A642B8BFEF
:10DDC000134643F04002A042D8BF1A463C4C92088A
:10DDD00094F88AC042F080037645B8BF1A4642F0F4
:10DDE00040037045D8BF13469B0843F08002B742FA
:10DDF000C8BF134643F040028742ACBF18461046E6
:10DE0000844501F00E840B46A4F88C1084F88E1023
:10DE10002E4A84F88A001678002E01F0E1825F28ED
:10DE200001F0A0836F2801F0C383059B1B78DB07FB
:10DE300000F16A8394F88E10002940F06583B4F9EC
:10DE40008C30322B40F3608394F88A200120572ACB
:10DE500084F88E0001F04587049B1B685D0741F143
:10DE600038825A2A41F0358294F89030002B42F0E3
:10DE7000FE8094F8923083F0010384F89230002BF6
:10DE800042F07B810C20124E11F06AFA049B114A79
:10DE90001B68079203F00403002B40F03F830E4BF6
:10DEA0000DF1400B089640F6330A1D460A930023F5
:10DEB000192740F28334029ECBF80430109310E00F
:10DEC00050290120342F01206B760120EC22012003
:10DED0005C79012064790120B451012004354D455D
:10DEE00022D0A978EB7817FB01409942F6D295F839
:10DEF00001E017FB03410EF1040336F913305345DB
:10DF0000A8BF5346B3F5617FB8BF4FF46173984221
:10DF1000E4DA9942E2DB29782729DFD8043558462C
:10DF200005F052FD4D45DCD1654B089E1B789BE802
:10DF3000030088E80300002B40F0E787614B1B7863
:10DF4000002B00F05D8701215F4805F04DFD0028A2
:10DF500040F02683069BDB78002B40F02183DFF81E
:10DF6000849133881CB224F00104A7B2BB423780ED
:10DF700000F0E687554C4FF002084FF0140B4FF0BD
:10DF8000FF0A0E2084F8008084F801B084F802A013
:10DF900011F0E6F941464C48378805F025FD002888
:10DFA00041F0AC8227F002039BB2BB4233800AD01F
:10DFB000464B02201421FF2218700E2059709A70CF
:10DFC00011F0CEF93788424BBC07424A19785068A5
:10DFD00008BF81F0020108930992C1F3400103F0E8
:10DFE000FBFF2421384805F0FFFC30B9059A13786F
:10DFF000590744BF23F004031370D9F8003013F01D
:10E000000A0F1DD00521304805F0EEFC002801F074
:10E010005B803488620741F1F88106212A4805F0C7
:10E02000E3FC002801F03D80630641F1E681072111
:10E03000254805F0D9FC002840F09887D9F8003031
:10E040009F0600F15B86B6F80080234F0C211E4826
:10E0500005F0CAFC002800F0E98248F480734345CB
:10E06000338009D0194B02201421FF2218700E2092
:10E0700059709A7011F074F9184B1B78082B00F046
:10E08000E1820E2B00F0DE82049B1C68600563D5E4
:10E09000134B1B79002B00F0658214210A4805F010
:10E0A000A3FC002840F0638220F0DAFE012011F08A
:10E0B00061F80024DFF830B04FF0CC0AA94616E032
:10E0C000F4A3012028740120D8B80120AC54012009
:10E0D000F4B80120F8B80120EC8101206071012022
:10E0E000DC81012004790120989F0120DCB20AFB29
:10E0F00004F8631C68B3022C2BD85BF80850002D81
:10E10000F4D1C3784FF0030EE5492A4690F9020096
:10E1100051F8233001210195CDF800E025F060FF92
:10E120000346CC2204EB440029460B9353B100EB89
:10E13000001001340BEB800031F0E3F90B9BE4B2EB
:10E140004BF8083028F0B4FD0AFB04F8631C0028E3
:10E15000D1D14D46049B1C68059B93F800A0D14B80
:10E160001AF0010A00F09B8201221A70079B4FF0FF
:10E17000010E02991868B1F906104289CA4B914202
:10E1800083F800E080F271824FF07E52C74B1A6034
:10E19000C74A039B0298B3F81880B0F900E092F9DF
:10E1A00004301078002BAEEB080392F801C014BFC6
:10E1B00001224FF0FF32002BB8BF5B42B3F5FA7F6C
:10E1C000A8BF4FF4FA73984280F22D821B1A07EE13
:10E1D000903AF8EEE77AC645C7ED007A03DAF1EE39
:10E1E000677AC7ED007A029BB3F902E0AEEB080351
:10E1F000002BB8BF5B42B3F5FA7FA8BF4FF4FA73A8
:10E20000984280F20D821B1A07EE903AF8EEE77AF8
:10E21000F045C7ED017A03DDF1EE677AC7ED017ACB
:10E22000029BB3F90400A0EB0803002BB8BF5B42CC
:10E23000B3F5FA7FA8BF4FF4FA736345CCBFA3EBE5
:10E240000C030023404502FB03F307EE903AF8EE7F
:10E25000E77AC7ED027ABCBFF1EE677AC7ED027AC2
:10E2600014F4805400F0B981B1F5FA6F914BA8BF56
:10E270004FF4FA611A78B1F57A7FB8BF4FF47A712A
:10E28000A1F57A71002A40F0C1818B48CA17DFF8E6
:10E2900040E26FF0630380FB019CC2EB6C1202F161
:10E2A000010C03FB02133EF912203EF91C10891ADF
:10E2B00003FB01F380FB0310DB17C3EB60131A446D
:10E2C00012B207EE902AB8EEE78A87ED038A002C97
:10E2D00040F0268533885A0640F1FF807749B6EE34
:10E2E000000A774A13F0030391ED011AD2ED014AB7
:10E2F000D2ED025A91ED035A74EEE57A92ED038A5B
:10E3000031EE457AD1ED000AD1ED028A71EE05AA0F
:10E31000D2ED003A34EEA5AA27EE274A97ED012A5E
:10E3200070EEA89A674A33EEC89AD7ED002AB0EE8D
:10E33000446A08BF97ED023A73EE887A18BF9FEDE2
:10E34000623A70EEE86A6149A9EE896A30EE81BAF4
:10E3500066EEA76AF0EE447A30EEC11AB0EE667A45
:10E36000DAEE8A7AAAEE8A6AA9EE897A73EEA40AAC
:10E3700073EEE43A72EE021AF0EE674A36EE266A5F
:10E38000AAEECA7AE9EEC94A20EE466A77EEE67A44
:10E39000ABEE206A37EE447A74EEA66A35EE684A30
:10E3A00027EE007A35EE285AF0EE460A66EE806ACD
:10E3B00035EEC86AE9EE897AC2ED010AE5EE236A14
:10E3C000A4EE067A20EEA05A75EE885A32EEA28AA2
:10E3D000B0EE456A67EE807AC2ED036AA7EE075A8F
:10E3E00082ED007A97EE076AE1EE257AB1EE669A41
:10E3F000F1EE478A20EEA64AF0EE454AF0EE465A84
:10E40000F1EE679AC2ED027A20EEA70AE9EE265AEB
:10E4100067EEA63AE9EEA74AB0EE405AB0EE631AAC
:10E42000A9EEA76AA7EE265AE7EEA75AE9EE264A12
:10E43000A8EEA01AB0EE449AA8EEA60AE7EE203A9B
:10E44000A7EE279A25EE827A65EE215AB0EE445A5D
:10E45000A6EEA66A21EE022AA8EEA75AF0EE656A99
:10E46000A8EE007AA2EE892AE2EEA46A66EE037AAA
:10E4700073EEA33A35EE055AB0EE006AA3EE237AA6
:10E48000E3EE056AE2EE067A87ED017A81ED377AEE
:10E49000C1ED366AC7ED006AC1ED387A1AE000BFF7
:10E4A000241C0408358101206C2F0120E42E01205A
:10E4B000C8700120843001201F85EB51D422012037
:10E4C000FC1F012034200120000000005029012001
:10E4D0003C8001200BB9C7ED027ABAF1000F40F081
:10E4E00065812EF047F913B0BDEC088BBDE8F08FC5
:10E4F000B54A1278960741F10884B44A127D042A7D
:10E5000041F203841AF06EFD049BB14A1B68B14EC0
:10E5100003F004030792002B3FF4C1ACAE4C94F817
:10E5200092305BB1059B1B78DA0707D5029BB3F9E4
:10E530000620039B5B8B9A4201F33C811121A74883
:10E5400005F052FA002800F0D48594F896302BB9E3
:10E5500094F8903013B93223A4F89430012384F84E
:10E5600096309CE4059B1B78D9077FF59DAD4FF451
:10E570000F7029F0C1FF00283FF4ECAD10F0D8FD7A
:10E580004FF40F7029F05AFF00283FF4E3AD10F06C
:10E59000CFFD4FF40F7029F051FF0028EED1D9E5DF
:10E5A000DFF88492D9F8003099077FF5DAAC378824
:10E5B000FA073FF5F7AC47F001039F4233803FF481
:10E5C000F1AC874B02201421FF2218700E205970E5
:10E5D0009A7010F0C5FE3788E4E4039B5A8B914291
:10E5E000C0F2AB84B1F5FA6FD4BFC2EB0101C2F542
:10E5F000FA614FF47A7303FB01F17A4BC2F5FA62C8
:10E600001878B1FBF2F100283FF43FAE5B78764A10
:10E6100001FB03F182FB0123C917C1EB631134E64F
:10E62000DFED727AF4E5DFED717AD4E528F48073DA
:10E630009BB2434533807FF415AD6D4B1B78082B9F
:10E640007FF41FAD328822F040039BB29A423380A0
:10E650003FF41AAD624B02201421FF2218700E20E5
:10E6600059709A7010F07CFE0EE5B1F5FA6F9FEDCF
:10E67000617ABDBF8B1A007AC2F5FA62037ABCBF19
:10E68000434393FBF2F3C3F1640307EE903A5A4B12
:10E69000F8EEE77A67EE877AC3ED007A78E51B78C3
:10E6A0000493002B7FF462AD544A1268002A3FF4B1
:10E6B0005DAD534ADFF874B1114612F8030CA2F1B4
:10E6C000030905929BF8048022F042FE059A002877
:10E6D00000F07C85049BB8F1000F59D109F10801C5
:10E6E00099F8050022F034FE002841F09184454954
:10E6F00099F80A0022F02CFE002800F07C85B8F181
:10E70000020F41F09C84404999F80F0022F020FE4E
:10E71000002841F090843D4999F8140022F018FE39
:10E72000002800F07C85B8F1040F41F0808438495E
:10E7300099F8190022F00CFE002841F07484354944
:10E7400099F81E0022F004FE002800F07C85B8F144
:10E75000060F41F05984304999F8230022F0F8FD62
:10E76000002841F04D842D4999F8280022F0F0FD51
:10E77000002800F07C85B8F1080F41F03D8428495D
:10E7800099F82D0022F0E4FD00283FF4EFAC0923B6
:10E790001A4602EB82028BF80430224B914499F81E
:10E7A000011099F8022019705A70DFE4089B19785B
:10E7B000099B01F00101186803F00EFC13B0BDECD9
:10E7C000088BBDE8F08F00BF5E790120589F0120C3
:10E7D000647901205C79012050290120D8B80120FA
:10E7E000AC540120843001201F85EB510000000053
:10E7F000607101200AD7233CE42E012038810120DA
:10E800005E530120685301206D5301207253012093
:10E81000775301207C53012081530120865301202E
:10E820008B5301203C810120047901200400012048
:10E8300013B90123069A9370B24B1B201D46059312
:10E84000069B93F8214022F0BBFD2D788146012CD8
:10E8500005F0010800F09C8605F00205069AAA4E14
:10E8600092F820309346DFF8C0A2A84FCDF81C9054
:10E87000052B00F29980DFE803F0877D03C7CABB50
:10E88000012C04BF05238BF82030B8F1000F00F0F5
:10E89000E680039B00213588B3F918000A46DFF8AB
:10E8A0008C9260F30F0160F30F0265F31F41029D2C
:10E8B00060F31F42D9F800006960DBF814102A6089
:10E8C000814280F06886032547F230510322CBF85D
:10E8D0001C108BF8202002200FF078FD2BF054F94B
:10E8E000D9F80000DBF81C20042102448BF820102A
:10E8F000CBF81820012C40F01287D9F80020DBF863
:10E900001810914250D29AF8000018B922F058FD20
:10E91000002849D13A6822F002023A60D9F8001082
:10E9200064207388002200FB03134FF480608BF88F
:10E930002020CBF810308BF803200FF017FD9BF848
:10E94000203095E722F042FD012801F0BE81079BAF
:10E9500013B1B379002B4ED1012C25D0DFF8CC9127
:10E96000DBF81010D9F800209142C0F0E3860123B3
:10E970008BF82030012C3BD0F379012B74D022F09E
:10E98000A5FC9BF8203073E7B8F1000FDAD1DDF871
:10E990001C904FF48060B9F1000F00F0E4820FF09A
:10E9A000FDFC0023069A1361002D3FF429A9284697
:10E9B00010F0D6FC049B1E6816F480573FF426A97D
:10E9C0001D21534805F010F800287FF41FA9514B72
:10E9D00003F1500903E00433994500F061861A7889
:10E9E000262AF8D19978DA789142F4D2FFF710B953
:10E9F000DFF8389192E722F069FC03224FF47A7332
:10EA00008BF82020CBF81C30DFF8209163E7DFF88B
:10EA10001C916FE7039A0299537DD27D013B31F936
:10EA200013301AB140F6B832D21A13B2A3F57A7382
:10EA30009FED397A40F2FF31384A07EE903AF8EE0E
:10EA4000E77A67EE877AFCEEE77ACDED057ABDF8D6
:10EA500014308B4228BF0B461380FFF7C5B8DFF890
:10EA6000CC90D9F800202FE722F030FC032240F6AA
:10EA7000B833DFF8B8908BF82020CBF81C302AE7A9
:10EA8000274F3B78002B59D0DFF8A4804FF47A79D8
:10EA9000DFF8A0B0234B4546DFF89CA05E46039309
:10EAA00026E0039A115D9847032C02B219DC024656
:10EAB000B8B138F824E040F6CA016B88A0EB0E022A
:10EAC000A3EB0E0040F2EE2309FB02F292FBF0F200
:10EAD00002F57A728A42A8BF0A469A42B8BF1A461D
:10EAE00012B201343B782AF8022F04359C4227DA0F
:10EAF000072C3046DBF80430E1B2D2DD30469847CF
:10EB000002B2EEE7348101203480012058790120DF
:10EB1000D8B80120B45101206F12833F7A5C0120E4
:10EB2000A4540120AC8F0120EC2201202CB901203B
:10EB300008530120309201204E2901209A4A039265
:10EB40009A4942F201069A4A049107980968A2FB81
:10EB5000002B0E404FEA9B1B00F0DC829548964A42
:10EB600090F800E0954C1078954A84F800E0107019
:10EB7000BEF1000F04D0924A92F800E08EF0010E30
:10EB8000904C0F2284F82420002B00F05B848E4BE5
:10EB900011F4805F8D490E931B7894F825A01846D8
:10EBA000039B0C9204F12802A1FB00C19D8C0B90E9
:10EBB0004FF0000303984FEA5101CDF814E0B64638
:10EBC000B0F818C001EB41010398CDF834C0B0F89B
:10EBD00026C00D98CDF828C084467D4808BFAC46B5
:10EBE000CDF818A00290A2460B98CDF83CC00BF5CA
:10EBF000967C411A97F80080CDF820C0C9B2DFF8A2
:10EC0000FCC1734C09910599002900F088833AF9F9
:10EC1000130059001FFA80F9A94503D30A9EB14594
:10EC200040F2BC835CF82300834580F08083605E03
:10EC3000BEF1000F40F09483013360520632434529
:10EC4000E1DB0C9A5446634B0F2A84F82420DDF84C
:10EC500018A00CBF0122002284F825A01A7000F031
:10EC6000F88301235449564A04200B7013700FF0A7
:10EC7000ADFBDFF884B1584BDBF800101C4606935F
:10EC80009B686268CB1AE160934284BF002384F8DA
:10EC90002130049B3C781E68002C01F09A80039A76
:10ECA00016F480564D4DB2F824E0178B40F03884AE
:10ECB0003246474928460DE0437803EB830303EBD4
:10ECC000830303F2EE239BB20132023021F8023BB0
:10ECD00094420DD015F81230002B00F06383022B04
:10ECE000EAD00B880132023021F8023B9442F1D184
:10ECF0000E9A137801331370FEF761BF384B1B78FF
:10ED00009C0704D5374C237D042B00F21E85B6F8F2
:10ED1000008018F0300F40F0B882334FFFF796B9FB
:10ED20001D21324804F060FE002840F092840A9BC6
:10ED300003E00433AB423FF4CDAA19782629F8D179
:10ED40009878DA789042F4D2069BDB78002B7FF437
:10ED5000C1AA264804F048FEDFED257A002801F01C
:10ED60002B8038EE678AC8F57A73114901201AB2F0
:10ED7000204BFDEEC87ACDED027A1870BDF908304F
:10ED80001B0381FB0301DB17C3EBA11302FB03F39E
:10ED900043F30F33434407EE903AF8EEE77AC7EDBA
:10EDA000037AFFF797BA00BFAC8F0120D49C0120F3
:10EDB000D34D62100C920120FC200120715C0120D7
:10EDC000FD20012050290120E4530120ABAAAAAA6A
:10EDD000CC5C01206C710120805C0120B2530120C9
:10EDE0005E790120589F0120EC810120D8B80120D4
:10EDF00000007A44602F01202CB90120E853012043
:10EE0000DFF878B39846DFF870A34FF001090BF1F3
:10EE10005A07C54C59461BF8010C22F099FAF8B173
:10EE20009BF804209BF8023002EB420E9BF8030093
:10EE3000013B09FA02F204EB8E0E03EB4303DEF80A
:10EE40009C1053448B420BD094F8C8108EF8980055
:10EE500021EA0202CEF89C30CEF8A08084F8C820C7
:10EE60000BF1060BBB45D5D1B04B4FF0FF3AB04A82
:10EE70004FF0000B1B78DFF8089312680893A9F194
:10EE80009808079B17461B680993D9F804309BB371
:10EE90001C788CB3D9F80820BA1A002A10DB01219B
:10EEA00098F8C82007F5FA7E4FF0FF3001FA0BF111
:10EEB000C9F808E022EA01029E4988F8C8200860E3
:10EEC000089ACAB199F8002059780432D2B20029C0
:10EED00040F0588103990298098B30F9122001F112
:10EEE000C800824240F3ED8398F8C8109A7841FA3E
:10EEF0000BF3DB0740F16F840BF1010B09F10C09F7
:10EF0000BBF1040FC1D1FFF71EB88B4B03E00433F4
:10EF10009D423FF413A819782329F8D19878DA781C
:10EF20009042F4D2854804F05FFD00283FF406A823
:10EF3000142010F015FAFFF701B82146FFF75DBB6A
:10EF400002217E4804F050FD00283FF42BA83480B5
:10EF5000BB073FF538A847F00203BB4233807FF47C
:10EF600027A8FFF730B80FF001FA1AE5744AB2F992
:10EF70000030002BB8BF5B42B3F5E17FBFF65EA85F
:10EF8000B2F90230002BB8BF5B42B3F5E17FBFF6A8
:10EF900055A86C4BB0EE007AF7EE000AD3ED077A75
:10EFA000B6EE008A93ED096A93ED030AD3ED056A84
:10EFB00077EE867A30EE260AE7EEC70A30EE000AD0
:10EFC00004F072FA20EE488ADFED5F7A38EE270A05
:10EFD000FDEEC07A17EE903A2033402B40F2F883D2
:10EFE0009FED5A0ABDEEC87A594ADFED587A82ED94
:10EFF000000A17EE103AC2ED017AC2ED027A203310
:10F00000402B47D8DFED537AB4EEE78AF1EE10FAE1
:10F0100041F33F80DFED506A9FED507AB4EEC78A2E
:10F0200078EE667AF1EE10FAB0EE678AF6DC9FEDC4
:10F030004C7AF4EEC77AF1EE10FA41F114809FEDAC
:10F04000466ADFED486AF4EEE67A37EE867AF1EE4C
:10F0500010FAF0EE477AF6D4DFED3B7AB4EEE77AB9
:10F06000F1EE10FA40F39086DFED3A7A37EEC77A88
:10F0700027EE076ADFED3C5ADFED3C6ADFED3C7AB4
:10F08000E6EE256A67EE065AE6EE267AA5EEA77A40
:10F09000F0EE477A0A20C2ED037A10F061F9FEF72C
:10F0A000CDBF24F040039BB2A34233803EF4BFAFF8
:10F0B000304B02201421FF2218700E2059709A70D4
:10F0C00010F04EF9FEF7B3BF338823F00404A4B266
:10F0D000A34234803EF4A1AF264B02201421FF222C
:10F0E00018700E2059709A7010F03AF93488FEF7B3
:10F0F00094BF94F89030002B3EF4D1AE059B1B7862
:10F1000013F0010302BF012284F8903084F89120AB
:10F11000FEF7C5BE054A92F800E029E5024C012140
:10F1200084F88810FEF724BE50290120715C01206C
:10F130002CB9012004000120B4510120D8B80120CD
:10F14000087901200C200120DB0FC93F00000000DE
:10F15000D4220120DB0F4940DB0FC940E4CB16412C
:10F16000DB0F49C0E4CB16C192E741B99730083CA8
:10F1700015A82ABEAC54012050F6030855520120B0
:10F18000E8290120012900F05D85BAF1FF3F0BD08D
:10F190001B780C2B08D0BB4B03EB8404BA4BC3F891
:10F1A00000A0636CC8F8D030012398F8C82009F19A
:10F1B0000C0903FA0BF30BF1010B1343BBF1040F22
:10F1C00088F8C8307FF461AEFEF7BDBE511D99F8D6
:10F1D000050022F0BDF800283FF489AAB8F1010F1C
:10F1E00040F0168709F10D0199F80A0022F0B0F8F5
:10F1F000002840F02487A54999F80F0022F0A8F8CC
:10F2000000283FF488AAB8F1030F40F01487A04902
:10F2100099F8140022F09CF8002840F008879D49D6
:10F2200099F8190022F094F800283FF488AAB8F160
:10F23000050F40F0F886984999F81E0022F088F8EA
:10F24000002840F0E186954999F8230022F080F8E3
:10F2500000283FF488AAB8F1070F40F0D186904902
:10F2600099F8280022F074F8002840F0C5868D49EE
:10F2700099F82D0022F06CF800283EF477AFB8F131
:10F28000090F3EF473AFFFF782BA1020864F0FF0DC
:10F290006DF820200FF06AF8844B0022B6F8008049
:10F2A0001A7000218248834B834A016011608348B1
:10F2B000834A196000234160816103608360436178
:10F2C000C36113605160936053619161D361FEF734
:10F2D000BDBE5D2A00F084825B2A00F08D855E2A27
:10F2E00000F0C885562A00F03486972A00F09486EC
:10F2F000A72A00F0C385734E3388990740F08085B4
:10F30000A2F1B703072B00F2B882DFE813F0AF02D7
:10F31000B602B602B6028302B60274027402002D6F
:10F320003AD05CF8230059008345FFF480AC66486E
:10F330005FFA83F9644E405C0E4400283DD00228F9
:10F340004CD1707800EB800000EB800000F2EE20E2
:10F3500080B2032B39DD00B2BEF1000F3FF46CAC7C
:10F36000099E22F81600069E1EB90B9E022E7FF6FD
:10F3700063AC0120B2F80090544E06905088484487
:10F38000B2F80490484400B286FB0069504E7052B7
:10F39000A9EBE07000B24FE428465900089E4CF8F3
:10F3A000236045E4D3B2022B05D9032B73463FF407
:10F3B0008BAC0B8896E43B4686E4B9F1020F40F231
:10F3C0003E84B9F1030F09D10F98012600B206FA65
:10F3D00003F90C9E26EA09060C9629E4605AB8E760
:10F3E00031463C4804F000FB002800F0F68084F829
:10F3F0008F602BF009F8FEF718BD44F04003A342DC
:10F4000033807FF455AEFEF712BE44F004039C42F5
:10F4100033800AD0304B02201421FF2218700E20B6
:10F4200059709A700FF09CFF34882C4B2C4AB3F91A
:10F4300004302C4982FB0302DB17C3EBA2030B80D1
:10F44000FEF7EBBD284B012228491A70284B0E917C
:10F4500002931B211F4804F0C7FA00287FF401AC77
:10F46000244BDFF894B019460693DBF80030CA68E5
:10F470008B609B1AC82B00F2B084049B1E6806F4B4
:10F48000805635E450F60308040001206D53012036
:10F4900072530120775301207C53012081530120B6
:10F4A000865301208B530120EC810120F65D012061
:10F4B000082F0120C82F0120E05E0120905E01206E
:10F4C000B85E01205C790120B25301205655555594
:10F4D000C0290120D8B80120AC54012008790120AE
:10F4E00067666666005F01206C710120E4530120AD
:10F4F000CC5C0120805C01202CB9012027F00103A5
:10F500009BB2BB4233803FF423AD0E2084F80080D1
:10F5100084F801B084F802A00FF022FF378817E5C5
:10F520000022C04928460EE0437803EB830303EB37
:10F53000830303F2EE239BB2013221F8023B023037
:10F5400094423FF4D5AB15F812301BB1022BEBD02F
:10F550000B88F1E75FFA82FE3B46BEF1030FEBD961
:10F560000B88E9E7B3F5FA7FFEF6CEAF94F88E305C
:10F57000002B7EF4C9AF059B01221B7884F88E20F6
:10F5800013EA020500F0C8832AF0FEFAFEF7BCBFBA
:10F590000025FFF763B9A44A1278002A7FF493A9E3
:10F5A000012C40F0CB859BF820300325FFF760B994
:10F5B000B3F5FA7FFEF6A8AF94F88E20002A7EF409
:10F5C000A3AF059B01211B7884F88E10D90700F1A9
:10F5D000E8832AF019FFFEF797BF059B934A1B7833
:10F5E0001060D8077EF526AC914B1B78002B3EF4BB
:10F5F0008BAF069BDB78002B7EF486AF94F88F30C0
:10F600000133DBB2032B84F88F307EF67DAF894B5C
:10F610005B7813B9002D7EF477AF2AF0B5FAFEF7C8
:10F6200004BC854B47F6FF76844A1968B4F98C30E0
:10F63000C96982FB0172C91792118F1A3E44B34205
:10F640003EF7E6AB521A13441BB2A4F88C30FEF717
:10F65000DFBB069BDB78002B7FF469ABDFED787AAC
:10F66000C8F5FA63754938EE678A1AB2FDEEC87AB2
:10F67000CDED027ABDF908301B0381FB0301DB17D6
:10F68000C3EBA11302FB03F343F30F33434407EE31
:10F69000903A0A9BB8EEE78A87ED038AFFF74DBBE5
:10F6A000684A039BD5881B8B029AB2F906105A1B35
:10F6B00091427CDD2B449942B4BF00250125FEF721
:10F6C000B0BAC8398A4263DA98F8C8109A7841FA11
:10F6D0000BF3D8073FF510AC524201200B920FF00C
:10F6E00071FF631E0B9A162B00F2BC83DFE813F048
:10F6F000C201AA018E01EF01DB011C024901700267
:10F700004D0287027401BA03EF01A5021C024901F0
:10F7100070024902A102020134011B01EA000699AC
:10F72000D9F80020CB6913448B61002D3EF468AA00
:10F73000FFF73DB921F0CAFD032140F6B8328BF83E
:10F740002010CBF81C20FFF7C6B80A2021F038FEA5
:10F75000B6F800808146002800F0F18218F0100F02
:10F7600000F09A83384C94F8D490B9F1000F7FF4EC
:10F77000D4AA364F0D200FF0F3FD0123B6F8008018
:10F7800084F8D430B9F1000F7FF48BADFEF75EBC86
:10F79000012298F8C83007F5FA7102FA0BF2C9F89D
:10F7A000081023EA020388F8C830FFF7A5BB01253B
:10F7B000FEF737BA0021264804F016F900287EF437
:10F7C000BDAE322384F89200A4F89430FEF7B6BEA2
:10F7D00003F0F2FD06E4002A0CBF012002207DE7C1
:10F7E0001C4B002201201C4C1C4922700B600FF0A6
:10F7F000E9FEFEF789BE184B022219495A70194BCF
:10F8000007910B6021F040FE049B1B6803F004038A
:10F81000FEF742BB104B002211495A700791124B60
:10F82000EFE700BFCC5C0120242F0120B0B60120FF
:10F83000715C0120F0700120547A0120D34D6210D8
:10F8400000007A441C80012050290120EC81012015
:10F85000D8B80120DE550120149F012060790120D5
:10F860006479012002570120EA560120D44B01227D
:10F87000D4495A700791D44BC3E79E2A00F04D84B7
:10F880009D2A00F04284AE2A00F03784AD2A00F0B1
:10F890002C84EF2A00F01584FD2A00F0FE83FB2A59
:10F8A00000F04684FE2A00F04084F72A00F04384EA
:10F8B0007B2A7EF4EBAA4FF4FA6102202BF0D0F9F8
:10F8C000FEF7E4BAD8F8CC00C04B90F836A09B788D
:10F8D0009244BAF1640FA8BF4FF0640A2AEAEA7AA8
:10F8E00080F836A0002B40F02C8420F08DFED9F853
:10F8F00004304DE4D8F8CC00B44B90F802A0924408
:10F90000BAF1C80FA8BF4FF0C80A2AEAEA7A80F80D
:10F9100002A09B78002BE8D01420514621F09AFDDC
:10F92000D8F8CC00E1E7D8F8CC00A84B90F837A085
:10F930009B789244BAF1FE0FA8BF4FF0FE0A2AEA64
:10F94000EA7A80F837A0002BCFD01620514621F05C
:10F9500081FDD8F8CC00C8E709999C4B91F801A02B
:10F960009244BAF5967FA8BF4FF4967A2AEAEA7ACB
:10F9700081F801A09B78002B40F01184D8F8CC00CE
:10F98000B3E7D8F8CC00914B90F804A09978924452
:10F99000BAF1C80FA8BF4FF0C80A2AEAEA7A80F87D
:10F9A00004A0002940F00C84102C9ED090F801A0F7
:10F9B0009244BAF1C80FA8BF4FF0C80A2AEAEA7AFF
:10F9C00080F801A09B78002B8FD01320514621F0A6
:10F9D00041FDD8F8CC0088E7D8F8CC007B4B90F8F4
:10F9E00008A09B789244BAF1C80FA8BF4FF0C80A8C
:10F9F0002AEAEA7A80F808A0002B3FF476AF0B20C1
:10FA0000514621F027FDD8F8CC006EE709996F4BDD
:10FA100091F804A00B939244BAF1640FA8BF4FF081
:10FA2000640A2AEAEA7A81F804A021F02DFD0B9BF2
:10FA30009B78002BA2D00320514621F00BFDD8F873
:10FA4000CC0052E70999614B91F802A09244BAF1B7
:10FA5000640FA8BF4FF0640A2AEAEA7A81F802A08C
:10FA60009B78002B8AD00220514621F0F3FCD8F875
:10FA7000CC003AE70999554B91F800A09244BAF1AD
:10FA8000FA0FA8BF4FF0FA0A2AEAEA7A81F800A032
:10FA90009B78002B3FF472AF0120514621F0DAFC35
:10FAA000D8F8CC0021E70999484B91F807A09B783A
:10FAB00092448AF3080A81F807A0002B3FF45EAF56
:10FAC0000520514621F0C6FCD8F8CC000DE7099876
:10FAD0003E4B90F806A099789244BAF1640FA8BF03
:10FAE0004FF0640A2AEAEA7A80F806A0002940F07A
:10FAF0005E830D2C3FF442AF09989B7890F805A0E7
:10FB00009244BAF1640FA8BF4FF0640A2AEAEA7A75
:10FB100080F805A0002B3FF431AF0E20514621F0B4
:10FB200099FCD8F8CC00E0E6D8F8CC00274B90F848
:10FB300003A099789244BAF1C80FA8BF4FF0C80A41
:10FB40002AEAEA7A80F803A0002940F0FF820F2C0D
:10FB50003FF4CBAE90F800A09244BAF1C80FA8BF12
:10FB60004FF0C80A2AEAEA7A80F800A09B78002BB6
:10FB70003FF4BBAE1220514621F06CFCD8F8CC000B
:10FB8000B3E6D8F8CC00114BE4E7D8F8CC000F4B23
:10FB900090F806A09B789244BAF1C80FA8BF4FF026
:10FBA000C80A2AEAEA7A80F806A0002B3FF49DAE44
:10FBB0000920514621F04EFCD8F8CC0095E600BF54
:10FBC000149F012064790120F6560120225701205C
:10FBD000D8F8CC00BE4B90F805A099789244BAF1C1
:10FBE000C80FA8BF4FF0C80A2AEAEA7A80F805A031
:10FBF000002940F0F182112C7FF47FAE75E6D8F831
:10FC0000CC00B34B90F807A09B789244BAF1C80F90
:10FC1000A8BF4FF0C80A2AEAEA7A80F807A0002BAA
:10FC20003FF463AE0A20514621F014FCD8F8CC0012
:10FC30005BE6D8F8CC00A64BB8E6A54B5CE70D9880
:10FC4000FFF787BB02994FF4966A31F91220997831
:10FC5000B2F5617F9AFBF1F1C0F28C8040F6330A75
:10FC60009245A8BF92460C2CAAF5617A9AFBF1FA4C
:10FC70005FFA8AFA00F07C81182C7FF489AA524638
:10FC8000C82AA8BFC822D8F8CC10D0B291F817E083
:10FC900070453FF47DAAB2EB0E028D4BC87548BF8C
:10FCA00007329978D2100132D3B239B913B118465C
:10FCB0000FF088FCD9F80430FFF76ABA51461820D3
:10FCC0000B9321F0C7FB0B9BF0E7DFF85092642108
:10FCD0007288D9F8003001FB0233CBF81030FEF700
:10FCE00036BE7C4B4FF47A727B491B68B2FBF3F251
:10FCF000049BC2EB42101B6802EB80021F064FEA16
:10FD0000C202A1F8AC203EF5F3AB744A03F0040341
:10FD1000734E0792FEF7C0B80F20714E0FF020FB14
:10FD2000B4F88C20049BFA3A84F88E501B68A4F82F
:10FD30008C206A4A03F004030792FEF7ADB818F06E
:10FD4000100F40F047810B2021F03AFB002840F0D3
:10FD50001181644F18F0200F40F04781624C94F8F5
:10FD6000D430002B3FF406ADB9F1000F7FF499AA0F
:10FD7000FEF76CB90C2C00F0D380182C40F0A48056
:10FD80004FF0000A52467EE7DFED587AB4EEE77A8C
:10FD9000F1EE10FA44BFDFED567A37EEC77AFFF77F
:10FDA00067B95449049B0A601B684C4A03F004037A
:10FDB0004B4E0792FEF770B838EE678AC8F5FA63C3
:10FDC0004D491AB24D4BFDEEC87ACDED027AFEF7E1
:10FDD000D4BF06F48056FEF78BBF0846484A01217F
:10FDE000136880F82110049923F004030E6813604F
:10FDF00006F48056FEF77CBF424B01220220F2E45B
:10FE00000023BB2A109300F04181B72A00F03A8109
:10FE1000BE2A00F03581BD2A7FF42FAD4FF6FE716A
:10FE2000394A2E48D589079090892B440144D381C3
:10FE3000918126F0CBFA02F0C5FD26F0AFFA02F070
:10FE4000EBFB01200FF0BEFBB4F88C20049B0021DB
:10FE5000FA3A1B6884F88E1003F00403A4F88C208F
:10FE6000FEF71AB8D8F8CC004FF0FF3A20F0CCFBE0
:10FE7000FFF79AB9254B02220320B4E42449049BDE
:10FE80000A781B6842F00402144803F00403144E7D
:10FE900007900A70FEF700B81020124F0EF07EFA9D
:10FEA00020200EF063FA1B49081F1DF04FFE1A4B6D
:10FEB00002221A700C4C94F8D430002B00F06381AD
:10FEC000B6F80080FFF7EDB94FF0000AFFF760B910
:10FED00022570120C49C0120D09401206479012084
:10FEE0005C790120EC81012050290120DB0FC9BF82
:10FEF000DB0F49C0B0B60120D34D6210602F012046
:10FF0000587901202C560120D07001207A5601200A
:10FF10005E790120D05D0120F65D01202CB9012021
:10FF200000229246B249497891423FF431A9B14B3F
:10FF300010460B920C932AF005FF0C9B0B9A9B78B2
:10FF400023B151460C2021F085FA0B9A531CDBB2E9
:10FF5000ACE626F03BFA02F035FD26F01FFA02F07F
:10FF60005BFB01200FF02EFB94F88A20FFF7BDB950
:10FF70005246D7E7A04BA14F5B8997ED007A07EE79
:10FF8000903AB0EEC77AF8EEE77AB4EEE77AF1EE9F
:10FF900010FA7FF5DFAE97ED017AB0EEC77AF4EE96
:10FFA000C77AF1EE10FA7FF7D5AE18F0200F7FF484
:10FFB000D5AE20200EF0F2F9914B60681946226808
:10FFC00041F8040F18461A601DF0C0FD8D4B012248
:10FFD0001A706FE710200EF0C9F98A4BB6F800804E
:10FFE00083F800904FF00109ADE620200EF0BEF935
:10FFF000844B00221A705DE708231A46FEF7C9BB3E
:020000040801F1
:1000000007231A46FEF7C5BB06231A46FEF7C1BBF7
:1000100001231A46FEF7BDBB7B4A4FF4C871049B0F
:1000200011801B6871E605231A46FEF7B2BB042354
:100030001A46FEF7AEBB03231A46FEF7AABB0223FD
:100040001A46FEF7A6BB002D3DF436AE6F4C94F871
:100050008930002B3DF492AE0FF066F9002384F84E
:100060008930FDF78BBEB0EE677AFEF7F5BF684BBF
:1000700084F8901084F89100664E0793FEF74FBA0B
:100080000221CDE619464FF6FE73C9E61946022352
:10009000C6E6F0EE487AFEF7CABF002101202AF03A
:1000A000DFFDB4F88C20049B0021963A1B68A4F86D
:1000B0008C20574A03F0040384F88E100792FDF752
:1000C000EBBE0021524B084607932AF0C9FDB4F855
:1000D0008C20049B0021963A1B6884F88E1003F054
:1000E0000403A4F88C20FDF7D7BEFF21002022F0E6
:1000F0000FF894F88A20FFF7CCBB0121002022F0F2
:1001000007F894F88A20FFF7C1BB0021FF2021F0F7
:10011000FFFF94F88A20FFF7B6BB0021012021F0F1
:10012000F7FF94F88A20FFF7ABBB00210320B6E766
:1001300000210220B3E700210420B0E70325FEF7E9
:1001400036BC5146172021F085F917E40F2051469F
:100150000C930B9221F07EF9D8F8CC000C9B0B9AF3
:10016000F5E4002B3FF472AF2B494FF47A702B4A21
:10017000096800FB0313136068E70B20254E0FF09E
:10018000EFF8FDF783BE4FF00109FFF7F3BA29F04E
:10019000FBFC1E4C002384F88930FDF7EFBD1520D1
:1001A000514621F057F9D8F8CC00FFF79EBB5146D5
:1001B0000D200C930B9221F04DF90C9B0B9A98E4B7
:1001C000102051460C930B9221F044F9D8F8CC0042
:1001D0000C9B0B9AFFF7E8BB112051460C930B9236
:1001E00021F038F9D8F8CC000C9B0B9A03E500BF3E
:1001F000149F012022570120845E0120EC81012000
:10020000902D0120F65D01207EC90120502901209A
:10021000647901205C7901202CB90120ACB6012061
:100220002DE9F84FCC4C636820469847002800F031
:10023000CA80CA4B01221B7884F84020042B00F0AE
:10024000C480B4F91A10B4F91C20B4F91E306163EB
:10025000A263E363C24B1B88002B6FD0D4ED0D7AF1
:10026000C04DF8EEE76A95ED056AD5ED007AD5ED5B
:10027000015AA7EEA66A95ED067AD5ED047AA5EEA9
:10028000A67A95ED035AD5ED025A67EEC67AB0EE1E
:10029000460AA5EE467AE5EEA67A85ED057AC5ED25
:1002A000067A2EF073F994ED0E7AD5ED097AF8EE10
:1002B000C76A95ED0E6AD5ED0A5A95ED0F7AA7EE4D
:1002C000A66AD5ED0D7AA5EEA67A95ED0C5AD5ED78
:1002D0000B5A606367EEC67AA5EE467AB0EE460A20
:1002E000E5EEA67A85ED0E7AC5ED0F7A2EF04EF981
:1002F00094ED0F7AD5ED127AF8EEC76A95ED176A8C
:10030000D5ED135A95ED187AA6EEA76AD5ED167AB3
:10031000A6EEA57A95ED155AD5ED145AA06367EEB1
:10032000C67AA6EE457AB0EE460AE6EEA57A85EDE7
:10033000177AC5ED187A2EF029F9E0638A4F94F800
:1003400022108A481BF01CF93B88002B40F0868065
:10035000874ED6F8E450874B1B685B0743D4B5F94A
:100360000020616BA36B891A834AE06B07EE901A39
:100370006163B5F90210B8EEE77A92ED006A5B1A94
:100380007E4ED2ED026A07EE903AA363B5F90430CF
:1003900036EE077AF8EEE77A92ED016AC31A316811
:1003A00082ED007A07EE103A77EE867A0131E36348
:1003B000B8EEC77AC2ED017A316076EE877AC2ED87
:1003C000027ABDE8F88FBDE8F88F6D4BB4F91A00DA
:1003D000B4F91C10B4F91E20606318805980A16321
:1003E0009A80E26336E7B6F89430322B00F08980C9
:1003F000002B67D196F89130002BB0D0DFF88CC17C
:100400000020D6F800115F4F4FEAE17E8CFB0131EE
:1004100086F89100CEEB21112980D6F804218CFBBF
:100420000213D217C2EB23126A80D6F80831218B4F
:100430008CFB03E2DB17C3EB22135B1AAB80F86083
:1004400025F0C4FF02F0BEFA25F0A8FF02F0E4F8A0
:1004500001200FF0B7F8D6F8E45080E7444EB3F52A
:10046000C87F626B4FF0000314BFD6F8E81000217C
:10047000D6F8E450002063630A442B803988B7F82B
:100480000080B1F5C87FA16BC6F8E82018BFD6F888
:10049000EC30B8F5C87FA0630B446880C6F8EC3038
:1004A00053D0D4F83CE0B8F1010FD6F8F010E06377
:1004B0007144A880C6F8F0106AD008F1FF38A7F898
:1004C000008048E7D6F800010022616B012B6263CF
:1004D0000144C6F800112A80D6F80401A16BA2637A
:1004E0000144C6F804116A80E16BD6F80801E263A2
:1004F0000144C6F80811AA807AD0013BA6F89430CE
:1005000078E7B5F800C00022676B1F491D48B5F8B1
:1005100002E0C068A6F8F4C0B5F804C04A608A607A
:100520006263C6F800712A80A16BA263C6F8041149
:100530006A80E16BA6F8F6E0C6F80811E263A6F857
:10054000F8C0C6F8FC00AA80D7E7E36BE063C6F802
:10055000F030A880B1E700BF10790120C8800120E9
:10056000389301203C9301207EC901204479012069
:1005700050290120D49C0120947A0120907A0120F6
:10058000CC800120D0700120502A01201F85EB5122
:10059000DFF894C0C832C833C8314FEAE27A8CFB26
:1005A00002924FEAE3798CFB03B3CAEBE2128CFBB5
:1005B00001ACC9EBE319DFF86CE0CB172A80A5F892
:1005C0000290C3EBEC13228B9B1AAB80CEF80C008D
:1005D00025F0FCFE02F0F6F925F0E0FE02F01CF832
:1005E00040460EF0EFFFB7F80080D6F8E45064E71D
:1005F0000B2086F8962086F890300EF0B1FED6F8E3
:10060000E450B6F8F430B6F8F670B6F8F800D6F85C
:10061000FC10044A2B806F80A880B6F89430D1601B
:100620006BE700BFD07001201F85EB512DE9F84F1B
:100630008F4B06461B78DB074ED58E4A8E4C92F8C0
:1006400000808E4DB8F1010F00F0818020D3B8F109
:10065000020F08D18A498B4B09881B88994202D91D
:10066000012398461370E37A0BB32389FBB1864BC1
:100670001B78E3B10EF002FA00287FD0237B83427F
:1006800035BF0022012313462B7038BF2A700FE0BC
:100690007B497E4B0888B3F800E0637BAEEB030E2A
:1006A0008645DDDAE37A4FF00008002BDDD12B78A8
:1006B0002179632907D87648B8F1020F027800F053
:1006C000A380002A3CD143457249A27A38BF4346F1
:1006D0000B7062BBBDE8F88F694B674C188859886E
:1006E000E378411A0029B8BF494298420FD32278D3
:1006F00082420CD35F4A92F80080A8F10303012BD9
:100700003FD9654B1B78022B73D05C4D9AE7B0EB59
:10071000430FEFDC574A92F80080B8F1030F40F026
:100720008B805D4B1B78022B63D0544D9BE7012BD4
:100730007DD0022B1CD10720BDE8F84F0EF010BE73
:100740004268B61A554A964264DD4170BBE74D4B8C
:10075000607B1B884A491B1A098899420ADD4B4B6A
:100760001B888B42BFF47FAF0023137098467AE753
:10077000BDE8F88F02231370984674E702232B70AC
:1007800096E70229BDDC27784FF00003424D4FF079
:10079000640994F802E095F8008094F801A0374DC0
:1007A00013702B70374BDFF8E0B090FBF7F7013791
:1007B000082FA8BF0827B8F1020F1FFA87FC8BF893
:1007C00000701EFB0CFE1AFB0CFC1FFA8EFEA3F839
:1007D00000C02E4BDFF8B8C0A3F800E04FF00003D4
:1007E0008CF80190CCF804307FF457AF3FB29846B4
:1007F00002E0254B214D1F780229294BCCBF002157
:1008000001219F80D9801DE7002A99D101254660EA
:1008100016460570C1F16401224A06FB01F682FB0F
:100820000612F617A6EBA256643646704BE7082070
:10083000BDE8F84F0EF094BD02293FF762AF1648AD
:100840000027DFF844E0032300788EF80070984614
:100850000A4D0228DFF834C0DFF828E013702B704F
:10086000ACF80070AEF800707FF4FDAEC4E700BFD6
:10087000348101207C300120F47801208C3001206B
:10088000D481012080300120EA8101207E300120C6
:10089000843001207D5C0120C88001207F96980073
:1008A000CC8001206BCA5F6B0228094B094928BF25
:1008B000022000EB8002C0EBC20230B4064D441CA3
:1008C00003EB42032870E0B20B6030BC0EF07ABE3E
:1008D000DE55012060790120149F012008B525F024
:1008E00075FD02F06FF825F059FD01F095FE01202D
:1008F000BDE808400EF066BE08B50121022001F0F7
:10090000A3FB094B1B7803F00503052B08D000213E
:10091000012001F099FB0021084601F095FBFEE75C
:1009200020F0D8F8F3E700BFF44C012008B503F03D
:1009300001F925F04BFD02F045F8BDE8084025F02F
:100940002DBD00BF08B525F041FD02F03BF8BDE824
:10095000084025F023BD00BFA94B2DE9F04F1E78BC
:100960008BB0002E7ED1A74BA74C1D78A74FA4F1CA
:100970000A0A05F00105DFF8B49207F5887B54F800
:100980000A0CB8B14FF0CC0808FB06A801F066F9D4
:1009900080B154F80A0C01F05DF914F8023C0246EB
:1009A0007BB9242837D055B354F80A0C01F056F916
:1009B0000028EED10136CC34032EE0D10BB0BDE8D7
:1009C000F08F012B2BD0022B30D0032B3DD0042BEA
:1009D00000F07481052B00F06281062BE4D114F83D
:1009E000013C002B00F0E781012B00F02C82013646
:1009F0000023CC34032E04F8CE3CC0D1DEE7232AFA
:100A000054F80A0C00F08F81814B93F832309342F6
:100A1000BCD1F9F7B3FF012304F8023CC4E74D2829
:100A200000F07581002304F8023CBDE700233C2858
:100A300004F8023C00F065813E28B5D10122032371
:100A400004F8012C04F8023CAEE7C028EAD80021E3
:100A5000042304F8050C04F8040C04F8061C04F83C
:100A6000023CA1E76B4B18680028A7D0DFF8C0A1B3
:100A700001F094FD684DDFF8B091DAF8000001F064
:100A8000EDF800289AD0DAF8000001F0E3F8092820
:100A900031D03F282FD02B680428B3FA83F24FEAD5
:100AA000521202D1002A40F0C6810C2800F0F080DA
:100AB000002B00F0A0800A2800F0BC80A0F10D01FE
:100AC000B1FA81F14909002940F0B4807F2800F093
:100AD0002281A0F12001C9B25E29CED8FF2BCCD84B
:100AE000202801D1002AC8D15A1C09F803002A6025
:100AF00015F0FCFCC1E72C68002C59D1474B264669
:100B000003F51478002E08BF1E4610334345F9D173
:100B1000A3F1100B002E69D03068DBF80010075DE0
:100B200020440B5D21449F4240F03E8117B9FD2CCB
:100B300040F28781671E22464F44013207F8013F89
:100B40002A6010F8013F11F801EF9E450CD1002BEF
:100B5000F3D1FD2AF1D8531C2020002109F802000E
:100B60001A462B6009F80310B34500D192B92C48FE
:100B700015F0C4FCB34508D356F8100B15F0BEFCB5
:100B8000092015F0B3FC5E45F6D92648002415F07F
:100B9000B5FC2A689442BFF470AF661E4E4416F846
:100BA000010F013415F0A2FC2B689C42F7D364E7D7
:100BB0004FF0000B194F5E4607F5147802E010372E
:100BC00047450DD022463968484602F05BF90028B7
:100BD000F5D1BB46002EF2D13E4610374745F1D144
:100BE000002E99D1BBF1000F3FF447AF0C4800260F
:100BF00015F084FCC0E77F287FF46BAF3DE700BFB2
:100C00002874012034810120A29F01205029012055
:100C1000D88F0120A8540120FC4E0120B4100408F4
:100C2000542904085C290408FC4D0120F8F6030847
:100C3000F84D012015F0E3FC232192482EF078FCBA
:100C4000002800F0F680A0EB0900286088B1431E60
:100C500019F80310202940F0128109EB03023BB17F
:100C600012F8011D581E202933D10346002BF7D15D
:100C70002B604FF48072002148462EF042FC824BDC
:100C80001B78002B3FF49AAE804815F037FCF4E651
:100C90007F4815F033FC7D4815F030FCEDE614F884
:100CA000063C14F8051C99426FD814F8043C8342A2
:100CB0007FF4B8AE062304F8023C90E614F8043C36
:100CC000052104F8030C5A4004F8021C04F8042C13
:100CD0006AE62B6000226F4C09F8032004F51478B3
:100CE00002E0103444455BD02168484610F05CFDBA
:100CF0000028F6D0444553D2E368984700232B6080
:100D0000B7E7032204F8013C04F8022C4CE6022366
:100D100004F8023C48E6013B5F482B6009F80310E9
:100D200015F0ECFBA9E65D4B0121DFF88CE14022D8
:100D3000DB7887F818210033C7F80C01C7F81401D5
:100D400018BF012387F819518EF800304E4BDFF899
:100D50006CE119705249534BCEF80000C7F81011DE
:100D60005148C3F800B015F09FFF484815F0C6FB86
:100D70004FF400600DF02AFB4C4B93F83230232BDC
:100D80003FF447AE14F8023C27E614F8041C581C44
:100D90004344514004F8060C04F8041C9A7203E61C
:100DA000434815F0ABFBA9E7002C3FF4E0AEB34598
:100DB0007FF4DDAE61E614F8052C0DF1280E14F871
:100DC000030C012122440DF108084EF8243DADF832
:100DD00022300792ADF820008DF82410069499E88F
:100DE0000F0088E80F007246414606A805F05CFD3A
:100DF00040B1029A41462F4BA4F10A00039202939C
:100E00000EF040F80023DDF8048004F8023CB8F14D
:100E1000000F3FF4CFAD54F80A0C01360EF0BEF8C7
:100E200054F80A0CC047032E04F1CC047FF4A7AD9C
:100E3000C4E528680AE713480FF0ACFC0BB0BDE826
:100E4000F08F224687E614F8032C002114F8053CA5
:100E50006E2A08912344069409910793ADF8202047
:100E60007FF4C5AD06A802F095F806A802F086F852
:100E700006A802F083F806A802F080F8B7E503465A
:100E800028E700BFFC4D0120287401205C290408DC
:100E900064290408B41004088C290408149F012054
:100EA0006D0F0108A854012090290408D88F012053
:100EB0007029040890C90120EC300120F84D012070
:100EC00000210B4B10B40A460424017202E00729EA
:100ED0000BDC9C79A40702F1010202D51C79445471
:100EE0000131042A03F12403F1DD5DF8044B70475E
:100EF000A81E040810B404230E4C0022214613F04F
:100F0000010301F1240107D10132052A0DD08B79AB
:100F1000243113F00103F7D002EBC20204EB82028A
:100F20005DF8044B13790370704703705DF8044B50
:100F3000704700BFA81E04080B4B30B503F1140422
:100F400093F90020043313F8035C072AC8BF143A4E
:100F500081188D7213F8025C855413F8012CA3429A
:100F60000A75EDD130BD00BF08F7030803682DE90D
:100F7000F041DF691FB13B46BDE8F0411847002A48
:100F8000164611DD04460D460E4400E023689B68BA
:100F9000204698470028F9D02368204615F8011B01
:100FA0001B689847AE42F1D1BDE8F08100233C2197
:100FB0004222017042708370C3707047094B03F185
:100FC0000C0110B593F90020043313F8034C84543A
:100FD000024413F8024C147113F8014C8B42147242
:100FE000F0D110BD1CF70308002830B41FDB09281E
:100FF000044622DD012303EB83035B00B0FBF3F225
:10100000092AF8D87BB10F4DA5FB0320B4FBF3F2FE
:10101000092A03FB1244CCBF57233023134401F8A1
:10102000013BC308F0D1002330BC0B7070472D2367
:101030004042013101F8013CD9E7303001F8010BA1
:10104000F1E700BFCDCCCCCC884230B44FF00104E6
:101050002ED301FB04F4B0FBF4F58D42F9D284B138
:10106000AAB901E0B0FBF4F5092D04FB1500CCBFD3
:1010700057223022B4FBF1F4154403F8015B002C35
:10108000F0D1002230BC1A707047B0FBF4F5092D86
:1010900004FB1500CCBF37223022B4FBF1F4154419
:1010A00003F8015B002CF0D1002230BC1A707047AD
:1010B0000546002AEBD1D7E72DE9F84F14461D4627
:1010C00006464FF47A72002320462946DFF84CA1E9
:1010D0002CF016FB4B4A4FEAE07C4B4982FB007335
:1010E00040F2B55881FB0071484F034487FB00E78D
:1010F0000144CCEB63130744CCEBE12182FB03E218
:101100004FEAE379CCEB27478AFB01EA1A44C3EBA9
:10111000031BC9EB62193E4AA0EB8B0BC9EB091903
:1011200082FB07E24FEAE17E86F806B0A3EB890373
:10113000DFF8EC90CEEBAA0E737189FB0030FB1741
:101140000EEB4E0EC3EBE212A1EBCE0E08FB1272B9
:10115000CCEBE05C86F804E0B2F5896F4FEA8C0CCA
:101160003FDA40F2DA239A4243DCB2F5B77F294BEB
:10117000B4BF4FF000084FF001084FEA48091FFACA
:1011800088FE09EB080103EBC103DF8E224809EB5F
:1011900008010B2300EBC101163101E031F8027D9B
:1011A000BA421BDA013BF9D1C8441A49012301EBC9
:1011B000C808B8F820700CF2B27C01322046B37037
:1011C000E644D41B29464FF47A720023A6F800E0C7
:1011D000F4702CF095FA3281BDE8F88F0133DBB260
:1011E000E9E74FF0030E40F296574FF00609F0463C
:1011F000CCE74FF0020E40F229474FF00409F046C9
:10120000C4E700BF89888888C5B3A29107452EC26C
:1012100073B06D1608F7030828F70308ABAAAA2ACB
:10122000792D031103685A1C02601970704700BFC2
:101230002DE9F047089C002B8846074621780CBF13
:101240004FF020094FF03009651C39B3002A2ADD20
:101250002B4601E00246A8B113F8016B501E002E88
:10126000F8D1961E70B1B2460AF1FF3A49463846A7
:10127000C0470AF10103002BF6DC26EAE67021786C
:10128000013049B1041B3846C047281915F8011B25
:101290000029F8D1BDE8F087BDE8F087002A04DC1A
:1012A0000846BDE8F0870020ECE7561EDBE700BFEC
:1012B0008368D0ED037A416800EB8302013370EE5E
:1012C000277A82ED040A8B428360C0ED037A1ED038
:1012D00000EB8303026893ED047A914277EEC77ABC
:1012E000C0ED037A0CDA0132B7EE007A06EE902AEE
:1012F0000260F8EEE66A87EEA60A30EE070A70474B
:1013000007EE101AB8EEC77A87EE870A70470022F8
:1013100013468260DCE700BFD0ED007AB0EE406A91
:10132000D0ED056AD0ED015AE7EE806A90ED067ABD
:10133000D0ED047AA0EE257A90ED035AD0ED025A52
:1013400067EEE67AB0EE660AA6EEC57AE6EE257A94
:1013500080ED057AC0ED067A704700BF90ED057A02
:10136000F0EE406AD0ED017A90ED006A27EE270A90
:10137000D0ED064A90ED024AD0ED077AA6EE260A95
:1013800090ED035A90ED086AD0ED045AC0ED056A5D
:1013900080ED067AC0ED087AA4EE240AA5EE670A6D
:1013A000A5EEC60A80ED070A704700BFD0ED007AAF
:1013B00090ED017A30EE670AE7EE007AB0EE670A48
:1013C000C0ED007A704700BF704700BF0A449142E9
:1013D0001AD0013930B4551E41F2210411F8012F01
:1013E000082380EA022002E0013B90B209D010F409
:1013F000004F4FEA4002F7D084EA4000013B80B240
:10140000F5D18D42EAD130BC704770B544880D46A5
:1014100006460021C4F30B04284622462EF071F83C
:1014200033690A4A934209D3094A934206D22246B3
:1014300028461946BDE870402CF03CBE23B1214639
:101440002846BDE87040184770BD00BF4806000838
:10145000400700082DE9F0410F46016886B00546B7
:10146000C1F30D043B4E002C48D11022214602A8A6
:101470002EF047F8384B394801220221834204926A
:1014800005911FD900F58040834225D9344A934203
:1014900019D902F58042934220D902F58032934255
:1014A0001ED902F5003293421CD902F50032934254
:1014B0001AD902F50032934218D905202AF04CFDC2
:1014C000F9F75CFA2146337D0391012B10D14FF0DF
:1014D000FF3006B0BDE8F0811146F4E70321F2E7E2
:1014E0000421F0E70521EEE70621ECE70721EAE712
:1014F00001A902A814F008FE0028E8D1337D012BD1
:1015000002D16FF00100E4E70123D5F800803375C4
:1015100025F050FBB0B9134C236923F440732361C9
:10152000236943F400732361236943F001032361BA
:10153000C8F80070BFF34F8F25F03CFB236923F000
:1015400001032361002333750028DAD12B680433AB
:101550002B60BEE7CC93012000400008FF3F00084D
:10156000FFBF0008003C0240F8B504460D468E1847
:101570000027B54201D12069F8BDE368591C234416
:10158000E160042915F8012B1A72F2D1206918B90B
:10159000A1682046FFF75EFF2061E760E9E700BF32
:1015A000434B99895A89914210B501D300225A813F
:1015B000198ADA89914201D30022DA81DA78072A7E
:1015C00018BF002A3B4A3CD092F8572001213A4CE0
:1015D00000200A2A99702170D8715FD00C2A5BD143
:1015E000364CDFED377AA278062A3DD92179DFED36
:1015F000356A002940D19B782F4A07EE103A1178BE
:10160000B8EEC77A27EE277A07EE901AF8EEE77A57
:1016100067EE877AF4EEE76AF1EE10FA3BDDC6EE8C
:10162000877AFDEEE77A17EE903A102BA8BF1023C9
:10163000012BB8BF0123DBB28B4238BF0B461370BE
:1016400010BD92F857200A2A2BD00C2ADA792CD117
:10165000DFED1D7A002A9FED1B7A18BFF0EE477A66
:10166000164CA278062AC1D8184901EB8201D1EDA7
:10167000206A21790029BED0013A032A0BD8B7EE9F
:10168000000A80EE260A2CF081FF2388984228BFAA
:101690001846208010BD10BD0A2AA1D1DFED0C7ABA
:1016A000DEE7DA79DFED0B7AD4E7DFED0B7AD1E70D
:1016B000B09C0120D0940120C4700120D0A301204F
:1016C0006F12833A6F1203380AD7A33908F7030859
:1016D0000F506E3A5304E9386F12033901302DE987
:1016E000F04FC3B285B08D4C03930B4602918C4EE4
:1016F000002B00F09A8032208A4D2AF0CBFA8A4FD4
:101700004FF4FA7ADFF824924FF0100C4FF47A700D
:10171000D9F80430C3F30803002B40F0DE80EFF368
:101720001183002B40F0D9802968A26800BF2B6884
:101730009942F9D1D7F800E000FB0EF39B1AB3FBF6
:10174000FEF300FB01314FF0010E0191D9F8043096
:10175000C3F30803002B40F08780EFF31183002BC5
:1017600040F082802B68A16800BF2A689342F9D1BB
:10177000D7F800B000FB0BF2521AB2FBFBF200FBF1
:101780000323019A9B1AB3F57A7FDFD3BAF1010ADA
:10179000BED1039B002B40F0BD804FF47A7ADFF876
:1017A0008C914FF0100C5046D9F80430C3F3080365
:1017B000002B75D1EFF31183002B71D12968A2683A
:1017C00000BF2B689942F9D1D7F800E000FB0EF377
:1017D0009B1AB3FBFEF300FB01314FF0010E0191A8
:1017E000D9F80430C3F3080313BBEFF31183FBB93B
:1017F0002B68A16800BF2A689342F9D1D7F800B0DE
:1018000000FB0BF2521AB2FBFBF200FB0323019A1E
:101810009B1AB3F57A7FE3D3BAF1010AC4D1029BD4
:10182000013B0293002B7FF466AF05B0BDE8F08F5B
:10183000EFF311888CF31288A1682368DB0302D5CB
:10184000C6F800E0A1682B685FFA88F8326888F370
:101850001188D7F800801A4400FB08F35B1AB3FB29
:10186000F8F300FB0233D2E7EFF311888CF3128810
:10187000A1682368DB0302D5C6F800E0A1682B68E5
:101880005FFA88F8326888F31188D7F800801A4424
:1018900000FB08F35B1AB3FBF8F300FB023370E7BD
:1018A000EFF311828CF31288D4F808E02368D9038F
:1018B00003D501233360D4F808E02B68D2B2316835
:1018C00082F311883A68194400FB02F3A3EB0E037C
:1018D000B3FBF2F300FB01317FE7EFF311828CF3EE
:1018E0001288D4F808E02368D90303D501233360B4
:1018F000D4F808E02B68D2B2316882F311883A68D4
:10190000194400FB02F3A3EB0E03B3FBF2F300FB5D
:10191000013118E718462AF04FF83EE710E000E0E2
:1019200028B901202CB9012030B9012000ED00E0D8
:10193000214B5B68C3F3080310B4C3B9EFF3118301
:10194000ABB91E4B1E4C1868A16800BF1A689042C4
:10195000F9D11C4B4FF47A721C6802FB04F3591A3C
:10196000B1FBF4F15DF8044B02FB00107047EFF39C
:101970001182102383F3128811498C680B6813F4C9
:10198000803F114B02D0012018608C680B49D2B205
:101990000968186882F311880A4B4FF47A72084478
:1019A000196802FB01F31B1B5DF8044BB3FBF1F359
:1019B00002FB0030704700BF00ED00E02CB90120B1
:1019C00010E000E030B9012028B901202DE9F84FDE
:1019D00080461027FFF7ACFF244E844624494FF47D
:1019E0007A74DFF898E00120224A234DDEF80430B3
:1019F000C3F30803D3B9EFF31183BBB90B68D2F873
:101A000008A000BFD1F800904B45F7D1D6F800B040
:101A100004FB0BF9A9EB0A09B9FBFBF904FB0393DF
:101A2000A3EB0C034345E1D3BDE8F88FEFF3118A34
:101A300087F31288D2F808B01368DB0302D5286058
:101A4000D2F808B00B685FFA8AFAD5F800908AF3EA
:101A50001188D6F800A0994404FB0AF3A3EB0B030A
:101A6000B3FBFAF304FB0933DAE700BF30B9012016
:101A70002CB9012010E000E028B9012000ED00E0C1
:101A80002DE9F04FDFF830C180461027464A47491C
:101A9000474E484D18F1FF38C0F08480DCF8043020
:101AA000C3F30803002B5CD1EFF31183002B58D153
:101AB0000B68946800BF08688342F9D1D6F800909B
:101AC0004FF47A7000FB09FEAEEB040EBEFBF9FE8C
:101AD00000FB03EEDCF804304FF47A740120C3F30A
:101AE0000803FBB9EFF31183E3B90B68D2F808A040
:101AF00000BFD1F800904B45F7D1D6F800B004FBF9
:101B00000BF9A9EB0A09B9FBFBF904FB0393A3EB5F
:101B10000E03B3F57A7FBDD2DCF80430C3F30803BB
:101B2000002BDFD0EFF3118A87F31288D2F808B0C8
:101B30001368DB0302D52860D2F808B00B685FFA9F
:101B40008AFAD5F800908AF31188D6F800A0994453
:101B500004FB0AF3A3EB0B03B3FBFAF304FB093317
:101B6000D5E7EFF3118487F31288D2F80890136851
:101B7000D80303D501232B60D2F808900B68E4B298
:101B8000286884F311884FF47A74D6F800A000EB2B
:101B9000030E04FB0AF3A3EB0903B3FBFAF304FB04
:101BA0000E3E97E7BDE8F08F10E000E02CB9012071
:101BB00030B9012028B9012000ED00E030B4EFF386
:101BC0001183102282F3128808490025084CDBB2E9
:101BD0000A68084801320A602560026883F31188A8
:101BE000054A1368013330BC136070472CB90120DB
:101BF00028B9012010E000E0E893012003682DE9F6
:101C0000F041DF691FB13B46BDE8F0411847002AAB
:101C1000164611DD04460D460E4400E023689B681D
:101C2000204698470028F9D02368204615F8011B64
:101C30001B689847AE42F1D1BDE8F08103689B690B
:101C4000184700BF03685B69184700BF03681B693A
:101C5000184700BF0368DB68184700BF03685B686C
:101C6000184700BF03681B68184700BF014B18687E
:101C7000F8E700BF5C2A012038B50C46097849B165
:101C8000054601342B6828461B68984714F8011B49
:101C90000029F7D138BD00BF054B53F8203033B1D0
:101CA0001A689B8851690B4218BF1B0493617047E7
:101CB000F8B801202DE9F04FC1F3810383B0D0F8CB
:101CC00000E001F003088788C1F3411B009397FAF5
:101CD000A7F6B6FA86F608F1FF3A37FA06F363D0AC
:101CE0004FF001094FF0030C019103E0013637FA80
:101CF00006F358D009FA06F33B40F7D0DEF800505F
:101D000093FAA3F4B4FA84F493FAA3F0B0FA80F04F
:101D10006400BAF1010F4FEA40000CFA04F408FA2B
:101D200000F025EA040440EA0400CEF800004CD993
:101D3000DEF80C5093FAA3F4B4FA84F493FAA3F007
:101D4000B0FA80F06400B8F1020F4FEA40000CFADC
:101D500004F40BFA00F025EA040440EA0400CEF88B
:101D60000C00C3D193FAA3F0B0FA80F01C0A072844
:101D700042DCDEF8204093FAA3F0B0FA80F093FA48
:101D8000A3F30F21B3FA83F3800001369B0001FA1D
:101D900000F002FA03F324EA00000343CEF82030F7
:101DA00037FA06F3A6D10199BAF1010F0AD8DEF885
:101DB0000430C1F3001107FB01F123EA07070F43C9
:101DC000CEF8047003B0BDE8F08FDEF8085093FA47
:101DD000A3F4B4FA84F493FAA3F0B0FA80F06400A8
:101DE000009940000CFA04F401FA00F025EA04041A
:101DF0002043CEF808009BE7DEF8240094FAA4F311
:101E0000B3FA83F394FAA4F40F21B4FA84F49B0098
:101E1000A40001FA03F302FA04F420EA03032343C3
:101E2000CEF8243062E700BF10B50409013C042C51
:101E300017D80D4B00F00F0033F8142042FA00F3CE
:101E400013F001030DD0012303FA00F00138104014
:101E50002BF0A6FC054A064B125D104403EBC000B4
:101E600010BD002010BD00BF1C1E0408141E040875
:101E70007C8501202DE9F04F4C484FF0010A4C4978
:101E80004FF002094B4B4FF004084FF0080C4FF095
:101E9000100E202740268025474C30F8022B12F0E8
:101EA000010F03D01960083323F804AC12F0020FBD
:101EB00003D01960083323F8049C12F0040F03D0F8
:101EC0001960083323F8048C12F0080F03D019604E
:101ED000083323F804CC12F0100F03D01960083334
:101EE00023F804EC12F0200F03D01960083323F814
:101EF000047C12F0400F03D01960083323F8046CFF
:101F000012F0800F03D01960083323F8045C12F438
:101F1000807F05D04FF4807B1960083323F804BC20
:101F200012F4007F05D04FF4007B1960083323F8CA
:101F300004BC12F4806F05D04FF4806B1960083335
:101F400023F804BC12F4006F05D04FF4006B196045
:101F5000083323F804BC12F4805F05D04FF4805B93
:101F60001960083323F804BC12F4005F05D04FF465
:101F7000005B1960083323F804BC12F4804F05D0CD
:101F80004FF4804B1960083323F804BCD20B05D002
:101F90004FF400421960083323F8042C01F58061E6
:101FA000A1427FF47AAFBDE8F08F00BF1C1E040889
:101FB000000002407C8501200014024000B179E657
:101FC000704700BF08B1002274E6704710B1036883
:101FD00082889A61704700BF38B1002983880268FF
:101FE00014BF002110218B4093617047104B0146B4
:101FF0001B883BB90F4B104A1B7810680BB981F056
:102000000101E9E70D4B5A6982B118B91A681060ED
:10201000587470470A4801210A4A10B404881868A5
:1020200092FBF4F25DF8044B02605974704700BFF4
:1020300004B9012006B9012008B901200CB901201A
:1020400024B9012020A1070001230A4A10B48340CB
:10205000094C127854F82000134029B9B3FA83F1DF
:102060005DF8044B4909B7E7191C5DF8044B18BF2C
:102070000121B1E7F4B80120F8B801202DE9F041C1
:102080000B4E356873691D400FD0DFF8288001279B
:10209000B5FA85F4C4F11F0458F8240007FA04F4D3
:1020A00003689847A5437461F2D1BDE8F08100BF91
:1020B000003C0140F84C01202DE9F0410B4E356801
:1020C00073691D400FD0DFF828800127B5FA85F429
:1020D000C4F11F0458F8240007FA04F40368984771
:1020E000A5437461F2D1BDE8F08100BF003C01401E
:1020F000F84C01202DE9F0410B4E356873691D4005
:102100000FD0DFF828800127B5FA85F4C4F11F0449
:1021100058F8240007FA04F403689847A54374614B
:10212000F2D1BDE8F08100BF003C0140F84C012035
:102130002DE9F0410B4E356873691D400FD0DFF873
:1021400028800127B5FA85F4C4F11F0458F824004B
:1021500007FA04F403689847A5437461F2D1BDE817
:10216000F08100BF003C0140F84C01202DE9F04116
:102170000B4E356873691D400FD0DFF828800127AA
:10218000B5FA85F4C4F11F0458F8240007FA04F4E2
:1021900003689847A5437461F2D1BDE8F08100BFA0
:1021A000003C0140F84C01202DE9F0410B4E356810
:1021B00073691D400FD0DFF828800127B5FA85F438
:1021C000C4F11F0458F8240007FA04F40368984780
:1021D000A5437461F2D1BDE8F08100BF003C01402D
:1021E000F84C01202DE9F0410B4E356873691D4014
:1021F0000FD0DFF828800127B5FA85F4C4F11F0459
:1022000058F8240007FA04F403689847A54374615A
:10221000F2D1BDE8F08100BF003C0140F84C012044
:1022200003681B6A184700BF70B44E1C0568C27271
:102230008672AC69A44670BC604700BF2DE9F041CE
:102240000D4604461846164698462AF08FFD284447
:102250002768E6722946A07243467D6932462046C9
:10226000AC46BDE8F0416047036810B504461B6802
:102270009847236820469B689847A37B0133A37344
:1022800010BD00BF03681B69184700BF036810B585
:102290009B68044698470122FF232273637310BD95
:1022A00070B50546C06818B1848806682404B46116
:1022B00041F08001686840F2E93400E0E4B18668EA
:1022C000013C16F0020FA4B2F8D0017340F2E931DC
:1022D00000E039B38468013914F0010F89B2F8D0F5
:1022E000C16868680021F8F7BDFDEB6813B11A6892
:1022F0009B889361012070BD1849884228D0A1F5C0
:102300007841884226D001F580618842EAD10221D5
:10231000134CD82606FB01418C890134A4B28C8170
:102320008989DFE70D4CA04207D00E49884213D0BF
:1023300001F580618842D4D102210948D82404FBE8
:1023400001018889013080B2888189896868C9E77C
:102350002146DDE70121DBE70121EEE70030014006
:102360001C8201200038004030B4C3681BB19C8837
:102370001D682404AC61446840F2E93301E0002B9D
:1023800046D0A568013B15F0020F9BB2F7D0217330
:1023900040F2E93301E0002B4FD0A168013B11F07E
:1023A000010F9BB2F7D0E368446840F2E93300E0E4
:1023B000CBB1A168013B11F0020F9BB2F8D02273A0
:1023C00040F2E93300E073B1A268013B12F0010F63
:1023D0009BB2F8D0E368C36813B11A689B88936115
:1023E000012030BC7047234A944207D0224B9C42C4
:1023F00039D003F580639C42EDD102231F4AD821D6
:1024000001FB03239A89013292B29A819B89E2E708
:1024100018498C4207D0184B9C4226D003F58063A4
:102420009C42C2D102231549D82505FB0313998983
:10243000013189B299819B89B7E70E498C4207D057
:102440000D4B9C4213D003F580639C42ACD1022318
:102450000A49D82404FB03139989013189B299816F
:102460009B894468A1E70123C8E70123DBE7012337
:10247000EEE700BF00300140003800401C82012020
:1024800030B4C36801F07F011BB19C881D6824042F
:10249000AC61446840F2E93301E0002B46D0A56806
:1024A000013B15F0020F9BB2F7D0217340F2E933E4
:1024B00001E0002B4FD0A168013B11F0010F9BB24E
:1024C000F7D0E368446840F2E93300E0CBB1A1689B
:1024D000013B11F0020F9BB2F8D0227340F2E933B6
:1024E00000E073B1A268013B12F0010F9BB2F8D07B
:1024F000E368C36813B11A689B889361012030BCFC
:102500007047234A944207D0224B9C4239D003F5AE
:1025100080639C42EDD102231F4AD82101FB032393
:102520009A89013292B29A819B89E2E718498C42DA
:1025300007D0184B9C4226D003F580639C42C2D141
:1025400002231549D82505FB03139989013189B266
:1025500099819B89B7E70E498C4207D00D4B9C426D
:1025600013D003F580639C42ACD102230A49D824DE
:1025700004FB03139989013189B299819B894468CD
:10258000A1E70123C8E70123DBE70123EEE700BF52
:1025900000300140003800401C820120427A02B91C
:1025A0007047036800F10A0110B504464068984777
:1025B0000023637210BD00BF437A5A1C0344D2B299
:1025C00042729972037A93420AD84AB1036800F1C1
:1025D0000A0110B50446406898470023637210BD95
:1025E0007047074B07498B4202D3002318467047B8
:1025F0001A88C2F30B029042F8D01433F3E700BFFD
:10260000E801000848060008024A136823EA0000AF
:1026100010607047505701202DE9F047AC4F23F070
:10262000D5FEAC4EBE421ED2DFF82483DFF82493E1
:102630004446258862197DB14A450DD2052D0BD936
:1026400033886188C3F30B03994200F0E680144697
:1026500025886219002DEFD1716830461436FEF7D7
:10266000D4FEBE42E4D39C4A1378A3F11701022999
:1026700014D99A4911F83300002800F00081D800DD
:102680000C186468002C00F01B810144497829B1C2
:10269000934911F833300BB91823137091494B78D3
:1026A000022B00F2D980904A03EB43038F4802EBE0
:1026B00083030A78022A036000F2D78002EB8201CA
:1026C0008B4BC2EBC10203EB4203998C5A8C894CB1
:1026D0009142236001D300225A84874B9A78042ABE
:1026E00000F0E58022B91A88B2F5F07F00F2C380CD
:1026F000824DFEF755FF824A2B681A40002A00F0EF
:10270000E280D80700F1CE80590400F1C6801A0794
:1027100000F1BE809B0400F1B48021F029FE10B9C5
:1027200078480BF071FF4020FFF76EFF4FF4007008
:10273000FFF76AFF4FF40030FFF766FF4FF4001019
:10274000FFF762FF4FF00070FFF75EFF4FF0806011
:10275000FFF75AFF1EF098FE002130226A482CF045
:10276000D0FE20681DF0F2FD684B256803F1500192
:1027700002E0043399427CD01A78002AF9D19C787F
:10278000D8788442F5D262492846624BC8240A7040
:102790001D601BF02FFA604A6421604B15790022FE
:1027A0005F4811FB05415F4C9A605960DA601A611D
:1027B0005A619A61DA6183F8202083F8212004604D
:1027C00023F0F6FB584B9FED595A1B88584A06EEEA
:1027D000903A9FED586A1388F8EEE66A507907EE52
:1027E000103A53881279C5EE265A07EE903A524BAA
:1027F000524918725A72B8EEC77AF8EEE77A27EEA5
:10280000067A67EE867ABDE8F04783ED017AC3ED7C
:10281000007AC1ED005A23F0C1BD63799B077FF4B4
:1028200016AF7168304694F804A0FEF7EEFD3388C9
:10283000BAEB133F04D01436BE42FFF4F9AE12E7F0
:102840007388AA1FA11D7068C3F30B039A42A8BF27
:102850001A462BF02FFCEEE70022234B23484A7048
:102860000A780360022A7FF629AF0022204B0A7003
:102870002BE7012287E74FF4F0721A8038E7D8007F
:1028800003E72F48FFF7C0FE4020FFF7BDFE44E7F7
:102890002C48FFF7B9FE2B683CE72B48FFF7B4FE46
:1028A0002B6834E72948FFF7AFFE2B682CE79A8A9C
:1028B000B2F57A7FBFF41CAF4FF47A729A8217E7B1
:1028C00017241470E1E643F400532B6019E700BFAE
:1028D00048060008E8010008607101205C1F040838
:1028E000D0160408149F0120EA56012064790120C3
:1028F000DE55012060790120D0A30120505701202E
:1029000009600002D88F0120E8290120B45101207C
:10291000EC2201201C2A012034800120805C01204F
:10292000342A0120D6700120642F0120C0C9FB4841
:102930009C2D012017B7D138A07A0120682F0120E3
:102940000940000201600002092000020860000244
:102950000240000800800008F8B5174D2B78A52B21
:1029600028D16B78BE2B25D1AC1C144F02222946EE
:102970004FF6FF70FEF72AFD22884AB1A618BE4224
:1029800018D2052A16D921463446FEF71FFDF3E773
:1029900021460222FEF71AFD0222A1180634FEF794
:1029A00015FD074B641B1C8041F60F53C31A584298
:1029B0005841F8BD0020F8BD004000080080000824
:1029C000D44D01202DE9F04FDFF850918BB04E4FE0
:1029D0000326A7EB09071822002104A82CF091FD7B
:1029E0004A4BCDF8109005971A69002A04DA484A34
:1029F0005A6002F188325A6001230222694604A813
:102A00008DF824304FF0000B424B434C1B88DFF80D
:102A100010A1ADF80030FEF7A7FD022269464FF67F
:102A2000FF70FEF7D3FC804654453BD30AAC00252B
:102A3000022204A824F8245D2146FEF795FD022217
:102A400021464046FEF7C2FC40BA022202A9C0431A
:102A5000ADF8080004A8FEF787FD079878B106AB2B
:102A6000C0F10402294618442CF04BFD089818B90F
:102A7000069904A8FEF7EEFC0023089007939DF842
:102A80002430089A23B121490B6943F000430B61BC
:102A9000013E32D0002A9ED1FFF75EFF78B30BB023
:102AA000BDE8F08F658802A904A88DF80DB0C5F3C4
:102AB0000B051434AB1DADF8083034F8143CC3F3E7
:102AC0000B021B0BADF80A2006228DF80C30FEF726
:102AD0004BFD062202A94046FEF778FC804654F8DA
:102AE000101C2A4604A8FEF73FFD54F8101C40466F
:102AF0002A46FEF76BFC804696E7002ACCD00520DC
:102B000029F02AFAF7F73AFF00800008003C02405B
:102B100023016745A4F70308E80100080040000806
:102B2000480600080378092B01D0202B05D110F8A6
:102B3000013F202BFBD0092BF9D02D2B00F08980F1
:102B40002B2B00F08B80B7EE000AA3F13002D1B23C
:102B5000092900F29080F2EE046ADFED4A7A07EE6E
:102B6000102A10F8013FB8EEC77AA3F13002D1B2B3
:102B7000A7EEA67A0929F0EE477AF0D92E2B4BD092
:102B800003F0DF03452B39D110B442782D2A6AD0E7
:102B90002B2A6CD0411C0024A2F13003092B6DD8E4
:102BA000002303EB830302EB430311F8012FA2F18F
:102BB0003000303B0928F4D9B3F59A7FB7EE007A9C
:102BC00028BF4FF49A73072B09D91A46DFED2E6AF6
:102BD000083A27EE267A072AFAD803F007032BB122
:102BE000F2EE046A013B27EE267AFBD16CB1C7EE08
:102BF000876A5DF8044B20EE260A7047B7EE007A2C
:102C000067EE876A20EE260A704767EE876A5DF8EE
:102C1000044B20EE260A704743780130A3F13002BE
:102C2000D1B20929ACD8B2EE047AF0EE475A06EEDA
:102C3000902A10F8013FB8EEE66AA3F13002D1B253
:102C4000C6EE076A092927EE257A77EEA67AEED92D
:102C500096E74378BFEE000A013076E74378B7EE97
:102C6000000A013071E7811C8278012494E7811CFD
:102C70008278002490E7DFED037A7FE7B7EE007AF1
:102C8000B4E700BF0000000020BCBE4CB5EEC00A97
:102C9000DFED357A0023F1EE10FA30B5C8BF30EE23
:102CA000270A87B0D8BF30EE670ADFED307A0546D5
:102CB00003A9019320EE270A00930293FDEEC07A48
:102CC00017EE904A84EAE470A0EBE47020F08AFBEF
:102CD000002C03A8ACBF20232D238DF800302AF050
:102CE00045F8012829D0022833D003281DD003A994
:102CF00068462CF00EFC68462AF038F8C41E694677
:102D00002846E4B222462CF03BFC002328462B55F3
:102D10002AF02CF82E22431C0DEB04012A54E8184B
:102D20002CF014FC284607B030BD302303A96846B8
:102D30008DF801302CF0EDFBDDE7302303A9684668
:102D40008DF801308DF802308DF803302CF0E1FB66
:102D5000D1E7302303A968468DF801308DF80230A1
:102D60002CF0D7FBC7E700BF6F12033A00007A448C
:102D70002DE9F041064615460846B6FBF2F43CB98B
:102D800005FB1464124B1B5D00F8013BBDE8F081AC
:102D9000B4FBF2F767B90E4B05FB174705FB14644C
:102DA000DA5D1B5D00F8012B00F8013BBDE8F08106
:102DB000B7FBF2F8B8F1000F02D04046FFF7D8FF9A
:102DC00005FB1878024B13F8082000F8012BE3E705
:102DD000D82A0408104A2DE93048D2E9004554EABF
:102DE00005020CD103460022012110461A801A71F7
:102DF0005A719A711A819970D970BDE83088074B61
:102E00001A6814EB020B45F1000C5A466346FEF7B4
:102E100053F90120BDE83088A82D01202CB90120EC
:102E20000288A2F2B272F0B502F003048178C3788E
:102E300040F2B556013904EB4404013B9208DFF837
:102E400040E04FF47A7506FB023201EB8403067909
:102E500000210EEB4303447987791B8C00891344CE
:102E600003EB430306EBC303C3EB031304EB83033E
:102E7000C3EB031307EB8303C5FB0301F0BD00BFE6
:102E800008F70308FAB170B48E18044603E0101A6C
:102E900014D1B14214D014F8012BA2F14103192B23
:102EA00011F8013BA3F1410598BF203203F1200046
:102EB000192DECD9D01A01D1002BEAD170BC704782
:102EC000002070BC70471046704700BF4FF0FF32C3
:102ED000FFF7D8BFA0F16103192B98BF20387047C6
:102EE000A0F14103192B98BF2030704720280BD048
:102EF000092809D00A2807D00D2805D00B38012849
:102F00008CBF0020012070470120704761381928CC
:102F10008CBF002001207047413819288CBF002049
:102F200001207047303809288CBF002001207047ED
:102F3000A0F13003092B07D920F0200041381928CF
:102F40008CBF00200120704701207047026830B418
:102F50001146541CD31C151D046011F8024B01606E
:102F600051780360937805601B04D07843EA01230D
:102F7000234330BC43EA0060704700BF0368591C1C
:102F80001A46016012F8021B0260587841EA0020DC
:102F9000704700BF03685A1C02601878704700BF72
:102FA00038B50446006815462BF084F822682A4498
:102FB000226038BD03680A0A70B45E1C0D0E0C0C4A
:102FC00006601D7003685D1C05601C7003685C1C56
:102FD00004601A7003685A1C0260197070BC704754
:102FE00003680A0A10B45C1C04601A7003685A1C57
:102FF000026019705DF8044B704700BF03680A0E49
:1030000070B45E1C0D0A0C0C066019700368591C24
:1030100001601D700368591C01601C700368591C15
:1030200001601A7070BC704703680A0A10B45C1C17
:10303000046019700368591C01601A705DF8044B34
:10304000704700BF2DE9F047002488B080460F4646
:103050001E46A14605AD531C0393117841B32529A3
:1030600035D1931CCDF8109003935378302B52D068
:103070004FF0000AA3F13002D2B2092A44D96C2BD6
:103080001AD0642B00F09C8026D8252B1ED06BD93B
:10309000582B7ED0632B1DD1331D3178404601342F
:1030A0001E46B847039A531C039311780029D6D1C2
:1030B000204608B0BDE8F087039B5A1C03921B789A
:1030C000642B00F084802CD8252B5AD12521404632
:1030D0000134B847039ABEE7732B37D04AD9752B12
:1030E00055D106F1040E30682B4600220A2176469F
:1030F000FDF7AAFF049A5346009539464046FEF76D
:1031000097F8039A0444A6E7184604AA03A920F0F6
:1031100045F90346B3E7D31C4FF0010A03939378B4
:10312000A8E7732B12D060D9752B3FD0782B92D1A2
:10313000A3F1580206F1040E30682B46B2FA82F26F
:10314000102176465209FDF77FFFD3E7306806F17C
:10315000040E049A00230090394640467646FEF756
:1031600067F8039A044476E7002BB3D1204608B0F1
:10317000BDE8F0876E2BADD1039A336804361C602E
:1031800069E72BD9582BD3D0632B85D063E7782BF5
:10319000A0D1A3F15802311D30682B46B2FA82F259
:1031A0000E4610215209FDF74FFFA3E706F1040E6A
:1031B00030682B4600220A217646FDF745FF99E745
:1031C000331D306829461E46FDF70EFF92E7331D7A
:1031D000306829461E46FDF707FF8BE7002B7FF47A
:1031E0003AAF204608B0BDE8F0876E2BC5D032E775
:1031F0000EB410B585B0094907AC019001A854F888
:10320000042B23460394FFF71DFF019B00221A7035
:1032100005B0BDE8104003B0704700BF251201089B
:103220002DE9F04707468CB01E469246002A6BD126
:10323000154614460A8840F2B1739A423AD98B78FF
:10324000581E0B2836D891F803E00EF1FF301E28E7
:1032500030D891F804C0BCF1170F2BD891F8059025
:10326000B9F13B0F26D888793B2823D8B1F80880DC
:10327000B8F57A7F1ED24FF00108002E35D1002C10
:103280000E8903903846B4BF2D212B21002C0795C1
:103290000591B8BF64420496CDF80890CDF804C0FB
:1032A000CDF800E006943049FFF7A2FF40460CB08D
:1032B000BDE8F08700234FF0010A09A91846ADF8D0
:1032C00024308DF8283099468DF829309C468DF8A9
:1032D0002A301A46ADF82C309846D6468DF826A0EE
:1032E00053468DF827A0002EC9D003903846CDF85C
:1032F0000890CDF804C0CDF800E01C49FFF778FF36
:1033000040460CB0BDE8F087194BD417084683FB44
:103310000A235344C4EB6314C4EB041524B2AAEB90
:1033200085052DB2002DB8BF6D42FFF779FD4FF432
:103330007A720023804689462AF0E2F93C214FF454
:103340007A7200230AFB010A404649462AF0D8F95E
:103350004FF47A7192B2002309A8C1FB0A23FDF74A
:10336000ABFE09A966E700BF202B0408002B040868
:10337000898888880FB430B583B00C4B0C4806ACF4
:103380001968006854F8042B23460194FFF75AFE8D
:10339000084C05462068FEF755FC0028FAD0284660
:1033A00003B0BDE8304004B0704700BFEC4C0120D2
:1033B000F04C01205C2A0120DFED2A7AB4EEE70A06
:1033C000F1EE10FA4BDDDFED286A9FED287AB4EEBE
:1033D000C70A70EE667AF1EE10FAB0EE670AF6DC14
:1033E0009FED237AF4EEC77AF1EE10FA34D5DFEDD3
:1033F0001E6A9FED207AF4EEC77A37EEA60AF1EE48
:1034000010FAF0EE407AF6D4DFED1B7AB4EEE70A5C
:10341000F1EE10FA14DDDFED137A37EEC00A60EE3C
:10342000006A9FED166A9FED167ADFED167AA6EE1A
:10343000867A20EE266AE6EE877AA6EE270A70479D
:10344000DFED117AB4EEE70AF1EE10FAE7D5DFED21
:10345000087A37EEC00AE2E7B0EE670AD4E7F0EE8A
:10346000407ABDE7DB0F4940DB0FC940E4CB164192
:10347000DB0F49C0E4CB16C1DB0FC93F92E741B96E
:103480009730083C15A82ABEDB0FC9BF09B909E06F
:10349000194690FBF1F301FB13030846002BF7D10B
:1034A000084670470146FBE7B0EEC07AF0EEE06AEE
:1034B00086FE876AB5EE406AF1EE10FA39D0C6FE94
:1034C000C75AC5EE867ADFED1F2ADFED1F3ADFED22
:1034D0001F4A9FED1F5A9FED1F3AB7EE006A9FEDFE
:1034E0001E4ADFED1E5AE7EEE23AA7EE834AE7EE08
:1034F000A34AA7EE846AA7EEA45AE7EE855AC5EE62
:10350000867AF4EEC76AF1EE10FA03D59FED147ACD
:1035100077EE677AF5EEC00AF1EE10FA0CD4B5EE4C
:10352000C00AF1EE10FA48BFF1EE677AB0EE670A12
:103530007047DFED0A7AE4E79FED0A7A77EE677A63
:10354000EDE700BF39094E3DE3B59E3E88FA163ED1
:1035500045FE7F3F99FB243F69A2163EA7DFA834B2
:10356000DB0FC93FDB0F4940DFED307A30EE277AC1
:10357000FDEEC76A16EE903A2033402B02D99FED3C
:103580002C0A7047B4EEE70AF1EE10FA4BDD9FED1E
:10359000296ADFED296AB4EEE67A77EE467AF1EE33
:1035A00010FAB0EE677AF6DC9FED247AF4EEC77A73
:1035B000F1EE10FA34D5DFED1F6A9FED217AF4EEBB
:1035C000C77A37EEA60AF1EE10FAF0EE407AF6D49A
:1035D000DFED167AB4EEE70AF1EE10FA1BDCDFED50
:1035E000197AB4EEE70AF1EE10FA03D5DFED137A9B
:1035F00037EEC00A60EE006A9FED136A9FED137A02
:10360000DFED137AA6EE867A20EE266AE6EE877A5A
:10361000A6EE270A7047DFED0F7A37EEC00AE9E71A
:10362000B0EE670AD4E7F0EE477ABDE7DB0FC93F9B
:1036300000000000DB0FC940E4CB1641DB0F49C09E
:10364000E4CB16C1DB0FC9BF92E741B99730083C04
:1036500015A82ABEDB0F4940FDEEC07A17EE903A5E
:103660002033402B4FD8DFED2C7AB4EEE70AF1EE91
:1036700010FA4BDDDFED296A9FED297AB4EEC70A17
:1036800070EE667AF1EE10FAB0EE670AF6DC9FEDA6
:10369000257AF4EEC77AF1EE10FA3AD5DFED1F6A1B
:1036A0009FED217AF4EEC77A37EEA60AF1EE10FA12
:1036B000F0EE407AF6D4DFED1D7AB4EEE70AF1EED3
:1036C00010FA14DDDFED147A37EEC00A60EE006AFE
:1036D0009FED176A9FED177ADFED177AA6EE867ACF
:1036E00020EE266AE6EE877AA6EE270A7047DFED1F
:1036F000137AB4EEE70AF1EE10FAE7D5DFED097AB6
:1037000037EEC00AE2E79FED0E0A7047F0EE407A0E
:10371000BDE7B0EE670ACEE7DB0F4940DB0FC940DB
:10372000E4CB1641DB0F49C0E4CB16C1DB0FC93F28
:1037300092E741B99730083C15A82ABEDB0FC9BFF4
:103740000000000007EE901A9FED827AF8EE677A8B
:1037500027EE800A20EE070AFDEEC07A17EE903AB7
:103760002033402B00F28A80DFED7B7AB4EEE70A4B
:10377000F1EE10FA40F3E180B0EE407A9FED776A07
:10378000DFED776AB4EEE67A77EE467AF1EE10FA7C
:10379000B0EE677AF6DC9FED737AF4EEC77AF1EE5D
:1037A00010FA40F1CD809FED6D6ADFED6F6AF4EEA7
:1037B000E67A37EE867AF1EE10FAF0EE477AF6D432
:1037C000DFED6A7AB4EEE77AF1EE10FA4ADDDFED6A
:1037D000627A37EEC77A67EE075A9FED655A9FED1A
:1037E000656AF7EE007ADFED646AA5EE856A9FED03
:1037F000635A67EE254AE5EE866AF0EE675AA4EE54
:10380000A67AE7EE055AE7EE457A87EEA55ADFED90
:10381000577A30EE277AFDEEC76A16EE903A2033DB
:10382000402B30D9F6EE006A9FED557AB7EE006A6C
:10383000F7EE004A002380ED045A8361C4EEA57AB6
:1038400043610362C36167EEA66A27EE866A27EECC
:10385000877AC0ED006AC0ED026A80ED016A80EDF2
:10386000037A7047DFED477AB4EEE77AF1EE10FAAB
:10387000B1D5DFED3C7A37EEC77AACE7B7EE005A48
:10388000F0EE455AC3E7B4EEE70AF1EE10FA5DDD5B
:103890009FED326ADFED326AB4EEE67A77EE467A71
:1038A000F1EE10FAB0EE677AF6DC9FED2E7AF4EEC8
:1038B000C77AF1EE10FA46D59FED286ADFED2A6A45
:1038C000F4EEE67A37EE867AF1EE10FAF0EE477A09
:1038D000F6D4DFED267AB4EEE77AF1EE10FA27DCC3
:1038E000DFED287AB4EEE77AF1EE10FA03D5DFEDDA
:1038F0001D7A37EEC77A27EE074ADFED1D6ADFED46
:103900001D4AB7EE006ADFED1C7AF8EE003AE4EEED
:10391000264A27EE043AF6EE006AE4EE247AA3EE95
:10392000277A36EE476A27EE237A66EE266A7FE725
:10393000DFED097A37EEC77ADDE7F0EE407A2AE765
:10394000B0EE677A3CE7B0EE677AC2E7F0EE477A0E
:10395000ABE700BF27D4D236DB0F4940DB0FC940AD
:10396000E4CB1641DB0F49C0E4CB16C1DB0FC93FE6
:1039700092E741B99730083C15A82ABEF304353FB9
:1039800000000080DB0FC9BF70B406688E4219D9F1
:103990004C1E751E002314F8011F08224B4002E044
:1039A000013ACBB207D059001B06F9D581F0D503F7
:1039B000013ADBB2F7D1A542EDD1721C026033703F
:1039C00070BC70470023F8E710B401224C0901F0E5
:1039D0001F0150F8243002FA01F10B4340F8243063
:1039E0005DF8044B704700BF01234A0901F01F0135
:1039F00050F8222003FA01F1114214BF18460020AA
:103A0000704700BF2DE9F8433D4B1B78012B6CD06C
:103A10003C4B012605223C4819461E72DA744FF0D1
:103A200002081E7522F09AFCDFF8FCE04FF0000C53
:103A3000364F4B25DEF800302422354C43F00E0083
:103A400034493B6866711943334CDFF8E090334BDF
:103A5000CEF800001E20267003F1EA0E396019240A
:103A600089F80760462789F802806421DFF8C08062
:103A70004FF4C87688F803C0DD704E3303F84A2C43
:103A800003F8494C03F84E5C03F84D2C03F84C4CFA
:103A900003F8487C03F8472C03F8390C03F8370C7B
:103AA00003F8171C03F8181C23F81C6C7345E3D1AA
:103AB0001B4B64200021502203F1240655254FF4AE
:103AC000C86418700C3303F80B0C03F80A1C03F8D5
:103AD000072C03F8062C03F8055C03F8041C23F8F4
:103AE000024CB342EDD1BDE8F8830E4B40F29A2070
:103AF0004FF487614FF4FA62188019825A8287E77F
:103B0000B4B60120AC8F0120502B0408505701207F
:103B1000706D012000204030C4700120DE5501206E
:103B2000EA560120D0A30120A8510120B09C012019
:103B3000E070012038B50D4C0D4DAC4206D26168E5
:103B400020461434FDF761FCAC42F8D3FFF75AFF6E
:103B5000084C094B0022094D09490A481A705A704D
:103B600025600860BDE8384015F0D2B8E8010008CB
:103B70004806000860790120149F0120DE550120CD
:103B800064790120EA5601202DE9F04F2DED028BDA
:103B900093B005461BF064F9B54B1E7826B113B0FF
:103BA000BDEC028BBDE8F08FB24B1B685C05F6D50F
:103BB000DFF82483D8F80020002A00F01D81AE4CE5
:103BC000AE4BD4F828110B449D42C0F0158194F8F7
:103BD0002C31AB4F0133C4F828513968DBB2880768
:103BE00084F82C3101F18486090700F17F8113F0FC
:103BF000070901F02785282B01F0C987A14B029303
:103C00005E209047A04B1B78002B6AD09A4C9F4AAD
:103C1000D4F83431EB1A934201F2CC83DFF8BC8242
:103C200098F800A0BAF1000F32D1DFF87092D9F8FD
:103C30000000FEF713F8C0B201280ED9022842F0A6
:103C40006980934F3B78002B42F04981D4F83C3196
:103C5000EB1AB3F57A6F82F02F828E4F3A68002A02
:103C60003FD098F80030B3B98B4B0221D9F800004F
:103C70001B689B781E3B012B42F28B8104301AF0AB
:103C8000A5FF0122002388F8002084F8483126E0AF
:103C9000804F3A682AB3D4F8443140F6B731EB1A72
:103CA0008B421ED994F84031002B02F02980013B51
:103CB000DBB284F84031002B01F0888694F848E1AB
:103CC00094F8493112F8011B744801338E443A606C
:103CD000006884F848E184F84931FDF7C3FFC4F86F
:103CE0004451029B6E4A1B6812780133012A0A93E1
:103CF00001F085826B4B1B787BB1DFF8E4B1DBF818
:103D0000003053B1029B5C4CD3F80080D4F85C3196
:103D1000A8EB0303632B01F2AF81DFF8C88198F8A9
:103D200000A0BAF1020F01F02D86594F97F87430B8
:103D3000032B01F04F845C4B1B7873B15B4E3368EF
:103D40005BB14D4CFDF7F4FD44F61F620390D4F8CF
:103D50006831C31A934200F20F81554B1B78002B38
:103D60004DD1544B1B7843B1434C48F2E803D4F88F
:103D7000B82213449D4281F0BA824F4B1B78002B2E
:103D80003FF40DAF3C4E4D4C06F2C1274C4D206820
:103D9000FDF764FF00283FF402AF2068FDF75AFFEB
:103DA0002B7880465A1E33B120682A70FDF756FFE3
:103DB0000028F2D1F3E603223946781E2BF087FB68
:103DC00096F8C0124FF6FF7396F8C12286F8C382A8
:103DD0001FFA88F84B409B1A9BB2B8EB132FD6D131
:103DE000DBB296F8C2229A42D1D1781E1EF046FF6D
:103DF0002B7818442870CAE7224B029302E7314C13
:103E00002278002A41F0F281DFF8DCA09AF8004025
:103E1000002C40F09C802C4E3178002941F0D8874E
:103E20002A4E2B4B3278144C93FBF2F3D4F8B02289
:103E300013449D4295D3274A94F8B432C4F8B05243
:103E4000D75CF80702F17A81BA0702F101827B0799
:103E500002F1C0813A0702F1D68094F8B432317889
:103E6000013393FBF1F201FB123384F8B43278E7AB
:103E700028740120D49C0120AC2A012048E80100CC
:103E8000047901202CB90120127A01203F0D030092
:103E90000C000120787901207479012070790120CB
:103EA000137A0120207A0120287A01202C7A01201F
:103EB000507A0120517A0120327A0120387A01208B
:103EC0003C7A0120047A0120585D0120605D0120C8
:103ED000A08601005C5D0120807901207C790120B1
:103EE000EC780120EE4F0120595D012013F0030A08
:103EF0007FF47DAE5E209047D8F8003014209847BC
:103F0000194B1A4AB3F9043082FB03124FEAE379E2
:103F1000C9EBA2090FFA89F95FFA89F01AF0A8FE35
:103F2000C9F307201AF0A4FED8F800305E209847A5
:103F3000D8F800301C20984750461AF099FE504699
:103F40001AF096FE94F82C31D8F800204FE6084F6E
:103F5000386E002841F0F9858046064B8AF80080CB
:103F6000C3F8B052FDE600BF0879012067666666B7
:103F7000685D0120AC2A012094F86E31002B41F0DD
:103F80003585DF4B48F603404AF60B474BF60F42A8
:103F90001B6849F6074803F0080100294FF0190192
:103FA00004BF80463A4613F0040F84F86E1118BF20
:103FB0009046980603D548F4804848F020080AF057
:103FC0004FFDC8F30909002842F07C82CD4B9F7950
:103FD000002F42F0DA8264204FF0FF3A00230121E3
:103FE000FE220DF1280EADF836704FF01F0CCDF803
:103FF0002880CDF82C80CDF83090ADF838A08DF821
:104000004600ADF83430CDF83A30CDF83E30CDF83A
:1040100042306371E171A270BB4F84F803C0BEE807
:104020000F000FC79EE80F0007C71A0C27F8023BC6
:10403000C8233946781CA37101F81E2994F87E2103
:1040400082F0F103571C227183EA031384F87E7116
:10405000DAB2130983F0E70343EA022383EAC203D7
:104060001BB283EA0312C3F30723D2B283EA12130B
:1040700043EA022383EAC2031BB283F0C802C3F3FC
:10408000072382EA0212D2B283EA121343EA02231E
:1040900083EAC2031BB283F00102C3F3072382EA5F
:1040A0000217FFB283EA171242EA072282EAC70226
:1040B0001746228011F8013B7B40814283EA0313BB
:1040C000DBB24FEA131282EA172242EA032282EAA3
:1040D000C3031BB29FB22780ECD183F07C03DFF8CF
:1040E00038C204F1220883EA03130CF5D379DBB25A
:1040F0004FEA131E8EEA172282EA032E8EEAC30EBF
:104100000FFA8EFE1FFA8EF35FFA8EFE4FEA132A25
:10411000238084F827E084F828A0DCF800000CF164
:10412000100C5CF80C1C4F465CF8082C09F11009C7
:104130005CF8043CC4450FC7EFD1DCF80000734FB6
:10414000C9F8000007F127089CF8043089F804300A
:1041500084F8CDE184F8CEA117F8011F3068FDF78F
:1041600081FDB845F8D194F86F31002B41F04384BC
:1041700002980A226649D0F80090087884F86F21E6
:10418000002801F0E385DFF894C10128BCF8002085
:1041900042F205820228BCF8027002F0A981BCF844
:1041A00004100328049102F09A820428BCF806B097
:1041B00002F090820528BCF808A002F08782062849
:1041C000BCF80AE002F0E8810728BCF80C1001D026
:1041D000BCF80E3094F87E014FF0000CDFF84081FF
:1041E000059080F0300062F30F0CB8F8002080EAF0
:1041F0000010CDF8289067F31F4CC2EB0222C0B22A
:10420000444FCDF82CC04FF000084FEA101987FB3F
:10421000027C049F89F07A0967F30F089DF81470F7
:1042200049EA002927710CEB020789EAC0094FF01F
:10423000000CD2176BF31F480FFA89F90020C2EB6C
:10424000672267466AF30F0C4FF0230A61F30F07EA
:1042500089EA09118DF83D206EF31F4CC9B263F352
:104260001F47C9F30723059ACDF834C04FF0C80C97
:1042700083EA11130132CDF830804FF0160843EA7B
:10428000012384F87E2184F803800DF1280E83EA4F
:10429000C10384F806C00E974FF0FE091BB28DF8DB
:1042A0003C00607183EA0C02C3F30723164F82EAD5
:1042B000021284F807A084F80290D2B283EA1213A3
:1042C00043EA022383EAC2031BB283EA0A02C3F36E
:1042D000072C82EA02185FFA88F8BEE80F008CEA21
:1042E000181C0FC74CEA08229EE8030082EAC802A5
:1042F00047F8040BB81C228027F81419114611E066
:1043000004790120F4780120B42A0120532C0120E3
:104310003092012003082080AE2A0120CC5C0120CD
:104320007A5C012017F8013B4B40874283EA031374
:10433000DBB24FEA131282EA112242EA032282EA36
:10434000C3031BB299B22180ECD183F0F403DFF8F0
:10435000E89304F2A71704F2C51883EA0313D9F807
:10436000000009F5D37CDBB24FEA131E8EEA112E52
:104370008EEA032E8EEAC30E0FFA8EFE1FFA8EF31C
:104380005FFA8EFE4FEA132A238084F81EE084F839
:104390001FA0D9F80410D9F80820D9F80C30ACE8DF
:1043A0000F00D9F81000D9F81410D9F81820ACE88B
:1043B000070084F8C5A184F8C4E117F8011F30682C
:1043C000FDF750FCB845F8D194F87231002B41F05C
:1043D0002283D64B19221B6884F87221990640F17A
:1043E000F782D34B1B789A0741F17987D14F3B7DF8
:1043F000042B8CBF4FF003094FF00209FDF798FA28
:104400003B8A3A894FF47A7103EB83030DF1280A52
:1044100001FB02F239685B000A900E924FF000082F
:10442000ADF842304FF0FF300C91D446FB893A7D15
:1044300079688DF844904FF01809CDF82C800D91D3
:10444000ADF840308DF845200F90DFF8F4E2BCE87D
:104450000F00AEE80F009CE80F00AEE807000EF179
:1044600002012EF81C3984F807901E2294F87EC1B0
:10447000C82384F80580FE208CF07808E270A371D0
:1044800088EA0818A07084F804C00CF1010C5FFAE7
:1044900088F284F87EC1130983F0F60343EA02230D
:1044A00083EAC2031BB283EA0312C3F30723D2B227
:1044B00083EA121343EA022383EAC2031BB283F0A6
:1044C000C802C3F3072382EA0212D2B283EA1213AC
:1044D00043EA022383EAC2031BB283EA0900C3F35F
:1044E000072280EA0013DBB282EA131242EA0322B7
:1044F00082EAC302104622801EF8013B43408E45EB
:1045000083EA0313DBB24FEA131282EA102242EA73
:10451000032282EAC3031BB298B22080ECD183F05D
:104520001803854904F1220983EA031304918E4696
:1045300001F5D37CDBB2190981EA102282EA032259
:1045400082EAC3031AB293B2D2B2190A2380059247
:10455000069184F8262084F82710DEF800000EF17A
:10456000100E5EF80C1CE0465EF8082C0CF1100CE6
:104570005EF8043CCE45A8E80F00EED1DEF800005E
:10458000DFF8C481CCF800009DF8143008F126094A
:10459000C34684F8CC319DF8183084F8CD311BF82F
:1045A000011F3068FDF75EFBD945F8D1FDF7C0F972
:1045B000624BDFF898E14FF47A7CB3F904300021C4
:1045C0003A898EFB039E4FEAE3793B680CFB02F2CB
:1045D0007F684FF01C0C0B93C9EBAE030D92D646CF
:1045E000ADF8423021230E92FE220C970A90ADF8CE
:1045F0003C10ADF83E10ADF840106171E371A2704F
:104600004F4F84F803C0BEE80F000FC79EE80700B5
:10461000C82307F10C0C87E80700A371A7F110036A
:1046200094F87E1181F06A02481C217182EA02121C
:1046300084F87E01D1B20A0982F0D50242EA012251
:1046400082EAC10212B282EA0211C2F30722C9B29F
:1046500082EA111242EA012282EAC10212B282F017
:10466000C801C2F3072281EA0110C0B282EA101128
:1046700041EA002181EAC00109B281F02100C1F3C1
:10468000072280EA0011C9B282EA111242EA01222D
:1046900082EAC1021046228013F8011B41406345A3
:1046A00081EA0111C9B24FEA111282EA102242EAEC
:1046B000012282EAC10109B288B22080ECD181F0E6
:1046C00068011D4F04F1220981EA011107F5D37C2D
:1046D000C9B20B0983EA102383EA012383EAC103E9
:1046E0001AB293B2D2B24FEA132B2380059284F808
:1046F000242084F825B03868103757F80C1CE6469B
:1047000057F8082C0CF1100C57F8043C4F45AEE854
:104710000F00F0D13B88C1460A4FACF800309DF83D
:10472000143084F8CBB184F8CA3111E00479012047
:104730005E790120589F0120AE2A012008790120CE
:10474000B42A0120772C0120532C0120676666666D
:1047500019F8011F3068FDF785FA4F45F8D194F834
:104760007E110023DFF890E6312781F0EB020C93F5
:104770006371FE20DEF8043082EA021221710131F9
:10478000D2B20B93DEF800304FF00C0E84F87E119D
:10479000C8210A931309E77183F0C503DFF85C961B
:1047A000A07043EA0223A17184F803E083EAC20304
:1047B0001BB283EA0312C3F30723D2B283EA1213B4
:1047C00043EA022383EAC2031BB283EA0102C3F372
:1047D000072382EA0212D2B283EA121343EA0223C7
:1047E00083EAC2031BB25F40C3F3072387EA0717BC
:1047F000FFB283EA171343EA07239AE8070083EA24
:10480000C703A9F5D0771BB287E8070094F808E042
:10481000677A8EEA030EC3F30723A07A8EEA0E1E90
:10482000E17A227B5FFA8EFE94F80DC094F80EA018
:1048300083EA1E1343EA0E2383EACE0394F80FE0C3
:104840001BB25F40C3F3072387EA0717FFB283EA6F
:10485000171343EA072383EAC703277C1BB2584098
:10486000C3F3072380EA0010C0B283EA101343EABF
:10487000002383EAC003607C1BB25940C3F30723C3
:1048800081EA0111C9B283EA111343EA012383EAE1
:10489000C103A17C1BB25A40C3F3072382EA021270
:1048A000D2B283EA121343EA022383EAC203E27C10
:1048B0001BB28CEA030CC3F307238CEA0C1C5FFACF
:1048C0008CFC83EA1C1343EA0C2383EACC031BB25F
:1048D0008AEA030AC3F307238AEA0A1A5FFA8AFA02
:1048E00083EA1A1343EA0A2383EACA031BB28EEA55
:1048F000030EC3F307238EEA0E1E5FFA8EFE83EAD1
:104900001E1343EA0E2383EACE031BB25F40C3F3B8
:10491000072387EA0717FFB283EA171343EA07233F
:1049200083EAC7031BB25840C3F3072380EA001091
:10493000C0B283EA101343EA002383EAC0031BB228
:104940005940C3F3072381EA0111C9B283EA111365
:1049500043EA012383EAC1031BB25A40C3F307238E
:1049600082EA0212D2B283EA121343EA022383EAF2
:10497000C2031BB283F02707C3F3072387EA07129A
:10498000D2B283EA121747EA022787EAC2073FB288
:10499000BBB25FFA87FA4FEA132E238084F814A083
:1049A000049F84F815E038687968BA68FB68B7F83E
:1049B00010C0A9E80F0029F803CB84F8BBE184F804
:1049C000BAA118F8011F3068FDF74CF9C145F8D1BC
:1049D00094F87621002A41F01980DFF808E40521D7
:1049E00094F87E910AAFBEF9023089F06A00BEF9F0
:1049F00000C05B42627180EA001006EE90CA07EECA
:104A0000903ABEF90430C0B21E2207EE103A029B63
:104A1000E271FE22D3F800C00309A2701C2283F0C9
:104A2000D5034FF0000EE270C82243EA0023CDF810
:104A300038E0A271F8EEE66A83EAC003CDF83CE004
:104A4000CDF840E0F8EEE77A1BB2CDF828C0B8EE1A
:104A5000C77A9FEDDD6A83EA0310C3F3072366EE8E
:104A6000866A84F87611C0B267EE867A27EE067AF7
:104A7000DFF88C8383EA1013CDED0B6ACDED0C7A51
:104A800009F1010A43EA00238DED0D7A83EAC003A0
:104A90001BB25A40C3F3072382EA0212D2B283EA5E
:104AA000121343EA022383EAC2031BB283F01E0EF1
:104AB000C3F307238EEA0E1C5FFA8CFC83EA1C1EEC
:104AC0000FCF4EEA0C2EA8E80F008EEACC0E08F1AC
:104AD0000C0C97E80700A8F1100788E8070084F895
:104AE0000490A4F800E084F87EA117F8013B83EA63
:104AF0000E03674583EA0313DBB24FEA131282EA1F
:104B00001E2242EA032282EAC3031BB21FFA83FE7B
:104B1000A4F800E0E9D183F02703AC4F04F12208A8
:104B200083EA031307F5D37CDBB21A0982EA1E2E4F
:104B30008EEA032E8EEAC30E0FFA8EFE1FFA8EF354
:104B40005FFA8EFE4FEA1329238084F824E084F86C
:104B500025903868103757F80C1CE24657F8082C97
:104B60000CF1100C57F8043C4745AAE80F00F0D1AF
:104B7000DFF890823B8808F12407ACF8003084F815
:104B8000CAE184F8CB9118F8011F3068FDF76AF884
:104B90004745F8D194F877B1BBF1000F40F030876A
:104BA0008B4B05221B6884F877219B0641F1DA8044
:104BB000884BDFED896ADA891B8907EE902A07EEB8
:104BC000103AF8EEE77AB8EE477A67EEA67A94F8EC
:104BD0007E814FF0640E814A0DF1280A88F022038D
:104BE0007F48B2F90620574683EA031384F804800D
:104BF000B2F5FA6F08F101085FFA83FC7949A8BFA2
:104C00004FF4FA6284F87E814FEA1C13B1F9041064
:104C1000B2F57A7FCDED0B7A83F059038DED0C7AE6
:104C2000B8BF4FF47A7243EA0C23A2F57A7283EA92
:104C3000CC030EFB02F2DFF8D0E11BB280FB028056
:104C4000D2178EFB01CEC917C2EBA0124FF0000C99
:104C500083EA0310C3F30723ADF83A204A22C0B217
:104C6000CDF828C0E271FE2283EA1013CDF834C0DB
:104C7000C1EBAE01A27043EA00231422ADF8381054
:104C8000C82183EAC003E2700022DFF874C11BB2BE
:104C9000A171627183EA0102C3F3072382EA02125F
:104CA000D2B283EA121343EA022383EAC2031BB29D
:104CB00083F04A0EC3F307238EEA0E185FFA88F8D2
:104CC00083EA181E0FCF4EEA082E3F68ACE80F00AB
:104CD0008EEAC80E6246A4F800E0111D42F8107971
:104CE00012F8013B83EA0E038A4283EA0313DBB224
:104CF0004FEA131080EA1E2040EA032080EAC30333
:104D00001BB21FFA83FEA4F800E0E9D183F014037C
:104D10002E4A04F2C31983EA0313114604F2A712C0
:104D2000DBB20868174601F5D37C1A09B84602972A
:104D300082EA1E2E8EEA032E8EEAC30E0FFA8EFE34
:104D40001FFA8EF35FFA8EFE1A0A23800B4684F850
:104D50001CE0627717460A46DB684968049292684D
:104D6000ACE80F00ACF5DB7210695169138BACE84D
:104D70000300ACF8003084F8C371474684F8C2E100
:104D800018F8011F3068FCF76DFFC145F8D1164BCC
:104D9000164A1B781278013B029712F00101DBB230
:104DA00014BF4FF0C00C4FF0400C172B03D8104A23
:104DB000134493F814B00F4B1B889F0701F08C80AD
:104DC0004CF0100C002221E088C3E43AAE2A012006
:104DD00004790120589F01200AD7233CCC5C012094
:104DE000D34D6210087901206071012034810120C7
:104DF000A8F703085C790120CC5D0120542C012028
:104E0000B42A0120532C01206766666613F4027FE2
:104E100018BF022213F0100F18BF062213F0200F44
:104E200018BF1022002941F037814FF0030E94F88B
:104E30007E0103230A92002180F046028DF8303073
:104E400000F10109207182EA0212C8208DF82EC0FB
:104E50004FF0090CD2B28DF82CB084F803C04FF09B
:104E6000FE0813098DF82FE08DF82D1083F09203C2
:104E7000E171617143EA0223A071DFF824E583EA5E
:104E8000C20384F87E9184F802801BB283EA031285
:104E9000C3F30723D2B283EA121343EA022383EA5D
:104EA000C2031BB283EA0002C3F3072382EA0212A1
:104EB000D2B283EA121343EA022383EAC2031BB28B
:104EC00083EA031CC3F307235FFA8CFC83EA1C13F9
:104ED00043EA0C239AE8070083EACC03AEE8030018
:104EE0001BB294F80890607A0EF5CC7C89EA03092D
:104EF000C3F30723A17A0EF5D47889EA09198EF84D
:104F00000020E27A5FFA89F994F80CA094F80DB0C9
:104F100083EA191394F80EE043EA092383EAC903EC
:104F200094F80F901BB25840C3F3072380EA001097
:104F3000C0B283EA101343EA002383EAC000237C53
:104F400000B24140C0F3072081EA0111C9B280EAF2
:104F5000111040EA012080EAC10109B24A40C1F3C0
:104F6000072182EA0212D2B281EA121141EA022139
:104F700081EAC20212B28AEA020AC2F307228AEA6C
:104F80000A1A5FFA8AFA82EA1A1242EA0A2282EAC4
:104F9000CA0212B28BEA020BC2F307228BEA0B1B86
:104FA0005FFA8BFB82EA1B1242EA0B2282EACB02F7
:104FB00012B28EEA020EC2F307228EEA0E1E5FFACA
:104FC0008EFE82EA1E1242EA0E2282EACE0212B25D
:104FD00089EA0209C2F3072289EA09195FFA89F905
:104FE00082EA191242EA092282EAC90212B283EA6B
:104FF0000201C2F3072281EA0111C9B282EA111249
:1050000042EA012282EAC10212B282F0320EC2F3F7
:1050100007228EEA0E11C9B282EA111E4EEA012E53
:105020008EEAC10E0FFA8EFE1FFA8EF25FFA8EFE26
:105030004FEA1229228084F811E084F81290049F2C
:1050400038687968BA68B7F80CA0029FACE8070026
:105050008CF80230ACF800A084F8B89184F8B7E17D
:1050600017F8011F3068FCF7FDFDB845F8D1039B28
:10507000C4F86831FEF771BEBA4F412019F0E4F967
:10508000DFF818A3B7F90230DFF818938AFB032082
:10509000DB17C3EBA00080B219F0BAF9B7F9003002
:1050A0008AFB0320DB17C3EBA00080B219F0B0F934
:1050B000B7F904308AFB0320DB17C3EBA00080B2F2
:1050C00019F0A6F999F80010DBF80000FCF7CAFD0A
:1050D00094F8607117F0010300F0C484A24B1B68C0
:1050E0009B0673D5A14B1B78980740F14E87A04FC4
:1050F0003B7D042B8CBF032302234720039319F02D
:10510000A3F9386819F04CF9786819F049F9B7F83B
:105110000EA0984ADBF80000A2FB0A3ACAF3471A2D
:105120005146FCF79FFD99F800103A8964208AEAFD
:10513000010A00FB02F089F800A019F031F9039B85
:105140003F7DDBF8000043EA8707FFB23946FCF7F2
:1051500089FD99F80030DBF800005F40394689F896
:105160000070FCF77FFD94F860717FBBDFF838A218
:105170004F2019F069F9DAF8000019F011F9DAF89E
:10518000040019F00DF9384619F00AF90121DBF88D
:105190000000FCF767FD754A99F80030177883F036
:1051A0000103DBF8000007F0010789F800303946F9
:1051B000FCF758FD99F80030DBF800005F403946F5
:1051C00089F80070FCF74EFD94F860717B1C6A4A08
:1051D000C4F85C81DBB2A2FB0312D20802EB8202AC
:1051E000A3EB420384F86031FEF797BD634B64493B
:1051F0001868FCF703FD00232370FEF705BE614F1E
:10520000386800283EF476AD4FF00009DFF89C8145
:105210005D4CFCF723FDB9F1000F22D108B34FF02C
:1052200001094FF0000A3868FCF714FD83B27E2BA9
:1052300000F0BD8398F80120002A4AD194F84C115F
:10524000B1B11B2B84F84C2100F08B830D2B46D081
:10525000386888F80190FCF701FD0028E3D14FF091
:10526000000948460AAA494919F008F9FEF742BD63
:105270007D2B00F0618594F8502122B180F020034D
:1052800084F85011DBB294F84B21062A10D8B4F8F8
:105290004E11501C2244194484F84B013868A4F87C
:1052A0004E1182F85431FCF7D9FC0028BBD1D6E767
:1052B000B4F84E2188F8019013449BB21A0A52FAAE
:1052C00083F3FF2BA4F84E3103D13868DFF8E09068
:1052D0009FE73868FCF7C2FC0028A4D1BFE7386814
:1052E000A4F84E21FCF7BAFC00289CD1B7E794F84B
:1052F000BC32C4F8B852012B40F2068594F8BD22A6
:1053000023499818013201EB800102F00102CE6AB4
:1053100084F8BD22CEB11F4B0DF1480A4FF0A50E07
:105320008022A3F112070B93152329464AF8207D0A
:10533000504684F810E184F8112184F81231B04706
:10534000002840F0608494F8BC320133124A82FB9A
:105350000312A2EBE37202EB42029B1A84F8BC3206
:10536000FEF70BBD08790120047901205E79012048
:10537000589F01201F85EB51CDCCCCCC545D012032
:10538000C47901206C790120AC2A0120F62B012080
:10539000A8F70308D12B0120565555556766666658
:1053A000B42A0120F0780120CC5D01200C000120FE
:1053B000002C0120924A4FF47A71924B4FF0000E6C
:1053C000D07A1B8801FB00F102988F4A5FFA83FCB8
:1053D00007681B0AD4F8380182F81EC0381AD37740
:1053E00082F814C08842537582F802E082F804E023
:1053F00080F0768485494FF0F40E854F01200B68CC
:105400004FF0750A896887FB03C8DB1787FB017CAF
:10541000C917C3EBA8037F4FC1EBAC01DFF808C28B
:1054200013771B129CF800C04FEA212953774FF0E5
:10543000300882F820101CF0020F397D764B82F87C
:105440001AE04FF0780E82F821909976D07682F8A3
:10545000228082F823A082F824E000F03E84D7F86E
:10546000009005296D4A79684FEAE97882FB090EB8
:105470006B48039182FB01C24FEAE17CC8EBAE515D
:10548000DFF8A881CCEBA25C039A00FB019E01EB44
:10549000810100FB0C200CEB8C0C0EEB4E0E00EB94
:1054A00040004FEA4E0E4FEA400088FB0EA201EB8F
:1054B00081014FEAEE7A88FB00B84FEAA2420591DB
:1054C000B7F808B04FEAA848F989A2EB0A074FEAF3
:1054D000E07A0BF5FA7B3A467FB201EBC101069701
:1054E0000CEB8C07DFF848C14FEA810107974FEAC0
:1054F000D9790CFB12E2A8EB0A0E04911FFA8BFA81
:105500000599F046069F0CFB1E0E4FFA88F8454899
:1055100007EB8107079983F8099008EB810C049940
:10552000DFF81081BFB21FFA8CFCDFF80C9188FB0A
:10553000011804999F724FEA17274FEAE17183F827
:105540000FC0049180FB021B4FEAE27280FB0E1039
:1055500004990497C2EB6B12039F4FEAEE7EC1EBF6
:10556000A811B9F800804FEAD77B9DF81070CEEBF8
:105570006010DFF8C8E0DF724FEA1C2783F80EB036
:105580004FEA222BBEF800E0C1F3072983F80DB0E3
:105590004FEA202C1F7438BF4FF0320B1A734FEABA
:1055A0001A274FEA182228BF4FF0330B587483F89C
:1055B00012C083F815A09F75D97183F8089083F8FD
:1055C00013801A7583F81BB083F81CE0C4F83451BB
:1055D000FEF724BBDFF86890D9F80000FCF732FB37
:1055E00000283EF4A8ABD9F800000121FCF726FB07
:1055F0000222002387F8742088F80030FEF79BBB56
:10560000DC810120D4810120FC5C01202C77012069
:1056100067666666589F0120285D01206BCA5F6B34
:10562000806967FF1F85EB515E79012083DE1B4394
:1056300040420F00D34D621068790120385E01208E
:105640007C5401205E209047D8F800300220984713
:10565000FF201DF093FA0378FF2B00F0938490F95C
:1056600001304FEAE379D8B25FFA89F919F000FB0B
:10567000484619F0FDFAD8F800305E209847D8F86F
:10568000003003209847FF201DF078FA0378FF2BA5
:1056900000F02B84B0F90830D8B2C3F3072919F011
:1056A000E7FA484619F0E4FADD4B1B78042B7FD06B
:1056B000DFF89CB34FF0640EB4F82E315E209BF8F7
:1056C0000090DFF890A393FBF9F2BAF8001009FB01
:1056D0001232D8F800300EFB019192B24FEA49091C
:1056E000A4F82E21B1FBF9F14FEA0219C1F303220C
:1056F0001FFA89F949EA01291FFA89F949EA0209D9
:105700009847D8F80030062098475FFA89F019F0DA
:10571000AFFA4FEA192019F0ABFAC24AB4F82E31A9
:10572000517A0133BAF800900129A4F82E3100F023
:10573000F58609EB8909537B1FFA89FA002B40F0A3
:10574000B584D8F800305E209847D8F800303A2069
:105750009847B54BA3FB0A394FEA59191FFA89FB41
:105760005FFA8BF019F084FA4FEA1B2019F080FAE7
:10577000D8F800305E209847D8F800303B20984792
:105780006423AA4803FB19A39BB2053380FB0320C3
:10579000DB17C3EBA000C0B219F06AFA002019F0C1
:1057A00067FADFF8B49299F80630002B40F0F583E1
:1057B0003B68980640F1BC81DFF8A0A29AF800305F
:1057C000990700F197839A4F4FF00009CB46D8F81C
:1057D00000305E209847D8F800300120984758469E
:1057E00019F046FA484619F043FAD8F800305E201E
:1057F0009847D8F8003009209847002019F038FA67
:10580000002019F035FA7B8A97F814B0B3F5967F2B
:105810000AD994F82C2102F00F02072A04D842F288
:105820000F7B9B4528BF9B46D8F800305E20DFF8F1
:10583000F4919847D8F800300520984799F8083037
:10584000002B00F05185ABF120039FED7A6AF6EE54
:10585000006A07EE903ABEEE007AF8EEE77A67EE5D
:10586000867AF5EEC07AF1EE10FA58BFB0EE667A9D
:1058700077EE877AFDEEE77ACDED027ABDF908B0D2
:105880005FFA8BF019F0F4F9CBF3072019F0F0F977
:1058900000239AF8002008930993930700F11183DD
:1058A00094F83031012B00F00C83B9F900300AA8CC
:1058B000DFED616A07EE103AB9F9023007EE903A6F
:1058C000B8EEC77AF8EEE77A27EE267A67EEA67A80
:1058D000BDEEC77AFDEEE77A8DED0A7ACDED0B7A53
:1058E00019F0E8F994F82C31D8F80020FEF783B9C4
:1058F000DFF86C914FF0240B9FED508A5E209047AB
:105900005846D8F800300BF1010B98474C4BF9EC96
:10591000016A5FFA8BFB1B8BF8EEE66A07EE103A22
:10592000B8EEC77AC6EE877A67EE887AFDEEE77A38
:10593000CDED027ABDF908A05FFA8AF019F098F966
:10594000CAF3072019F094F9BBF1270F02D0D8F859
:105950000020D3E794F82C313968D8F80020FEF7FE
:1059600043B93868FCF77AF900287FF471AC3868DD
:1059700084F84A9188F80190FCF770F900287FF4C8
:1059800052AC6CE4FBF7D4FF2E4A40F6B8331268F1
:10599000A0EB020B9B4500F2C4812B4B1A793A2AEB
:1059A00000F0AC84002388F80030FEF7C4B93868F2
:1059B00084F84AA184F84BA184F84C9188F801A09E
:1059C000FCF74CF900287FF42EAC48E494F8481119
:1059D00094F849311D484A1C0133006884F8482175
:1059E00084F84931FCF73EF9FEF779B9013B84F8B8
:1059F0006E31FEF7B8BB013B84F86F31FEF7E4BCB3
:105A00000BF1FF3A84F877A1FFF731BB013A84F834
:105A10007621FFF7BFB8013B84F87231FEF7D8BF9B
:105A20007D5C0120DC8101201F85EB516766666685
:105A3000589F0120E4380E3F0050C34700007A44CD
:105A400010790120F44F0120DC4F012070790120F2
:105A5000EA810120D4810120F47801205E790120BF
:105A600044790120C74A1288D10500F17981D00616
:105A700000F11083910600F14285530600F167851D
:105A8000100700F17C85D10700F17C8512F0020F30
:105A90000CBF04270C27BC4BBC4A1B78D27803F000
:105AA00001030AB143F0020353201F4318F0CCFC5A
:105AB000B74B1B8803EB830303EB8303980080B28F
:105AC00018F0A6FC002018F0A3FCB24BB24A1B88C9
:105AD000DBF80000C3EBC3135B0082FB03124FEA49
:105AE000E37A1344CAEB632A5FFA8AFA5146FCF759
:105AF000B9F899F800300021DBF800008AEA030ABF
:105B000089F800A0FCF7AEF83946DBF80000FCF796
:105B1000A9F899F80030DBF800007B40DBB21946A9
:105B200089F80030FCF79EF894F86071FFF71DBB10
:105B300018077FF5D7AE994A0AAB92E8030083E8CD
:105B40000300184619F0B6F8CCE60024DFF87C9282
:105B50004FF0500BA04601E081F311883E5D601CC0
:105B60003146384418F02CFB002840F00181731CAA
:105B70001C44EFF311838BF312883A6ED9B294422E
:105B8000EADB00223A6681F31188FEF7E6B9844B1E
:105B90004FF000095E20834F029384F82C911C681B
:105BA0009047D8F8003017209847484619F060F819
:105BB0007D4BA3FB04239B0BA7FB03125209C2EBF3
:105BC0000212A3EB8203D8B219F052F8D8F80030D1
:105BD0005E209847D8F8003018209847734BA3FBF5
:105BE00004239B09A7FB03125209C2EB0212A3EB89
:105BF0008203D8B219F03CF8484619F039F8D8F8C1
:105C00000020FDF7FDBF0A9EBE4240F29D843D4646
:105C1000002141F2210015F8013B81EA03235900DC
:105C200013F4004F80EA010289B292B208BF0A461B
:105C3000530012F4004F80EA03029BB292B208BFF5
:105C40001A46530012F4004F80EA03029BB292B24C
:105C500008BF1A46530012F4004F80EA03029BB2B9
:105C600092B208BF1A46530012F4004F80EA0302B2
:105C70009BB292B208BF1A46530012F4004F80EA5A
:105C800003029BB292B218BF1346590013F4004F9F
:105C900080EA010289B292B208BF0A46530012F4A8
:105CA000004F80EA03019BB289B208BF1946B54292
:105CB000B1D15046FDF7B8F93D4B0A9D19463D4814
:105CC000ED1A152DA8BF15252A4628F0F3F93A4AF2
:105CD00094F8BC321570FFF738BB2D22DA7675E4E4
:105CE000364B02991B780968013BC4F83811012B27
:105CF0003FF680AB1021022391701371FFF77ABB3E
:105D000018F098FFFDF7EBBF244A02EB8302D66A36
:105D1000FFF700BB18F07EFF294F01233B70FDF712
:105D20009CBF284A0021B2F8623188F80010013384
:105D3000A2F86231FDF7FFBF386884F85091FBF795
:105D40008DFF00287FF46FAAFFF789BA01468646C7
:105D5000824683460490074602460346FEF73ABA57
:105D60001F4698E6DFED187AB0EE677AFEF72FBF90
:105D700049463A2018F07EF940EA08085FFA88F8A8
:105D8000F5E600BF5C79012034810120805C0120B0
:105D9000D48101207A5C012003082080A8F7030841
:105DA0002CB901208988888873B2E745D34D6210E9
:105DB000BC2B01203C910120519101207D5C0120F0
:105DC0000C000120AC2A01200000000011EE0208A6
:105DD000CB490AA8CB4BA1F13F07CB4A00930991CD
:105DE000CA4B01F8404CCA490897FDF701FA089FD1
:105DF0002920EA21C8227B1C08933C70089B03F1F0
:105E0000010ECDF820E018700AA8089B03F1010EDE
:105E1000CDF820E01970089B591C08911A7026F0E3
:105E2000A5FF00F101080AA90898424628F042F9A6
:105E30000899012212A801EB08031344089301F802
:105E40000840089B991808911C70089B99180891A4
:105E50001C70089B991808911C70089B9918089150
:105E60001C70089B991808911C70089B9918089140
:105E70001C70089B991808911C70089B9918089130
:105E80001C70089B991808911C70089B9918089120
:105E90001C70089B991808911C70089B9918089110
:105EA0001C70089B991808911A7050F8283DDB1B4C
:105EB0003B7018F091FF974B3470C3F8B052FDF768
:105EC00050BF97E80C00012108A8089284F830110F
:105ED000099318F0EFFE05E50122FEF797BFC4F81D
:105EE0003C5187F800A0FDF7B8BE4FF000094846C6
:105EF000FFF7D5BB884F5E20D8F800304FF4F36B26
:105F00009847D8F800301120DFF828929847FA898E
:105F10000BFB02F289FB0239D217C2EB69395FFA37
:105F200089F018F0A5FEC9F3072018F0A1FED8F8F3
:105F300000305E209847D8F8003019209847FB8938
:105F4000764A64210BFB03F382FB03E0DB17C3EB10
:105F5000601382FB0320DA17C2EB601201FB1233DD
:105F6000D8B218F085FE002018F082FE9AF80030B2
:105F7000B7F808909A077FF527AC5FFA89FB4FEADC
:105F8000192924E44846FFF771BB0123624FFFF74C
:105F9000B4B8FBF753FEFDF774BED8F800305E20AE
:105FA000DFF894A19847D8F80030282098475C4A39
:105FB000DAF800304FEAE37B82FB0323CBEBA30B41
:105FC0005FFA8BF018F054FECBF3072018F050FE68
:105FD000D8F800305E209847D8F800300420984761
:105FE000B9F80830002B40F09082DAF8083083F3DB
:105FF00010095FFA89F018F03BFEC9F3072018F08A
:1060000037FEFFF7D5BB3E4B0DF1480A0020424F4B
:10601000A3F13D01A3F1400203F8400C4AF8201D12
:1060200011210B9302235170504693703968FCF78D
:10603000C1FF50467968FCF7BDFFFB8938495046DF
:1060400003EBC3039B00053381FB0321DB17C3EB89
:10605000A10189B2FCF7C4FF3B8A504603EB8303DE
:10606000590089B2FCF7BCFF2E4B1B789B0740F10F
:106070004982398901F57A7189B25046FCF7B0FF3F
:106080000A9B3A7D5046591C0A911A7018F0A4FEDA
:10609000FDF7E3BE3427FEE4234BDB78002B0CBF77
:1060A0004FF0040E4FF0050EFEF7C1BE9BF8003016
:1060B0009AFBF3FAFFF745BB0123D9F800003B70C8
:1060C000FBF7C8FD0746D9F80000FBF7C3FD7906CA
:1060D00002D080287DF4C1AD8A2800F03F828E284E
:1060E0007DF4BBAD98F80030002B7DF4D1AD0F4F9F
:1060F0002D220F4B84F840213B603A68FDF7B1BD7B
:10610000C47901201A9F0120802B0408782B0408F1
:106110008C2B0408AC2A0120589F01201F85EB51CD
:10612000676666665E790120805C012078790120CF
:10613000FC5C012089B5F8142C770120DFF87893F6
:1061400008229FEDCD8A0DF14808B9F9023007EE1B
:10615000903ACA4BF8EEE77A03F8401C03F83F2C5C
:10616000A3F13D011E220B9367EE887A48F8201DAB
:1061700003F83E2C4046FDEEE77ACDED027ABDF8FD
:106180000810FCF72DFFB9F90030404607EE903AB1
:10619000F8EEE77A67EE887AFDEEE77ACDED027ADF
:1061A000BDF80810FCF71CFFB9F90430404607EEB3
:1061B000903AF8EEE77A67EE887AFDEEE77ACDED71
:1061C000027ABDF80810FCF70BFF404618F004FEF9
:1061D000FDF73ABEA94B00222121A3F14009A3F10A
:1061E0003D0A03F8402C89F8021089F801200B932E
:1061F000CDF828A01BF0D4F8A14B0028A14A1B8899
:1062000018BF4FF00308A04904BF4FF0040811461F
:10621000580500F19581DA0700F19C81980702D5B5
:106220004FF0030899494246994827F043FF0AEB8B
:106230000803984A0021013312A80AF808109A1A94
:1062400040F8203D89F8012018F0C6FDFDF702BE98
:106250008A4A4FF000090DF148084FF00A0C4FF040
:10626000080EA2F13D008C4902F8409CDFF83892FC
:1062700048F8200D404602F83FCC02F83EEC098871
:106280000B92FCF7ADFED9F8003040468349DA178F
:1062900081FB0313C2EBA30399B2FCF7A1FED9F86B
:1062A000089008F0EBFB0A9B4FEA194103F1010E3D
:1062B0004FEA1922CDF828E019700A9B591C0A915F
:1062C0001A700A9B5A1C0A9283F800900A9B5A1C67
:1062D0000A921870404618F07FFDFDF7B8BD4FF0E8
:1062E00001096F4FFEF78AB85FFA8BF018F0C0FC17
:1062F0004FEA1B2018F0BCFCFFF7CABA9978184681
:1063000003930DF015F900287FF44CAB6249654FFB
:10631000654A0988654C9368F961DFF8A0911168B6
:10632000B4F86221F863C7F86CB0FB64F962D9F87D
:106330000000FA65F1F7D9FE834600287DF4F6AC3B
:106340005146D9F80000FBF779FC94F86421039BCF
:106350000421642ADB7887F87410059340F02781C4
:1063600094F86531072B524B08BF84F865B194F857
:106370006521039307EB021A0692DAF804B0584637
:1063800026F0F4FCDAF808305FFA80FA1846049335
:1063900026F0ECFC5946069A5FFA80FB444B22F04B
:1063A0000F000AEB0B0E02F00F0298720EF1080EAE
:1063B0000BEBCA005A7383F807E05246987303F157
:1063C0000F0027F077FE049B0AF109005A46194690
:1063D000384B184427F06EFE3549CB7903F1010A9A
:1063E000F3B103F1FF3CC81D0023DFF8D4E05FFAEE
:1063F0008CFC0CF1080C8C4410F8012B5A4084459D
:106400004FEA82034FEAD20183EA420301F0180106
:1064100083EA02034EFA01F283EA0203DBB2EBD114
:10642000244A05980AF8023027F020FE94F86531D6
:106430000022013384F8642184F86531039BDDF880
:106440000CA09B785BB11AF806100136D9F8000051
:10645000FBF708FC9AF80230F6B2B342F3D894F88E
:1064600064310322013387F8742088F8002084F80F
:106470006431FFF7B1B800BF58A08B41C479012047
:106480005C7901205C2B0408642B0408742B04083D
:106490008779012085790120D481012067666666AD
:1064A000589F01200C0001202C770120AC2A0120EC
:1064B000709F0120769F0120087901207C540120E3
:1064C0000007090E8C4B8D4A1B88927903EB8303DE
:1064D00003EB83039F00BFB2002A00F00681884BC4
:1064E0001B680FFA83FA08F0C9FA40B2FDF776BDCF
:1064F00019469E469A469B460493FDF76BBE242799
:10650000FFF7C9BA4FF47A71B7E508F0B7FA18F097
:10651000AFFB002018F0ACFBFFF74AB9D8F8003009
:106520005E209847D8F80030392098475FFA89F004
:1065300018F09EFB4FEA192018F09AFBFFF731B9CB
:106540004FF003086F496EE60021FFF7B2BB10273A
:10655000FFF7A1BA4FF004086B4964E66B4B1B6868
:106560009A067DF57AAB98F80030002B7DF490AB5D
:10657000674F2D22674B84F840213B60BDE5202703
:10658000FFF789BA0827FFF786BA5D4B07466420F4
:10659000B3F900A0FDF722BD1946FDF71BBE194651
:1065A0009E469A469B4604931F46FDF713BE97F8F6
:1065B0007520130701D10132D2B2072A564B28BFEA
:1065C00001221946039300234FEA021B01F10D003B
:1065D0008B7207EB0B035FFA8BF193F810E04F4BD4
:1065E00004917344197A049B012900F1010A43EADA
:1065F0000E0E07EB0B0380F800E0DB6810D9A1F169
:10660000020E51465FFA8EFE0EF1020C604401F854
:10661000013B81424FEA1323F9D10EF1010EF244FE
:10662000BB44013223F060030AF101009BF8111012
:10663000D2B20B43082A8AF8003059D004994FEAA5
:10664000021B374B01F1100E07EB0B0CC31A5FFA5C
:106650008EF19CF810E0049130497144097A03EB03
:10666000010CBCF1130FBEDDDBB20398DFF8B8C03C
:10667000991DC9B241F0400E01F1010A80F807E00E
:10668000E1B105330CF1010E0021DBB2083300EB60
:10669000030B1EF8010B4840F3454FEA80014FEA17
:1066A000D00381EA400103F0180381EA00011D488C
:1066B00040FA03F381EA0301C9B2EAD105980AF866
:1066C0000C1087F8752027F0D1FCB7E619469E46D6
:1066D000FDF780BD19469E469A46FDF77BBD1946DB
:1066E0009E469A469B46FDF775BD4FF0FF33F8E690
:1066F0000B4BC31AB8E700BFD4810120F478012006
:106700002C770120682B04086C2B040804790120E5
:1067100078790120285D0120709F0120A8F70308E7
:106720007D9F01200007090E769F0120F8B5554B8B
:106730001B681C0700D4F8BD534C0746534E544DFC
:1067400004F53171736830469847B4F9C622B4F93C
:10675000C8322846B4F9C4E2317F6A60AB60C5F83C
:1067600000E014F00DFF4B4A137859073ED4D4F8DB
:10677000CC02494B1B7883B1484B2968B3F90A20F6
:10678000B3F90CE0B3F90E60891AAB686A689B1B19
:106790002960A2EB0E02AB606A600028CBD0381AE9
:1067A0003F4B984242D9B4F9D0220021B4F9D832F3
:1067B000B4F9DA029B18C4F8CC12384948BF013347
:1067C0005A10B4F9D2321B184A81B4F9DC0248BF1E
:1067D00001335A10B4F9D4321B188A8148BF0133EF
:1067E0005B10CB81BDE8F840FAF778B823F00403DA
:1067F0002C4E4FF0000EB5F9001013703846B5F965
:106800000420B5F90830C4F8CC72C6F800E0A6F848
:1068100004E0A4F8D012A4F8D812A4F8D222A4F864
:10682000DA22A4F8D432A4F8DC32A2E70020FBF785
:1068300033FA2B68B4F9D0229342B4F9D822B8BF06
:10684000A4F8D0329342B4F9D222C8BFA4F8D83207
:106850006B689342B4F9DA22B8BFA4F8D2329342FB
:10686000B4F9D422C8BFA4F8DA32AB689A42B4F9BA
:10687000DC22C8BFA4F8D4329A42BFF65CAFA4F8B9
:10688000DC32F8BD04790120AC2A012070710120AE
:10689000187101205E79012094710120E0700120BF
:1068A0007FC3C901EA700120B0F908302DE9F04F2B
:1068B000DDB291B00C460B81442D00F0D882064623
:1068C00043D9812D00F00A8200F29A80542D00F005
:1068D000CE8040F2F2816E2D00F09782802D40F044
:1068E0002481C14B93F8009009F1020919F0FF09C6
:1068F00000F09A80BD4B0A25BD4F994403F1010871
:10690000BC4EDFF82CA317E0322D00F0E582A5F194
:106910003C00C0B2132840F2E78200232268C14540
:1069200002F1010121601570226802F1010121606C
:10693000137079D018F8015B0A2DE5D1BAF8003050
:10694000FF2BA8BFFF23DBB2E8E7052D00F07D8217
:106950001FD8022D00F0838040F29B81032D00F0B0
:106960004482042D40F0E1802A46A3492046FCF7EA
:1069700017FB00212046FCF757FB2168022001236A
:10698000CD181A46256008701846628111B0BDE81E
:10699000F08F242D61D040F20381282D00F0E78193
:1069A000382D40F0C2800A68012005270A261318F6
:1069B0000025924923600346107020681A4600EBB8
:1069C000030EC4F800E007702068C718276006703F
:1069D0002068C6182660057020680D78C6182660E5
:1069E000057020684D78C618266005702068897883
:1069F000C518256001701846628111B0BDE8F08F9E
:106A0000A02D18D040F21681B82D00F0EC81FE2D9B
:106A100040F08B807A4D05F1080635F8021B2046C0
:106A2000FCF702FBAE42F8D101231A4618466281F8
:106A300011B0BDE8F08F734B08461968FCF7DEFA19
:106A4000714B20461968FCF7D9FA704B196820463B
:106A5000FCF7D4FA01231A46E8E76D4BF6E7042267
:106A60006C492046FCF79CFA01231A46C3E70B68E1
:106A70001121694A20465D1C684F256007F14E06CA
:106A80001970BD1E23681278591C21601A70236882
:106A900097F85520591C21601A70236897F85420E4
:106AA000591C21601A70B7F85010FCF7BDFA236822
:106AB0000021282203F1010E2046C4F800E01970DD
:106AC0002368591C21601A70B7F85210FCF7ACFA11
:106AD00035F8021F2046FCF7A7FAAE42F8D122682B
:106AE0000D214F4B501C5D1820601170226813F867
:106AF000011F501C9D4220601170F7D123680222B3
:106B00002046591C21601A70B7F85610FCF78CFA11
:106B1000B7F858102046FCF787FAB7F85A10204605
:106B2000FCF782FA01231A4665E72146284606F05B
:106B300073FB00287FF478AF742D00F0C480772DAC
:106B40000AD1336872689A4240F09D810146354A05
:106B5000204625F0D3FB67E7762D00F09881392D8C
:106B6000376800F0598200F21982212D01F07882F5
:106B7000292D40F063827B1C33603B780A2B01F0A7
:106B8000C082502B41F04880274D3046FCF7F6F983
:106B900028803046FCF7F2F9012368801A462AE77C
:106BA000202DC2D10B680846204D591C6A782160FF
:106BB0001A7023682A78591C21601A702368AA78F1
:106BC000591C21601A702989FCF72EFA21680123CB
:106BD0006879CE181A46266008702168A879CD1801
:106BE0002560087007E700BF7CA20120E4F70308D6
:106BF000676666662C3001201A9F0120C955012066
:106C0000CC800120107AF01F147AF01F187AF01F40
:106C100050570120F42B040804890120FE54012060
:106C20005B55012089C1030814300120F47801204C
:106C300054300120822D7FF478AF0B680846B74AA4
:106C40005E1CB74D1178B74A266019701189FCF7A0
:106C5000EBF9B54B226820461B88511CFF2B2160A5
:106C6000A8BFFF231370A96881F3100189B2FCF754
:106C7000DBF92968204601F30F0189B2FCF7D4F94A
:106C80002168AA4A01231078CD181A462560087099
:106C9000B1E6012D7FF449AF096800262B46252077
:106CA0004F1C2A4627600E7021684E1C26600D700E
:106CB00021684D1C256008709DE6522D7FF435AF8C
:106CC000216800205BE6336872689A4240F0D78002
:106CD0000146974A204625F011FBA5E6954B1E7804
:106CE000033616F0FF063FF49FAE934B4FF00A08B1
:106CF000924F1E4403F1010920E0B8F1500F00F05B
:106D0000F180B8F1320F00F00481A8F13C00C0B26C
:106D1000132840F22B8100252946236820465A1C5F
:106D2000226083F80080FCF77FF929462046FCF7B3
:106D30007BF94E453FF478AE19F8018BB8F10A0F94
:106D4000DBD17F498B684FF6FF72096803EB830341
:106D500091424FEA4305A8BF1146954221EAE171ED
:106D6000A8BF154689B225EAE575ADB2D5E70B682F
:106D7000022101250627581C0A22DFF8EC81206039
:106D80002046197023686F4E591921601F702368BF
:106D9000591921601A7023685A1922601D70B8F8B9
:106DA0000010FCF741F9B8F802102046FCF73CF956
:106DB00023685021002203EB050E2046C4F800E0B2
:106DC0001F7023685F1927601970236859192160A3
:106DD0001A703188FCF728F971882046FCF724F9ED
:106DE0002B462A4607E6584B30E609680123002067
:106DF000CE181A4626600D702168CE1826600D70D8
:106E00002168CD1825600870F5E5474B08460A68EB
:106E10001B88511C424DFF2B2160A8BFFF2313701C
:106E2000A96881F3100189B2FCF7FEF8474B2046B0
:106E30001988FCF7F9F82968204601F30F0189B297
:106E4000FCF7F2F801231A46D5E50B22404920460B
:106E5000FCF7A6F808223F492046FCF7A1F80722D4
:106E60003D492046FCF79CF801231A46C3E5002A59
:106E70003FF4DAAD3949012311601A46BBE55A1CCB
:106E80003260197825E75A1C326019785FE633685A
:106E90005A1C32601B78002B01F00281102B01F08C
:106EA0002B8105462E4E014622682046571C27603E
:106EB0001370FCF7A3F829462046FCF79FF8B16849
:106EC0002046FCF79BF820460021FCF7ADF8002196
:106ED0002046FCF7A9F8F3E63388FF2BA8BFFF2371
:106EE000DBB21BE51F492DE71BF048FE00283FF4ED
:106EF00014AD03780A2B4FD8B0F9023087FB031288
:106F0000DB17C3EBA2039BB2FF2BA8BFFF23DBB2AF
:106F100004E57B684FF6FF72396817E7EA810120C4
:106F20002C770120F4780120D48101207D5C0120A0
:106F300095C103087CA20120F4F703082430012046
:106F4000E02F012014300120A85101207A5C01209B
:106F5000FC2B0408082C0408142C04080DD201088A
:106F6000902D012018300120C07001201BF006FE7A
:106F700000283FF4D0AE03780A2B3FF6CCAEB0F930
:106F80000430B0F9061003EB830321EAE17183F3C7
:106F9000500589B2ADB2C0E60023B8E7552D15D033
:106FA000572D4BD17B1C0DF1FF32336017F8370B97
:106FB000013333609F4213F8011C02F8011FF7D11F
:106FC0006946F5F733FA01231A4614E57B1C336052
:106FD0003D78FF2D01F0E480FE2D01F0A6803046C3
:106FE000FBF7CCFF96E80C009B1A002B41F37A804C
:106FF000531C33601378002B41F074800C2D01F288
